:020000040000FA
:1000000000F80202F13A0000DD13000011150000B3
:1000100000000000000000000000000000000000E0
:1000200000000000F004010038050100DD130000AD
:100030000000000000000000DD130000613D000032
:10004000ED0F0000DD130000DD130000153B000084
:100050000916000065350000B5120000A914000063
:10006000C10C0000BD0B0000DD130000E113000017
:10007000DD15000011420000E13800005D3900008C
:10008000DD130000DD130000DD130000913D0000D2
:10009000C93D0000DD130000DD130000DD1300008A
:1000A000F13E0000FB3E0000EF0F00006D37000046
:1000B000DD130000CD35000000000000000000004E
:1000C0000348854600F04AFD00480047698D00005E
:1000D00000F8020230B50B46014600202022012420
:1000E00009E00D46D5409D4205D31D469540491B6C
:1000F0002546954040191546521E002DF1DC30BDB5
:1001000070B500242546002801DA01244042002968
:1001100001DA01254942FFF7DDFFAC4200D0404241
:10012000002C00D0494270BDF8B5002425460029B6
:1001300004DA0E46012400214042B141002B04DACA
:100140001E46002352420125B34100F003FC8C46B9
:1001500017461E46AC4203D0002540428D41AC46B6
:10016000002C02D0002657429E4161463A46334653
:1001700001B0F0BD03460B439B0703D009E008C95B
:10018000121F08C0042AFAD203E00B780370401C47
:10019000491C521EF9D27047D2B201E00270401CD5
:1001A000491EFBD270470022F6E710B513460A46F7
:1001B00004461946FFF7F0FF204610BDF8B5024689
:1001C0004A40D40F42004B0052085B089A4202D2C8
:1001D0000246084611464A0023D0C30D4A00DDB24C
:1001E000120EAD1A202D35DA49020126490AF6050C
:1001F0008A19002C00D0524220214F1B1146B940D1
:100200002A411018C20D9A4221D0002C17D0012D7E
:1002100008DCDA05801AD20F8019D207DBB200F0B1
:1002200005FCF8BDDA05801A012340001B06C01842
:1002300080185A428018CA0F1043490007E0490845
:10024000C2071143DA05801A80194008801800F0AF
:10025000E5FBF8BD61000122511A001BF7E70122FE
:10026000D2075140AAE70122D2075040A6E7024632
:1002700070B54A40D30FDB0740002DD04A002AD08A
:10028000010E140E000212020919400A520A8418C3
:10029000E50104465443000A120A2E045043A419EF
:1002A0004219200CC543AA18120C0125AD03521C9B
:1002B000521912047F39240400D0521C104301D477
:1002C0004000491EC2B20C06C0092018401C40085C
:1002D000802A02D003E0002070BD400840000029C1
:1002E00000DA0020184370BD70B502464A40D50FB1
:1002F00040004A00ED0740085208002814D0002AA8
:1003000012D0C40DD30D41020120C0055202490A8A
:10031000520AE41A091812187D34914201D3641C60
:1003200000E04900002C01DA002070BD002391425A
:1003300001D3891A0343400849000028F7D1002956
:100340000AD0914202D10121C90705E0914201D2B0
:10035000012101E00121C943E005C018401900F066
:100360005DFB70BDF0B507460846584087B0C00F2A
:10037000049048000E46590040084908BC1A8841BC
:1003800005D2384631461E4617460B4602465800EF
:10039000400810434CD0300D039040055900400DEB
:1003A000490D0590401A0290402872DA1803012185
:1003B000000B09050843019004980092002805D01D
:1003C00001995242002088410092019002984021F8
:1003D0000A1A0199009800F0EDFA05460C466B46A2
:1003E00007CB00F008FBC0197141039A0E0D0023E2
:1003F000D71756401A467A40164344D0049A002A2A
:100400002DD0029A012A039A15DC1205C01A9141D7
:1004100001263605001C7141D20F059ED2070093BC
:10042000019202962A46234600F046FB07B0F0BD33
:1004300038463146FAE71605224A0F46B218C01A66
:10044000B74101210905001C4F4100187F411146A9
:1004500018187941E20F10436D19644113E0E20767
:100460006D0815436408C2071443039A0126120558
:10047000C01A91413605001C7141CE074008304337
:100480004908C01851412A46234600F008FBCDE731
:10049000FFE7049801224000C117121A00238B4184
:1004A00004983146C417381AA141EEE730B401244C
:1004B000E407634030BC55E730B40124E4076140F1
:1004C00030BC4FE70000E0FFF0B51FB488B00B99D7
:1004D0000998002448400999C00F4900490809912A
:1004E000C0070B990090490049080B910999089899
:1004F000A64608431CD00B990A98084318D00998BF
:1005000001244000420D4800410D099824050003D4
:10051000000B204309900B980003000B20430B9025
:1005200050181C494018002201901446104605E05E
:10053000002001460DB0F0BD032801DA034600E0BB
:1005400003239C46C11A0AAE0AE05F0008ADED5BCA
:100550004F00F75B7D430027AA187C41491C5B1EB6
:100560006145F2DD410004AB5A522104120C0A43EA
:10057000240C401C0828DFDB01980290009970468B
:1005800001910090059B049A0799069800F094FA4F
:10059000D0E700000DFCFFFFF0B50C465C4085B0D5
:1005A000E40FE40703944C000026640859009446C5
:1005B000490802460296224321D062460A431ED0D1
:1005C0006200570D4A000E032303550D0124024615
:1005D0002C492405781B1B0B360B4018234326435C
:1005E000614600901C46501AB44103D30098401C49
:1005F000009002E0921800985B41002803DA002086
:10060000014605B0F0BD00200121090507468646D8
:1006100011E064461D46141BB54106D36546521BC6
:10062000B341744607430C43A646CD07400849082A
:10063000284392185B4105460D43EAD11046184302
:1006400013D06046194650407140084306D06046BA
:10065000101AB34106D20122002306E00022012332
:10066000DB0702E00122D2435310009874460105D3
:10067000381C6141029C039D0019694100F00FFA8A
:10068000BFE70000FD0300000122D207002800DBC5
:10069000101A002900DB511A814201D8012070474D
:1006A000002070470122D207002800DB101A002921
:1006B00000DB511A814201D20120704700207047AF
:1006C0000122D207002800DB101A002900DB511A92
:1006D000814201D301207047002070470122D207D8
:1006E000002800DB101A002900DB511A814201D9D1
:1006F00001207047002070470122D207002800DB4C
:10070000101A002900DB511A814201D101207047E3
:100710000020704710B5002904DB0C460121C907F1
:100720004042A141002B04DB1C460123DB0752425F
:10073000A341801A994101D3012010BD002010BDB2
:1007400010B5002904DB0C460121C9074042A14134
:10075000002B04DB1C460123DB075242A341101A85
:100760008B4101D3012010BD002010BDC217C10F65
:10077000504010B54018CA079623002100F056F9E2
:1007800010BD10B500229623114600F04FF910BDA0
:100790000EB5C217C10F5040CA0740180021054BC3
:1007A0000293019200910A460B4600F085F903B0CE
:1007B00000BD0000330400000EB505490291002180
:1007C00000910A460B46019100F076F903B000BD96
:1007D000330400003EB5CA17CB0F002450405140EF
:1007E000C0186141DA07054B02930192009422463A
:1007F000234600F061F903B030BD0000330400006F
:10080000C20F410040020123400ADB05D207090E56
:10081000C0187F2901DA00207047962903DC96234F
:10082000591AC84001E096398840002AF4D0404265
:100830007047410040020122400AD205090E80188B
:100840007F2901DA00207047962903DC9622511A8D
:10085000C8407047963988407047000070B5CD0F8A
:100860004A0009030123090B1B0519430B4BED0734
:100870000024520D9A4201DA002070BD074B343338
:100880009A4203DC9A1A00F0A5F802E004495118D4
:1008900088402C43F1D0404270BD0000FF030000AF
:1008A000CDFBFFFF70B5CD0F4A0009030123090BF3
:1008B0001B0519430D4BED070024520D9A4202DA35
:1008C0000020014670BD094B34339A4203DC9A1A6A
:1008D00000F080F803E0064BD21800F06BF82C43D0
:1008E000F0D0002240428A41114670BDFF03000053
:1008F000CDFBFFFFC20FD207400040080BD0C10D57
:100900000723DB01C91840020905400A1143C20848
:10091000400711437047002001467047CB0FDB07AB
:10092000490010B5490802460A4307D00A0D0724BA
:100930000903E401090B121B002A01DC002010BD91
:10094000C900440F0C43C100E018D205801800F024
:1009500065F810BDF0B51FB40646002082B005460C
:100960004024019100901BE0019922460F46304639
:1009700000F030F8049A059B801A994110D3104674
:100980001946224600F016F8361A8F410197224682
:1009900001200021009F00F00DF838184D41009013
:1009A0002046641E0028DFDC019B00982946324661
:1009B00007B0F0BD10B5202A04DB0146203A914073
:1009C000002010BD914020239C1A0346E3401943A8
:1009D000904010BD10B5202A04DB0846203AD040D4
:1009E000002110BD0B46D340D0402024A21A9140D4
:1009F0000843194610BD10B5202A06DBCB17084660
:100A0000203A1041C1170B4306E00B461341D0407A
:100A10002024A21A91400843194610BD002904DA87
:100A2000401C490001D140084000704770B40024C8
:100A3000050C05D11024000402D1002921D0112475
:100A4000050E01D100020834050F01D10001241D5B
:100A5000850F01D18000A41C002801DB4000641C2C
:100A6000002908D020252E1B0D46F540A14000D0BE
:100A700001212943084301061B1B000ADB1D02D587
:100A8000002070BC7047DB05181880180029F8DAC0
:100A9000401C4900F5D170BC40084000704710B5BB
:100AA000002B08DA0024401C614192185B411A4374
:100AB00001D14008400010BDF0B51FB482B005461A
:100AC0000C0003D008460DF0EFF902E00DF0ECF950
:100AD00020300246009021462846FFF76BFF049B1A
:100AE000059A04460F4618431143084314D018468C
:100AF00010431BD0009840210A1A18460599FFF7A9
:100B000069FF05460E46009A05990498FFF752FFC3
:100B1000084305D0012004E02046394607B0F0BD67
:100B20000020C11705430E432C43374300990E980C
:100B30006305401A7905E40A00220C43FD0A0A30D5
:100B400002D500200146E9E70105101969410C9C16
:100B50000D9D00196941FFF7A2FFDFE7064C012553
:100B6000064E05E0E36807CC2B430C3C9847103455
:100B7000B442F7D3FFF7A8FA3CFF00005CFF000087
:100B800030B58C180278401C13071B0F01D1037875
:100B9000401C120906D10278401C03E005780D7054
:100BA000401C491C5B1EF9D101E00B70491C521E10
:100BB000FBD1A142E6D3002030BD000080B584B057
:100BC0003B480068806A039003A8007880070028EB
:100BD00007D5FFE7364880210161006802214162A4
:100BE00063E003A800784007002807D5FFE73048F6
:100BF0008021016100680421416255E003A800786A
:100C0000C007002848D0FFE72948408B00280BD0B8
:100C1000FFE72748016809694269131D43611160B4
:100C2000418B491E4183FFE72148408B00280BD0B0
:100C3000FFE71F48C068002805D1FFE71C4800688F
:100C400001218160FFE726E01948C06801280CD126
:100C5000FFE7174801688A6801239A438A600168A0
:100C60004B62406803F096FDFFE7114801210161E6
:100C7000006A00280ED0FFE70D48016A4269008B28
:100C80008300D21A02901046029A01911146019BEC
:100C90009847FFE7FFE706E006480749074BFF22B2
:100CA00068320AF051FCFFE7FFE704B080BDC046A0
:100CB00010900102DBE90000F4E90000C0E9000047
:100CC00080B58CB000200B900AA908700B988001A9
:100CD00097490858806A09900B9880010858406825
:100CE0001321084013280AD1FFE70B98800190498F
:100CF0000858C068022108404008049002E0002023
:100D00000490FFE704980B998901894A51184861BA
:100D100009A80078800700280CD5FFE70B98800110
:100D2000834908580221816283488449844B854A5B
:100D30000AF00AFC09A80078400700280CD5FFE754
:100D40000B9880017A49085804218162794A02206F
:100D500003210BF0D9FAE7E009A80078C0070028C2
:100D600007D0FFE70B988001714908580121816283
:100D7000D9E009A800780007002850D5FFE70B98B4
:100D800080016B490818818E008F081A112803DB37
:100D9000FFE71020039008E00B98800164490818D1
:100DA000818E008F081A0390FFE703980AA9087044
:100DB0000878002829D0FFE708A800210170FFE784
:100DC00008A800780AA90978884214DAFFE70B9886
:100DD000800157490818C26A008F08AB1B78C018F9
:100DE000105C0B9A920189580874FFE70898401C20
:100DF00008A90870E4E70AA800780B9989014C4A11
:100E000051180A8F1018088708E00B98800148498C
:100E10000858416A082291434162FFE7FFE709A8A9
:100E20000078C00600284FD5FFE70B9880014049A5
:100E30000858C0681F2292021040800A0790079845
:100E40000B9A92018918CA8E498F511A884203D28F
:100E5000FFE70798029008E00B98800134490818D2
:100E6000C18E408F081A0290FFE702980AA9087005
:100E700006A800210170FFE706A800780AA90978F2
:100E8000884217DAFFE70B98800129490858007D4E
:100E900005AA107005980B9A920189180A6B498F60
:100EA00006AB1B78C9185054FFE70698401C06A9EA
:100EB0000870E1E70AA800780B9989011C4A5118CB
:100EC0004A8F10184887FFE70B98800118490818C7
:100ED000408F0B9A92018918C98E884222DBFFE766
:100EE0000B98800112490818012202610B988001B9
:100EF0000858002242620B9880010818C06B002835
:100F00000FD0FFE70B98800109490818C16B408F8B
:100F10000BAA01901046019A00911146009B984738
:100F2000FFE7FFE7FFE7FFE7FFE70CB080BDC04644
:100F30003490010203EA00002FEA000048EA0000B2
:100F40001AEA0000CE02000082B0214800210170A0
:100F500001910091FFE700981E490978884234DA30
:100F6000FFE70098A549085C012822DBFFE700980D
:100F7000A2490A5C521E0A5415480278521C02709B
:100F80000098085C01998900134A5050009840006D
:100F90001249085A01994900114A5052009880009C
:100FA0009749085801994A1C019289000D4A5050EE
:100FB000FFE707480178074A117000780A4908706E
:100FC000FFE70098401C0090C5E702B07047C0469C
:100FD000FCA60102C8A6010220BD0102CAA60102A8
:100FE000E8BD010284BD010248A5010270477047B7
:100FF000B0B59CB00A4603461B911A900020199088
:10100000FFE71998182800DDF5E019987B49085C7E
:10101000052800D0E4E0199880007B4908587B49F6
:101020000860199880007A4A10587A4A1060486817
:1010300009685368126818900846189909F0A4FCCA
:10104000754A5160106019988000744908587449B5
:10105000086019988000734B1858734B18605868D3
:101060001B684C68096817901846179B169119461B
:10107000169D15922A46234609F086FC6B4A51605C
:101080001060106851686A4B5960186015980168C3
:101090004468684D6C60296010685168149213931D
:1010A0001295FFF797FB644A126811901046109151
:1010B000FFF76EFB614A526A0F9010460E91FFF7E0
:1010C00019FC0F9A0D9010460E9B0C9119460D9A23
:1010D0000C9BFFF761FA0022594B0B9010460A91C6
:1010E00019460B9B09921A460A9BFFF7DFF9119AE2
:1010F00008901046109B07911946089A079BFFF726
:10110000E3F9FFF7CFFB149A516010601068516843
:10111000139B59601860159801684468129D6C60B3
:10112000296011680468091BCC0F09194910454C46
:1011300021602068FFF72CFB434A444BFFF7C4F9BA
:10114000434A5160106010685168424A424BFFF7B1
:10115000BBF9424B099AFFF7B7F9414A5160106059
:10116000106851683F4B099C06922246FFF7FAF837
:10117000069A51601060106851683B4B099AFFF75E
:10118000C9FA00282BD1FFE73548016840680022E2
:10119000364B059008460599FFF7D2FA00281ED174
:1011A000FFE72F4801684068199A5300304CE35E0E
:1011B0000490184603910292FFF7EAFA039A01900D
:1011C0001046049B00911946019A009BFFF7CAF84C
:1011D000FFF744FB02998A00094B9850FFE705E0AE
:1011E000199880000649074A0A50FFE7FFE7199857
:1011F000401C199005E71CB0B0BDC0468C9E010292
:1012000064A60102FFFF010058970102B8A701027E
:10121000F496010250A7010200BD0102E8B30102E9
:1012200068A701024CB40102A8A7010210BD010287
:1012300018BD010208BD0102E8A00102C0DF0000E4
:101240000000F03FE0B40102699006699006903F0B
:10125000D8B4010252257997532ED33F000059404C
:10126000809E010200003E40000024C000408F40EC
:10127000C096010284B00390029101A80021018070
:101280000091FFE70098029988420CD2FFE703988B
:101290000099405C0199081801A90880FFE70098AF
:1012A000401C0090EEE70198C04301A9088008881F
:1012B00004B0704780B586B00020059046490968A3
:1012C0000968049103A90870FFE703A800780728BC
:1012D0007FDCFFE7049803A909781031C840C007F4
:1012E00000280BD0FFE703A80078103001210A4640
:1012F0008240394800684260059127E0049803A9BC
:1013000009780831C840C00700280BD0FFE703A8C0
:1013100000780830012181402F4800684160022098
:10132000059012E0049803A90978C840C007002876
:101330000AD0FFE703A80078012181402648006811
:10134000416003200590FFE7FFE7FFE705980328CA
:1013500004D0FFE70598022818D1FFE703A800781A
:1013600080001D490818806800280CD0FFE703A8FA
:1013700001788900184A51188968059A0291114626
:10138000029A9047FFE7002005901CE0059801288D
:1013900018D1FFE703A8007880000F490818806A79
:1013A00000280CD0FFE703A8017889000A4A5118E9
:1013B000896A059A01911146019A9047FFE700203A
:1013C0000590FFE7FFE7FFE70398401C03A90870BB
:1013D0007BE706B080BDC04684920102FFE7FEE7CE
:1013E000B0B581B00020009000987C210A464243AD
:1013F00010488258D36920242343D361009A514373
:1014000040180069032813D1FFE700987C210A46A1
:1014100042430848825813680124A505AB43136072
:10142000009A51434018C16E62021143C166FFE742
:1014300001B0B0BDF492010283B0014601AA108050
:10144000684600220270FFE7684600781449097870
:10145000884214DAFFE701A8008869460978490044
:10146000104A515A884204D1FFE7009802A9087037
:1014700011E0FFE70098401C69460870E4E7684601
:10148000007807490978884205D1FFE704480078C9
:1014900002A90870FFE702A8007803B07047C046B1
:1014A000C8A60102CAA6010280B584B01748006828
:1014B000806B039000200290FFE70298112822D849
:1014C000FFE703980299C840C007002816D0FFE73D
:1014D000029880000D490818C06800280ED0FFE768
:1014E00002988100094A5118C968019288470298F8
:1014F00001218140019802689163FFE7FFE70298AC
:10150000401C0290D9E704B080BDC0467893010228
:1015100004217046084204D0EFF30983EFF30882F8
:1015200003E0EFF30883EFF309829BB004A8F0C057
:1015300044464D4656465F4608A8F0C01846F0C8D7
:101540006846F0C018690C90202018440D90586926
:101550000E9098690F90D8691090EFF31080119059
:10156000EFF314801290094908681390084908683D
:101570001490084908681590074908681690179351
:1015800018927046199068460AF04AF804ED00E097
:101590000CED00E010ED00E014ED00E080B502F08D
:1015A00033FC0B2006F010FB00280AD0FFE70A48A6
:1015B0000078002804D1FFE7074801210170FFE708
:1015C00009E005480078012804D1FFE7024800211E
:1015D0000170FFE7FFE780BDD494010280B50748A2
:1015E00001210170064802680A430260054802684A
:1015F000002A02D000200146904780BD4EA501027E
:101600001C10005050A50102F0B599B0F548017BBF
:10161000C67A427B0E92F44C221F1368F34A12687A
:10162000069242780C9202790592C76A04931F4091
:1016300001200F907A0200D5BCE03A0200D5BFE04D
:10164000FA0102D50F9802062260502508968A19E1
:101650001826BB0102D50F98430623604123079546
:1016600069430A96354655431426FC0210D50F9857
:10167000040538463746DC4E3460DA4CA469B4645D
:10168000D84CE4697464DA4C241D34603E46074645
:1016900090000B90D8040D90681809900E9B73432E
:1016A0000F988203B902D04D22D50F9841052960C9
:1016B000CC480E961646024681692965C16969655E
:1016C00009990D9801430898000108180B994018D2
:1016D000C018C849098892794A4380180A301C46C4
:1016E00004F0E0FC234632460E9EC04988672A601B
:1016F0000F98C404380300D52C60F80302D50F9866
:10170000000428600F984104B80300D5296038040C
:1017100000D4E4E1039402910E9308920D980B9982
:101720000C180A980C9941430C910F98C0030B9028
:10173000286007F055FC002801D004F095FC0C98B7
:10174000005B410B43D1099800190E994018059987
:10175000090140180E90E74D287B079B4343E97A27
:101760000A010D9C2243D21841188B00D2180A9B03
:101770004B43D1186A7B564389190E9E2A7910185B
:10178000DF4A12884243881816903068C000800DE6
:1017900010A9C882002511957079C0077ED110A8C4
:1017A0000F998182069C00940020E8A2049B0AF015
:1017B000ABFD78E00F98820522603A0200D43FE743
:1017C0000F98C2052260FA0100D53BE73DE70721EB
:1017D00049030840032149038842089A00D07EE16A
:1017E000069707F01FF90020169009901590C14C3C
:1017F000E07A217B08180A99414380000D9A104332
:101800004118627B0E9672438A186178A379079E0D
:101810007343D718FA683F26324063789A420C9790
:101820006ED105960A9A4A4380580F210A07024052
:101830000398401EC04B1B68DB09034098181090AA
:101840000F98C0020B90B868800767D42C46283CDC
:1018500009F00CFE05462068000609D5C320840166
:10186000786A400704D409F001FE401BA042F7D972
:1018700005980002B96849080140B34803688268C6
:10188000B868C40C20202040DB0700D095E000237E
:1018900010221D461C460E9E0B9FB1E010A88582AB
:1018A000B0681190069C701D924B1979E20707D120
:1018B000491C1971D97A1A798A4202D31D7100E044
:1018C000D97001784278120251188278120489186E
:1018D00003229143017035715878401C5870D87AB2
:1018E000197B08185978884200D85D70D879401E55
:1018F000D871596B002901D010A888477E4DEDE0C2
:1019000010A80B998182F86830406378009000201D
:101910007CA20F990AF0F8FC0E9E94E0388A874A60
:10192000024010A8C2822022BA5C9307DB0F3C68F9
:10193000C3720F9B1A4082726205D20C0D9B1A4330
:101940001692FA68130E0372BB69FC697C4D2D6810
:101950002D0C05745204920F427211931394654C2E
:10196000A07B002809980E9E0B9F5FD075480068E9
:10197000007A0328099859D00C98007D084009285E
:10198000099853D1C320840109F070FD05460C98D5
:10199000406A41070BD4594909680906890F06D1E5
:1019A00009F064FD401BA042F1D90C98406A410344
:1019B0000898884310A9888237E0D2070E9E0B9FB3
:1019C00003D108230022154619E00C9B9A68029C5B
:1019D000224211D19A68520C0224944300221346E9
:1019E00015460DE024A6010228A000503CA100509D
:1019F000FC1F000022A60102042500221346144603
:101A00000843104318432843204310A988823842D2
:101A10000BD10C9B198A494A0A4010A9CA8219683D
:101A20004905C90C0D9A11431691324C2921615C6C
:101A3000002908D03037B84205D010A90846113027
:101A4000123108F029FEE77A2A48047BE519294873
:101A500000790E9027484078401C2946FEF73AFB53
:101A600088000D9A1043189007996143380110437C
:101A700040182049497B4E4380191C216943401876
:101A80000E9909191B4B1E4A12884A438018179059
:101A9000099A0C998A60987B002800D04A6298794C
:101AA000401C9871187B99798142069F00D39A71E6
:101AB0005978491C5970D97A0818597888420E4DBE
:101AC00000D85A70187A401E18722820185C002816
:101AD00004D0996B002901D010A88847089A1742B2
:101AE00002D00F98000328601C480449486019B0D0
:101AF000F0BDC04624A6010228A000503CA1005021
:101B000022A60102485720455420696478202564A4
:101B100020616E6420455420696478202564206922
:101B20006E2052582064657363206D69736D617413
:101B300063680D0A0000000038200040FF03000029
:101B40009430004028940102604000404D41432001
:101B50004556542025782025780D0A00FFFFFF0305
:101B6000F0B5A5B01E460C9208910024239422A93A
:101B70000C8016A90C8024A909250D80598C0D9183
:101B8000FEF7A8FA2A99012900D0DFE0318901295E
:101B900000D0DBE0318C012900D0D7E00D9900297D
:101BA00000D1D3E0224607962C990B912B990691F0
:101BB00080B205900F9415A8058090000E900C99A6
:101BC0000C582E460025204629461746FEF75CFD98
:101BD0000028119636D12C200A97784308990818C6
:101BE00017A90A4668C868C2E8C8E8C2E8C8E8C2D7
:101BF000079F119880B280000E5822AD019523A84E
:101C0000009020463946059A069B03F066FF0F9820
:101C1000401C0F90288800282DD03B8A239913ACB4
:101C2000039416A8029014A8019015AE009617A868
:101C300024AA04F03FF92588308811900120149ED1
:101C40000A9A05E013A8058014952E4628463A46C0
:101C50000E9F51000B9B119C5C52591808830D84F8
:101C6000D81986600F981885521C0D9882426DD045
:101C700024A805889FE7099616A8002505801495D5
:101C800024A80688239812902F46109503E06D1C17
:101C9000A8B2B04213D8A8B2800017A90C582046A9
:101CA0001299FEF7FFFC0028F1D1002FEFD115A803
:101CB000058016A80127078014941094E7E715A85B
:101CC0000288B01A012805D115A80680099F14972B
:101CD000119628E010200799095E0129119221DB55
:101CE000551CA8B20C18109F0E9B099403E06D1CA4
:101CF000A8B2844218DDAAB2B242F8D8800017AA6E
:101D000010581090394634461E46FEF7BDFC334647
:101D10002646099C0028EAD115A80580109F149733
:101D20001195E4E7109F0E9B1C463E4638461299DB
:101D3000FEF7DAFAFEF764FD0546052800D305250F
:101D400013A8058001200A9A274682E725B0F0BD36
:101D5000F0B58BB00243159A149C139E2BD0054608
:101D600001A856C0129CD869196A09900A911E46AA
:101D70009F6B0123009309A807AA0146059306F06B
:101D8000B9F8716C3846FEF7AFFA0746E06A616B46
:101D9000FEF7AAFA002D069613D004461198019971
:101DA000012924D10921081A0421069A515E88428A
:101DB00029D16425B1E000203080207010700BB074
:101DC000F0BDB08800226425002829D00592694919
:101DD0003846FEF783FC0028049C039E6FD16649B9
:101DE0003846FEF77BFC00281DD05A2567E03C25CD
:101DF000082800D191E05F492046FEF76FFC0028DB
:101E000019D0502589E00A291DDB1D293BDC5949E1
:101E10003846FEF763FC0022002854D05A253AE0E9
:101E20003346049C39E055493846FEF757FC0028F4
:101E300021D0502543E050492046FEF74FFC0028B2
:101E40002ED0462569E03C25012866D04949204628
:101E5000FEF744FC0028D4D147492046FEF73EFC5B
:101E60000028EED145492046FEF738FC002854D121
:101E7000434920466EE042493846FEF72FFC0028D1
:101E80001CD128251BE03B493846FEF727FC0022E1
:101E9000002832D05025049C069B0299039E41E005
:101EA00036492046FEF71AFC002836D13449204630
:101EB000FEF714FC00282FD114252EE037250299B7
:101EC000059A069B2EE005922B493846FEF706FC44
:101ED000002896D129493846FEF700FC0028B0D1E9
:101EE00027493846FEF7FAFB0028049C069B029916
:101EF000039E059A3BD11E2514E005921E493846E3
:101F0000FEF7ECFB00289CD11C493846FEF7E6FBA7
:101F100000281DD03C2500E02325049C069B029947
:101F2000039E059A258032700020087030780028C2
:101F30000CD118681349FEF7C3FB002806D120888E
:101F4000102803D30F3820800BB0F0BD0BB0F0BDCC
:101F50000B493846FEF7C2FB0028049C069B0299F9
:101F6000039E059A01D11425DCE72325DAE72D2508
:101F7000D8E7C046CDCCCC3DCDCC4C3DCDCCCC3C37
:101F80000AD7233C0000204070B588B00C460646B6
:101F90004088002820D0FEF7F4FB059005A804A98E
:101FA00001252A4606F010FA3088B188081AFEF793
:101FB000DDFB0390049903A807AA2B4606F0C4F999
:101FC0005249079D2846FEF789FB002808D0BF200C
:101FD0000006206008B070BD0020206008B070BD11
:101FE0004B492846FEF75EFB002804D03F20000640
:101FF000206008B070BD47492846FEF76FFB0028F7
:1020000001D0002010E000212846FEF767FB0028E1
:1020100001D0022008E040492846FEF75FFB002877
:1020200001D0042000E0062001957F21C90502911E
:1020300080003A49091801A806AA022306F038F9D7
:102040000698206008B070BDF0B587B00C46054614
:102050004768002638463146FEF74EFB002802D07E
:10206000266007B0F0BD049704A803A901263246F4
:1020700006F0AAF9A8682968FEF7F1F8029003991A
:1020800002A806AA334606F05FF92049069D2846B5
:10209000FEF724FB002804D0BF200606266007B008
:1020A000F0BD1B492846FEF7FDFA002804D03F206A
:1020B0000606266007B0F0BD16492846FEF70EFB5F
:1020C000002801D0002010E000212846FEF706FB82
:1020D000002801D0022008E00F492846FEF7FEFA4A
:1020E000002801D0042000E0062000957F21C905CA
:1020F0000191800009490918684605AA022306F0E3
:10210000D7F8059E266007B0F0BDC046CDCC0C3F89
:10211000295C0FBFCDCC4C3ECDCC4CBE30940102DF
:10212000F0B587B00C4606467F270088002801D00E
:10213000FD0503E0B08800282ED0334DFEF721FBCB
:1021400003907088FEF71DFB049003A802A90126E6
:10215000324606F039F9029904A806AA334606F079
:10216000F3F82A49069E3046FEF7B8FA002802D056
:102170003F20010641E026493046FEF793FA002849
:1021800002D0BF20010638E022493046FEF7A6FA09
:10219000002805D0002024E00020206007B0F0BD1A
:1021A0001D493046FEF79AFA002801D0022018E0B7
:1021B0001A493046FEF792FA002801D0042010E0B8
:1021C00017493046FEF78AFA002801D0062008E0B9
:1021D00014493046FEF782FA002801D0082000E0BA
:1021E0000A200096F905019180000F4909186846F8
:1021F00005AA022306F05CF805992846FEF737F891
:10220000206007B0F0BDC046000080BF000038432A
:102210003333733F0000C842000070420000204288
:102220000000A0410000C04050940102F0B59DB0F4
:1022300015460B917F210391C9051C9102911B91B9
:1022400019A900248C80199418941794598C06911C
:10225000198C0F91DE8B998B0791997805911F88C6
:102260002B21CA432799914201DB7F0015E04022D0
:10227000D243914211DC4922D243914202DB7908D8
:10228000CF190AE05322D2439142EEDA5D22D243C3
:10229000914201DBBF0000E0FF000A971396269EE3
:1022A000597E00290BD0002132460F46D170917023
:1022B00051701170121D7F1C5C7EA742F6D30C93E7
:1022C00011952599149122990D91159041088C42F0
:1022D00011D2FD4A2346A00084583454270A451CD5
:1022E0007755250C871CF555240EC01C34545B1CF7
:1022F0009CB2A142EFD82398109001200990009041
:1023000030463146149A159F3B4605F001FE0D9864
:1023100000060890400E139D00D186E068000490EE
:10232000002F3FD0002210461146144606E01C46FE
:102330001146159F401C82B2BA420ED283B2AB4204
:10234000F8D09200149B9A5E0FB2BA42034600DCAA
:102350002346BA42EBDC0A46E9E7002F25D00022EB
:1023600010461146129206E012931146159F401C2A
:1023700082B2BA4214D283B2AB42F8D0A5B2AB4219
:102380000CD09200149B9A5E0FB2BA42034600DC56
:10239000129BBA42139DE7DC0A46E5E7139DE6E788
:1023A000129903E00024214600E0002112911098C8
:1023B0000183C4828582049FF057FEF7D7F9792103
:1023C000C9050E91FDF753FF1099C861099807439D
:1023D000F057FEF7CBF90E99FDF749FF109F3862D1
:1023E0002004C40B3057FEF7C1F90E99FDF73FFFEB
:1023F0007862601C3056FEF7B9F90E9C2146FDF755
:1024000036FFB86212980004C70BF057FEF7AEF91A
:102410002146FDF72CFF109CE062781C3056FEF739
:10242000A5F90E99FDF723FF2063119805800C98FC
:10243000407E410000278D4228463A46149E1ED316
:102440000A9880B28AB29300F45E84420BDA491C87
:102450008AB2AA42F6D9002728463A4681B2691ABA
:10246000012910D01BE0F018119B1980078808047F
:102470000FD0500040008019001F0288084681B22A
:10248000691A01290BD1A800301811990D8007880D
:1024900026E00020024681B2691A0129F3D00A9988
:1024A00089B2079B4B43BB421AD306998A4217D87D
:1024B0000599002914D0401C82B2891803E0401C01
:1024C00082B291420CD983B2AB42F8D89200B35E8B
:1024D000BCB2A342F3DDB218119B18801788EEE757
:1024E00012970B980580119800882B1A002B16DD87
:1024F00002210F9A1143032942D10E93411C421E1F
:1025000010B281420EDA0E98032824DB0C98808CDE
:10251000012820D019A818A9FFF736FD1FE00020D8
:1025200018902BE00026F443374608E0B8B240008C
:1025300019AD2B527F1C521C10B28142E3DB13B247
:10254000A3423346F2DD159B98423346EEDA800013
:10255000149B1B5AEAE719A818A9FFF7E1FD149E7E
:10256000139D0F9A012A13D0032A11D0022A04D1F5
:1025700011980088281A02280ADA0020179034E0FF
:10258000022A01D1022BB8DA00201890012AEBD1DF
:10259000681C691E0FB2B84208DA0C98808C0128BA
:1025A0001DD119A817A9FFF7BBFD1CE00022D343DA
:1025B000144608E0A5B26D0019AF7E53641C491C97
:1025C0000FB2B842E9DB0DB29D421646F2DD159D11
:1025D000AF421646EEDABD00149E765BEAE719A814
:1025E00017A9FFF7D1FC149E139D249F189C1799DF
:1025F0002046FDF734FE0F99012900D820463860A7
:102600000D98002800D1CBE011990888109FB8865A
:102610000888281AB880129880B2FEF7B2F879219B
:10262000CC052146FDF723FE2146FDF720FEB863C9
:10263000119F3888002849D081008919091F09880D
:10264000129C0C191599884203D280008019808849
:10265000041915984300534916AA304605F036FE72
:10266000169810994864FEF7E4F8A4B2A04201D18C
:102670004D480FE0001BFEF784F81C901CA81BA916
:10268000012205F0A1FE2046FEF77BF801461B98CB
:10269000FDF7EDFD109908603988491B4A1C92B27C
:1026A000032A02D20021159F17E009B20229159FC3
:1026B00012DB3F210906FEF711F8002802990CD120
:1026C0000998810709E0C046402100400020129C83
:1026D00015998842B9D3BCE734491098016108982C
:1026E000800E5DD0002F1CD00022114614461046EB
:1026F0004B1B1DB2ED135B196B40139D1BB2920077
:10270000B25E53431818A418491C8AB2BA42EFD3D8
:10271000FEF737F806462046FEF733F8002C03D1C3
:1027200000E000260398C0051C901CA81BA90125E9
:102730002A4605F049FE1B9C20463146FDF797FDD1
:10274000014610988160002F119422D00024274662
:10275000264613951291B8B2FEF713F81299FDF7B9
:102760007EFD0546A0001499085EFDF7FFFF0146B7
:102770001398C00785432846FDF779FD014630468A
:10278000FDF71CFD06467F1CBCB215988442E2D3BF
:1027900000E0002611983146FDF769FD1099C860E8
:1027A0001DB0F0BDE09E010200002041000040404D
:1027B000F0B58FB00692F74A09AF70CA70C770CAF9
:1027C00070C70328079320D88800F3A10858F6495A
:1027D000FDF7F4FC0446F549FDF7F0FC0D90F449D3
:1027E0002046FDF7EBFC0C90F2492046FDF7E6FC95
:1027F0000B90F1492046FDF7E1FC0A90EF49204695
:10280000FDF7DCFC0990EE4969E0042822D0062897
:1028100020D88800EBA10858EE49FDF7CFFC04460C
:10282000ED49FDF7CBFC0D90EC492046FDF7C6FCC9
:102830000C90EB492046FDF7C1FC0B90E94920467E
:10284000FDF7BCFC0A90E8492046FDF7B7FC09906B
:10285000FD4944E00838022821D88800FBA1085827
:10286000D149FDF7ABFC0446FC49FDF7A7FC0D90F0
:10287000FB492046FDF7A2FC0C90FF208105204675
:10288000FDF79CFC0B90F7492046FDF797FC0A905A
:10289000CA492046FDF792FC0990FE491FE08800D6
:1028A000F1A10858F449FDF789FC0446F349FDF706
:1028B00085FC0D90F2492046FDF780FC0C90F14913
:1028C0002046FDF77BFC0B90EF492046FDF776FC98
:1028D0000A90EE492046FDF771FC0990EC490094FE
:1028E0002046FDF76BFCEC4909680E90EB48046844
:1028F000EB4801684808EB4F05463D400022002D9B
:1029000008922DD0CA01120E07D0280CE90D12D161
:102910004000E649085AE6490AE0C903090E0CD00E
:10292000280AE90B10D14000E049085A8F2189009C
:102930004018E4300DE0DC490AE081B27F2905D877
:102940004800DA49085A04E0D94901E08F2189009A
:10295000401800B2FDF70AFFD649FDF788FC024691
:102960000292039507252606D34B1A68002A089879
:1029700040D0791C8A420BD21102090E13D0110CDF
:102980001F46D00D1FD14800C849085AC84907E062
:102990001F46110E002A13D44800C449085AC249E0
:1029A0004018E4301FE011041F46090E0ED0110A32
:1029B000D00B12D14800BD49085A8F218900EFE79A
:1029C000BE4808180FE0B84808180CE091B27F29FB
:1029D00006D84800B549085A05E0B548081802E08D
:1029E0008F218900501800B2FDF7C0FEB149FDF7F4
:1029F0003EFC3B460590159F2C40F50E5B69B049A7
:102A00001940089810D0DA02D20E34D0C80B3E21FB
:102A10000140A648405AA6494018E43000B2FDF7EC
:102A2000A5FEA449FDF723FC0490149E6800A5A10F
:102A3000085EFDF79BFE0146A00009AA1058FDF7AD
:102A4000BDFB0146B8B20128089F019102D1022CBA
:102A50000AD9A74F052C24D1189808900C2D20D8FE
:102A60000B2D16D3A44918E00027022C089718D084
:102A70008120C70515E01A04120E00D1CAE0080A29
:102A8000C90B00D0CDE040008849085A8F21890049
:102A9000C2E7092D00D2C7E096490898FDF78EFBE2
:102AA000089001200021B542034600D30B46052CB7
:102AB00000D308461799169A1A9C199D1843069B2D
:102AC000012B12D1079B402B22D1002840D0384641
:102AD000FDF774FB01460198FDF770FB0146009875
:102AE000FDF7BDFB059A04998AE0079B402B1FD197
:102AF000002838D03846FDF761FB01460198FDF704
:102B00005DFB01460098FDF7AAFB059A049977E062
:102B1000002833D03846FDF751FB01460198FDF7F8
:102B20004DFB01460098FDF79AFB059A049967E072
:102B300000285BD03846FDF741FB01460198FDF7C0
:102B40003DFB01460098FDF78AFB059A049957E082
:102B500002981146FDF783FB0399002900D16748CD
:102B6000059A04994CE002981146FDF778FB039909
:102B7000002900D16148059A049941E00298114664
:102B8000FDF76DFB0399002900D15C48059A049973
:102B900036E0C046F4DE0000000068C1000088C1D5
:102BA00066665EC1000084C1000084410000B4413B
:102BB00000004841000020400000F0C0000084C137
:102BC0000000F841333323C1000050C19A9929C154
:102BD0009A9949C19A9949413333CB416666764106
:102BE000CDCCAC40333393C09A9949C10298114679
:102BF000FDF735FB0399002900D14048059A049957
:102C000028601046FDF72BFB0899FDF728FB206094
:102C10000FB0F0BD99B27F2911D848002349085A56
:102C2000FCE623494018F9E6C12001060898FDF7A3
:102C3000C5FA0890062D00D933E7002030E78F2130
:102C400089005818EAE6C0463333F341000058C102
:102C50009A9961C19A9969C1000084C10000AC4190
:102C600000003841000008C1CDCC80C1CDCC88C166
:102C700033338FC1333397C133339741CDCC8C413C
:102C80003333F3409A9919C0666646C1333397C10E
:102C9000CDCCB4410000D4410C0000405030004085
:102CA00068400040FFFFFF007C080000D0E2000009
:102CB0005C050000919AF63C642000409C0B0000EB
:102CC000FFFF1F00FAFFFCFFFEFF000002000400F0
:102CD000060008000A000C000E001000120014008C
:102CE000160018001A001C001E00200022002400FC
:102CF000000080BF0000A0C0000040C00000DCC297
:102D0000F0B5FFB0ECB017460E460D900021E991EA
:102D1000E891DC91999198919791969114911391E2
:102D200012919AA8F49DF39CF29A002E00D1E6E14C
:102D30000B938030F09B1180099529602546DBAC10
:102D4000218095AC21800C952980DA917F24E405BF
:102D5000B994B894B794B694B594B494B394B29427
:102D6000B194B094AF94AE94AD94AC94AB94AA9457
:102D7000A994A894A794A694A594A494A394A29487
:102D8000A194A0949F949E949D949C949B949A94B7
:102D9000046644668466C466046744678467C467DF
:102DA000046444648464C464046544658465C465DF
:102DB000046244628462C462046344638463C463DF
:102DC000046044608460C460046144618461C461DF
:102DD000B0090B250B2800D3AE011095012B0B9DDC
:102DE00000D070E12B89012B00D06CE1298C0029E7
:102DF0000E9200D18BE16B8C002B00D1FAE1AA8CF2
:102E00003021695C002900D188E10892109F5F435E
:102E10001196304639460F93FDF75CF90590FDF7A2
:102E2000A5FC01462046FDF75FFA8321C905FDF7A1
:102E30001EFA064696A8021D119887420A9200D8EB
:102E400079E155A811909AA9069196AF15463A4690
:102E5000059C234605F02CFA15A80F9006992A46E2
:102E6000234605F025FA02230D93384631463A46AB
:102E700005F06AFA012308930093E8AA10923846F5
:102E8000394605F037F8E898DD901198069D2946F7
:102E90003A46234605F00CFA0F9829460A9A23462B
:102EA00005F006FA384631463A460D9B05F04CFAD5
:102EB000089B009338463946109A05F01BF8E898AD
:102EC000DE9011982C4629463A46059D2B4605F082
:102ED000EFF90F9821460A9A2C462B4605F0E8F99F
:102EE000384631463A460D9B05F02EFA089B009372
:102EF00038463946109A04F0FDFFE898DF901198A3
:102F0000069D29463A46234605F0D2F90F982946F0
:102F10000A9A2346254605F0CBF9384631463A460B
:102F20000D9B05F011FA089B009338463946109A1C
:102F300004F0E0FFE898E0901198069C21463A469C
:102F40002B4605F0B5F90F9821460A9A2C462B46D8
:102F500005F0AEF9384631463A460D9B05F0F4F9D6
:102F6000089B009338463946109A04F0C3FFE8984E
:102F7000E1901198069D29463A46234605F098F9B6
:102F80000F9829460A9A2346254605F091F93846B6
:102F900031463A460D9B05F0D7F9089B0093384619
:102FA0003946109A04F0A6FFE898E2901198069C22
:102FB00021463A462B4605F07BF90F9821460A9A9E
:102FC0002B4605F075F9384631463A460D9B05F01B
:102FD000BBF9089B009338463946109A04F08AFFE3
:102FE000E898E390119821463A462B4605F060F99F
:102FF0000F9821460A9A2B462C4605F059F9384677
:1030000031463A460D9B05F09FF9089B00933846E0
:103010003946109A04F06EFFE898E4901198069DE6
:1030200029463A46234605F043F90F9829460A9A5D
:103030002546234605F03CF9384631463A460D9B75
:1030400005F082F9089B009338463946109A04F03F
:1030500051FFE898E5901198069C21463A462B4688
:1030600005F026F90F9821460A9A2B4605F020F91B
:10307000384631463A460D9B05F066F9089B0093A9
:1030800038463946109A04F035FFE898E6901198D2
:1030900021463A462B4605F00BF90F9821460A9A2D
:1030A0002B4605F005F9384631463A460D9B05F0AA
:1030B0004BF9089B009338463946109A04F01AFFE2
:1030C000E898E7907AE010880C9A1080999198918E
:1030D000DA9E08460F46099DF59CFDF7C0F828606A
:1030E000DC9827606060A6600C34DDA80EC80EC4B2
:1030F0002EC82EC42EC82EC47FB06CB0F0BDFF20E9
:1031000010800021296020807FB06CB0F0BD0022CB
:1031100001233021695C002900D076E6DDAA1ACFB0
:103120001AC23ACF3AC23ACF3AC20B213046FCF724
:10313000D1FF054642E000200690059D0796089FB6
:103140001190069801460D9C0F9A4A43D219109B84
:103150005A43119BD218D200A35889002E4655AD70
:103160006B503546121DA25815AB5A50401C01B287
:103170008E42E9DC55A89AAE96AC314622462B46E3
:1031800005F096F815A831460A9A2B4605F090F8F6
:10319000022320460799224605F0D6F80123009322
:1031A000E8AA2046214604F0A5FE119B9800DDA95F
:1031B000E89A0A505B1C0B2B1846C1D1F19EDDA882
:1031C0009AA9DCAA0B2305F073F809210E980F9138
:1031D00001800B98C168DC9C2046FDF748F8014649
:1031E000A8B2E69F0F281BD808280DD30846FCF785
:1031F000E5FF14E0FF2010800021099A11600C996E
:1032000008807FB06CB0F0BD042803D3812208464B
:10321000D10502E0412208461106FDF728F80146D3
:103220002B20C04386420D9704DB0846FCF7C6FFFF
:10323000014603E04020C043864244DD0E9A0C9CC8
:103240000B98408A002811D00B98038A95A8039008
:10325000DBA80290DAA801900094DDA80D4602F0E8
:1032600029FE29462488DA9E099D68E011910F986D
:10327000208000273D46109705E00E9804887F1CAB
:10328000B8B2A04211D8B8B28000DDA90C582046CF
:103290001199FDF707FA0028EFD1002DEDD10C9818
:1032A000078001250F971094E7E7DBA805800F9AA8
:1032B00090B2201A012811D10C9804800D9FDA9742
:1032C0003E46099D3AE04920C043864200DA8BE041
:1032D000FF2208469105FCF7CAFFA9E710200B99C9
:1032E0000E5E012E00DA90E0551CABB21846A1B27A
:1032F000AAB28A4217D805E00E990C88A1B2AAB2E8
:103300008A4210D88000DDA90C58204610991F462B
:10331000FDF7BAF93B46002805D10C9805800B98BB
:10332000068A0F95109430B2C1186D1CA8B2814264
:10333000E2DC109EDA960F9C099D0D9F1199304694
:10334000FCF7D2FFFDF75CFA052800D3052095A90C
:103350000880A0B20E990988814218D9401C611ECC
:103360000CB2A04218DA12A898A9FEF76DFE0E98CA
:103370000188481C491E0CB2A04221DA12A899A962
:10338000FEF762FE99999898099D0D9FA4E6002189
:103390009891999108469FE60022134608E09CB256
:1033A000A40012AF3D515B1C491C0CB2A042DADBF9
:1033B0008DB20A2D1546F2D8A400DDAD2D59EEE7E9
:1033C0000022134608E09CB2A40012AF3D515B1CE2
:1033D000491C0CB2A042D1DB8DB20A2D1546F2D8A1
:1033E000A400DDAD2D59EEE75320C043864200DB3B
:1033F0001BE70E460B9881692046FDF745F900282A
:103400000C9C08D10B98808B07E01446099D0D9FFA
:103410001199109E93E70B98C08BFDF7B2F9014606
:103420003046FCF724FF119021E70000F0B58BB087
:103430001C4609930E46034600200A904048008827
:10344000224F05970AA9049103940292109C0194BB
:10345000012500950B21414389B230331C4A304687
:10346000FFF74EFC3868079078680890B8680690B7
:1034700033480088334F009501940297324E30361E
:103480003249334A3346FEF76BFB0698F8620798D9
:10349000386308987863099800882E4905912E4969
:1034A00004912E4903910297019000962C4B2846D7
:1034B00029462A46FEF74CFC432001060A98FCF7F1
:1034C000D6FEFDF79DF90BB0F0BDC046A89E0102E7
:1034D000A0B30102F0B589B00F9F0E9C002815D053
:1034E0001098079016480088164E01250095019106
:1034F00002960893144B30331449154AFEF730FBFB
:10350000089BF76207983063746303E00D484763D4
:10351000C462002518880F4905910F4904910F498D
:103520000391084902910190074830300090012131
:103530000B4B28460A46FEF70BFC09B0F0BDC0460F
:1035400046A5010264A80102BC970102109601027F
:1035500000A701029C9B010244A50102F0A4010204
:10356000F8A4010280B5124801681F220A400260D7
:1035700003200840022812D10E480268D30D02D061
:10358000FF231B06D2180C4B1A600C4A12680C4B16
:103590001A6080680B4A1080000C0B4A10801A4891
:1035A0008268002A02D082680020904780BDC04611
:1035B000742000406440004014A7010278300040AD
:1035C00018A70102369801025CA8010280B50D48D7
:1035D000016889070FD5052101600B48C1780029D2
:1035E00008D00021C170C168002903D0C2684168B9
:1035F0000020904780BD054805A10B4A0BA307F0AA
:10360000A3FFC0462C040040189401024CF30000B4
:103610005048595F54494D45525F49525148616E77
:10362000646C6572000000008D0A0000556E6578BC
:1036300070656374656420696E7465727275707408
:103640000000000080B586B00590049104983149CF
:103650004018039003A80078800700282BD1FFE7CB
:103660000598002827D0FFE70598022823D8FFE710
:1036700003983F2189064018000B02900298059993
:103680004018802816D8FFE700200190FFE7019836
:10369000059988420DD2FFE71F480068029903F0A0
:1036A000D9FDFFE70198401C01900298401C029050
:1036B000EDE7FFE7FFE706B080BDC04680B582B00A
:1036C000019007480068002103F058FA002804D14F
:1036D000FFE7114800210160FFE702B080BDC0464E
:1036E0009895010280B584B00390029101920398ED
:1036F0000299FF22FCF750FD0198064940180090FE
:10370000054800680099039A029B03F0C5FB04B0CA
:1037100080BDC04600E00704709301020120000351
:10372000704701204003704780B50A480A4901608C
:1037300005F0B2FB0948817A094A11708188094A6B
:103740001180C1887D20C000FCF7C4FC06490870C8
:1037500080BDC04600960102DD3F0000ECA00102E2
:1037600045A50102789E0102E4B3010280B590B044
:1037700000200F900F981821414398484058C06B83
:103780000001800F002800D09EE00F9818210A4603
:10379000424392488258D26B07231B071A40120FEC
:1037A000082393400E930F9A0B465343C258D26B93
:1037B000464B1A400D92022203901046029101924C
:1037C00001F0FEFF0C900E980C994143C80B0B9032
:1037D0000B980D99411A3E4A4A43009010460099B1
:1037E000FCF78EFC0A900A9807F082FD0A9B394A82
:1037F0000321019808F088FD0F99029A4A43039922
:103800008A18D28A002A0BD1FFE70F98182141436A
:10381000724840580021C160112001F08BFF52E036
:103820000C9840010D99FCF755FC0E994143099104
:1038300009984009089009981F21084005A90870B7
:10384000087810280CDBFFE706A801210170059815
:103850002021081A05A908700898401C089003E068
:1038600006A800210170FFE708981B49884208D389
:10387000FFE707A800210170089818494018049034
:1038800007E007A80121017008981349081A04905D
:10389000FFE70798C007C00B0499490189B2401897
:1038A0000699C907C90E401805A909780F221140C9
:1038B00040180121490440180F9918224A434749EA
:1038C00089580863FFE7FFE710B080BDFFFF1F00C6
:1038D00040420F0052ED0000FF7F00000180FFFF1B
:1038E00080B588B0002007900798182141433B48D5
:1038F00040588069C00700282ED0FFE7079818219C
:103900000A464243354882580123D361079A5143FE
:103910004018006900281ED0FFE7079818210A46C2
:1039200042432E48825812680492049A05AB0390D1
:10393000104602911946019307F060F90798029921
:1039400041430398411809690022019800911146EA
:10395000009A9047FFE7FFE708B080BD10B588B038
:10396000002007900798182141431C484058006CDC
:103970008007002830D5FFE7079818210A46424300
:1039800016488258136C012423431364079A514349
:103990004018C06800281ED0FFE7079818210A4683
:1039A00042430E48825812680492049A05AB039071
:1039B000104602911946019307F020F907980299E1
:1039C000414303984118C9680022019800911146AB
:1039D000009A9047FFE7FFE708B010BDA8940102E6
:1039E00010B586B000200590FFE7059839490978A1
:1039F000491E88424BDAFFE700200490FFE7049855
:103A000034490978491E88423CDAFFE7049880006F
:103A100033490A180858516888422EDDFFE7049898
:103A200080002F4908580390049840002A4A105AF1
:103A30000290049880002C4B185801900498800044
:103A40000C1864680C5004984000141864881452D0
:103A5000049880001C1864681C500398049CA400FF
:103A600061184860029804994900891848800198B3
:103A700004998900C9184860FFE7FFE70498401CD3
:103A80000490BCE7FFE70598401C0590ADE70020D7
:103A90000090FFE700980F490978884217DAFFE79E
:103AA000009840000C49095A0C4A115200988000B5
:103AB0000B4909580B4A1150009881000A4A515885
:103AC0000A4A1154FFE70098401C0090E2E706B054
:103AD00010BDC04648A50102E8BD0102CAA6010208
:103AE00084BD010264A6010220BD01028C9E010278
:103AF00007480168032291430160016801221143D4
:103B0000016009F087FD00F03BF907F01DFCC0469D
:103B10002800004080B584B019480068039003A8CD
:103B2000C0780006002822D5FFE71948006803285E
:103B300004D1FFE712480421016006E01448006840
:103B4000042108430E490860FFE711480069002876
:103B50000CD0FFE70E480169406800220290104631
:103B6000029A01911146019B9847FFE705E005483D
:103B70000549064B9E2207F0E7FC04B080BDC04615
:103B80002C10014062ED000083ED00009AED000072
:103B9000C0940102F0B58DB00A4603460CAC20700B
:103BA0000BA801700AA900250D802B4955260E701F
:103BB000AA264E7003268E700C9F7F1DCF700E714B
:103BC0000B9E4E710C9E8E7100784000234E301873
:103BD0002478C91D08900846089907922246069342
:103BE0000595FCF7C7FA05990991FFE709980CA913
:103BF0000978491D88420DDAFFE7099816494018EF
:103C000080780A9908180AA90880FFE70998401CDB
:103C10000990EBE70CA80178491D0F4A931C04900A
:103C200018460392FDF726FB0AA90880049802783B
:103C3000039BD218497811720A99D1710178093120
:103C40000022104602911946029C01922246019BD5
:103C500009F0F0FA0DB0F0BD9C950102ECA0010254
:103C600080B582B0014601AA1070FFE707480068DE
:103C7000406A002801D0FFE7F8E701A901220020EF
:103C80000090009B09F0D6FA02B080BDF8940102C2
:103C900080B582B00190FFE701980078002808D035
:103CA000FFE701980078FFF7DBFF0198401C0190C7
:103CB000F2E702B080BD0000F0B58AB0119C109D03
:103CC0000F9E0746059009A8049005980391049952
:103CD000087003980890079206930A7892001B4B8D
:103CE00098180899029008789854C878029AD07069
:103CF0008878907048785070049801788900144B47
:103D00005818079A019010785854D0780199C870C3
:103D100090788870507848700498027892000D4B23
:103D2000069898500498027852000B4B98180F99F7
:103D30000090087898544878009948700498017861
:103D40008900064A119B53500AB0F0BDF496010257
:103D5000589701024CB40102C0960102E8B3010277
:103D600080B506480168491C01600069002804D03C
:103D7000FFE7024800698047FFE780BDCCB301023E
:103D80000148024901607047089001020026B8030B
:103D900080B582B00020019001990901194A51585B
:103DA000C860019800011018C06800280AD0FFE719
:103DB0000198000113490A18D2680858016801A83F
:103DC0009047FFE702B080BD80B582B0012001902E
:103DD000019800010B4908580022C26001980001B7
:103DE0000818C06800280AD0FFE7019800010549BB
:103DF0000A18D2680858016801A89047FFE702B086
:103E000080BDC046CC92010280B588B000200790EA
:103E10006420069003F0C4FE2F4908602F48007804
:103E2000002801D0FFE754E02D480078002801D099
:103E3000FFE74EE02A48012101702748006800286A
:103E400004D1FFE726480021017042E022480068C3
:103E50006421081A0790FFE72248006807990022AA
:103E6000884205920CD0FFE7069801210022002825
:103E70000492039101DC0498039003980590FFE7F6
:103E80000598C007002820D0FFE7174800681549AB
:103E90000A68164B9A5C02901046029A019190476C
:103EA00001980168491C01600168642904DBFFE78F
:103EB0000C4800210160FFE7074800686421081AE8
:103EC00007900698401E0690C6E70548002101703D
:103ED000FFE708B080BDC046989B010221A6010201
:103EE00020A601021CA6010200960102B8A501024B
:103EF00080B5002008F038FD80BD80B5012008F0B5
:103F000033FD80BD80B58AB0014608AA10701078D4
:103F1000642832D1FFE70020079006A92B4A0A80C7
:103F2000EFF3108172B609910590059902F026FE13
:103F300007900798002807D1FFE70120020300201F
:103F4000234902F061FCFFE70020224906AA022370
:103F5000049003F063FB079062B61F48FFF798FEDA
:103F6000AA486421049A425206F078FF1649039049
:103F7000084601F0A1FD00F093FE08A80078622831
:103F80000ED1FFE7A148622100224252028006F0D2
:103F900065FF0D490290084601F08EFD00F080FE9D
:103FA00008A8007860280DD1FFE79848602100221A
:103FB000425206F053FF04490190084601F07CFD8F
:103FC00000F06EFE0AB080BDA0860100AAAA000023
:103FD00000D0020410D002047EF1000080B586B04B
:103FE000014605AA107004A8002202807F480068DC
:103FF000082870D1FFE704A8002101800391FFE7A2
:1040000003987C490978491F88420CDAFFE7039836
:104010007D49085C0499081804A90880FFE7039803
:10402000401C0390ECE7754800780499081804A92F
:10403000088070480078049A101808806C4800784E
:10404000049A101808806E480078049A10180880A6
:1040500069480078049A1018088005980499401857
:10406000C0B2FF282DD1FFE76448007801280290F4
:104070001DD0FFE70298022821D1FFE75C480078B5
:10408000624908185E490A785F490191FCF772F8A5
:1040900001990A78012A05D1FFE755480078FFF712
:1040A00031FFFFE706F0DAFE009000F0F9FD54481A
:1040B00000784F4909784908FFF76CFD00E0FFE7F9
:1040C000FFE74A48002101604948017049480170F2
:1040D0004C48017088E045480068072814D1FFE784
:1040E000059848490A78484B98540878401C08704D
:1040F000087840490978491F884204D1FFE73B48C6
:1041000008210160FFE76EE038480068062807D103
:10411000FFE705983A49087034480721016061E0DB
:1041200032480068052807D1FFE705983049087034
:104130002E480621016054E02C480068042807D16D
:10414000FFE705982D49087028480521016047E0E0
:104150002648006803280AD1FFE70598254908701A
:1041600023480021017021480421016037E01F48E5
:104170000068002809D1FFE705A80078552804D178
:10418000FFE71A480121016028E01848006801286B
:1041900009D1FFE705A80078AA2804D1FFE7134852
:1041A0000221016019E01148006802280CD1FFE7E4
:1041B00005A80078032807D1FFE70C480321016018
:1041C00005980D49087007E008480021016008487B
:1041D000017008480170FFE7FFE7FFE7FFE7FFE72F
:1041E000FFE7FFE7FFE7FFE706B080BD0C9601029F
:1041F0000696010207960102089601020C90010240
:10420000059601020496010254A50102ECA00102E8
:1042100080B582B000200190019800010A49081879
:10422000C06800280DD0FFE7019800010649081872
:10423000C06801A90022009008461146009A9047E4
:10424000FFE702B080BDC0468895010280B584B00A
:10425000039000200290FFE70298514909688842C4
:104260000BD2FFE702990120FFF7ECF9FFE74C487A
:104270004068029908180290EEE749480021016061
:104280000398002807D0FFE7039801210190084612
:1042900001998847FFE704B080BDC04680B58AB069
:1042A00000200490FFF70AFAFFF73BFA3C498860C8
:1042B0000391FFF733FA039948600498079005AA21
:1042C0001070FFE7079A08A808210290FFF70AFA82
:1042D00002980188334A914201D1FFE732E008A8F1
:1042E0000088002812D0FFE708A80421019001F0FF
:1042F000BBFB06A90880088801998A88904204D0EF
:10430000FFE705A8012101701CE00EE008A88088E5
:10431000002805D1FFE708A8C088002804D0FFE7DF
:1043200005A8012101700DE0FFE708A84088079962
:10433000401808300790FFE70798194989688842B4
:10434000C0D3FFE707981649086005A80078012840
:1043500024D1FFE7FFE7079811498968884211D205
:10436000FFE7079A08A802210090FFF7BBF9009821
:1043700001880C4A914201D1FFE703E00798801CB5
:104380000790E8E7079806494A688018401E52429D
:10439000104008600020FFF759FFFFE70AB080BD1A
:1043A000E4BE0102FFFF0000B0B590B0159C149D63
:1043B0000F900E910D920C930E98002804D5FFE7F4
:1043C0000E984042099002E00E980990FFE7099884
:1043D0000A9001200B90FFE70A980D99884209DBAB
:1043E000FFE70A980D99FBF78BFE0A900B98401C8B
:1043F0000B90F1E70C980B99884203D9FFE70C98D2
:104400000B90FFE7149800280ED0FFE70E980028C5
:1044100006D4FFE715A800784007002804D5FFE779
:104420001498401E1490FFE715A800788007002814
:1044300004D5FFE70C98002833D0FFE715A80078D3
:10444000C00700282DD1FFE71498002828D0FFE7E7
:10445000FFE714980021002808910DD0FFE70B9882
:1044600014990122002388420793069201D30798EA
:10447000069006980890FFE70898C00700280ED01D
:10448000FFE71498401E14900F98202100F062F965
:104490000F98C068002801D5FFE700E0D9E7FFE7E3
:1044A000FFE70F98C06800286DD4FFE70E9800283A
:1044B00008D5FFE70E9840420E900F982D2100F08E
:1044C00049F90CE015A800784007002805D5FFE75A
:1044D0000F982B2100F03EF900E0FFE7FFE70F986F
:1044E000C06800284ED4FFE715A800788007002890
:1044F00037D5FFE715A80078C007002831D1FFE7BE
:104500000C9800282DD1FFE71498002828D0FFE749
:10451000FFE714980021002805910DD0FFE70B98C4
:1045200014990122002388420493039201D3049832
:10453000039003980590FFE70598C00700280ED068
:10454000FFE71498401E14900F98302100F002F9F4
:104550000F98C068002801D5FFE700E0D9E7FFE722
:10456000FFE70F98C06800280BD4FFE70F980E995B
:104570000D9A0C9B149C159D0195009400F006F873
:10458000FFE7FFE7FFE710B0B0BD0000B0B590B0A7
:10459000159C149D0F900E910D920C930E980990FE
:1045A00001200A900890FFE709980D99884209D3E5
:1045B000FFE709980D99FBF78DFD09900898401CBD
:1045C0000890F1E70C980899884203D9FFE70C9806
:1045D0000890FFE715A80078C007002840D1FFE742
:1045E000149800283BD0FFE715A800788007002822
:1045F00008D5FFE70C98002804D1FFE707A8302171
:10460000017003E007A820210170FFE7FFE714987D
:104610000021002806910DD0FFE708981499012287
:10462000002388420593049201D3059804900498CE
:104630000690FFE70698C00700280FD0FFE7149800
:10464000401E14900F9807A9097800F083F80F987E
:10465000C068002801D5FFE700E0D8E7FFE7FFE7E3
:104660000F98C068002870D4FFE7FFE70C98022875
:1046700004D3FFE70C98401E0C900BE00E980A99AB
:10468000FBF728FD0B900B980D99884201D2FFE7AC
:1046900005E0FFE70D980A9948430A90E6E7FFE72F
:1046A0000E980A99FBF716FD0B900B980A99414357
:1046B0000E98401A0E900F980B99254A515C00F005
:1046C00049F80F98C068002801D5FFE709E00D9967
:1046D0000A98FBF7FFFC0A90FFE70A980028DFD151
:1046E000FFE715A80078C00700282DD0FFE7149831
:1046F000002828D0FFE7FFE7149800210028039145
:104700000DD0FFE7089814990122002388420293F4
:10471000019201D30298019001980390FFE703985A
:10472000C00700280ED0FFE71498401E14900F9881
:10473000202100F00FF80F98C068002801D5FFE78E
:1047400000E0D9E7FFE7FFE7FFE710B0B0BDC046E4
:1047500038DF000083B00A46029001A80170029879
:10476000806800900098401C0299496888420ED8E1
:10477000FFE7019802990968009A88540098401C44
:10478000029988600298C168491CC160FFE703B0C4
:104790007047000081B000900098002808D4FFE71F
:1047A00000981F210840012181403A480160FFE73D
:1047B00001B0704781B000900098002808D4FFE74E
:1047C00000981F2108400121814032480160FFE725
:1047D00001B0704781B000900098002808D4FFE72E
:1047E00000981F210840012181402A480160FFE70D
:1047F00001B0704781B000900098002808D4FFE70E
:1048000000981F2108400121814022480160FFE7F4
:1048100001B0704781B000900098002808D4FFE7ED
:1048200000981F210840012181401A480160FFE7DC
:1048300001B0704781B000900098002808D4FFE7CD
:1048400000981F2108400121814012480160FFE7C4
:1048500001B0704781B000900098002808D4FFE7AD
:1048600000981F210840012181400A480160FFE7AC
:1048700001B0704781B000900098002808D4FFE78D
:1048800000981F2108400121814002480160FFE794
:1048900001B0704780E200E081B0009000980028ED
:1048A0000CD4FFE700981F210840012181400448F3
:1048B0000160BFF34F8FBFF36F8FFFE701B0704709
:1048C00080E100E081B000900098002808D4FFE764
:1048D00000981F210840012181402A480160FFE71C
:1048E00001B0704781B000900098002808D4FFE71D
:1048F00000981F2108400121814022480160FFE704
:1049000001B0704781B000900098002808D4FFE7FC
:1049100000981F210840012181401A480160FFE7EB
:1049200001B0704781B000900098002808D4FFE7DC
:1049300000981F2108400121814012480160FFE7D3
:1049400001B0704781B000900098002808D4FFE7BC
:1049500000981F210840012181400A480160FFE7BB
:1049600001B0704781B000900098002808D4FFE79C
:1049700000981F2108400121814002480160FFE7A3
:1049800001B0704700E100E070B582B00190009185
:104990000198002814D4FFE701980321C943084077
:1049A000BE4A8058019B9C07E40EFF25A540A84302
:1049B000009DAD01EDB2A54028430B40985018E092
:1049C00001980F21084008380322D2431040B24B0F
:1049D000C058019CA507ED0EFF26AE40B043009ED7
:1049E000B601F6B2AE4030430C40083C1440E050F3
:1049F000FFE702B070BDC04670B582B00190009173
:104A00000198002814D4FFE701980321C943084006
:104A1000A24A8058019B9C07E40EFF25A540A843AD
:104A2000009DAD01EDB2A54028430B40985018E021
:104A300001980F21084008380322D2431040964BBA
:104A4000C058019CA507ED0EFF26AE40B043009E66
:104A5000B601F6B2AE4030430C40083C1440E05082
:104A6000FFE702B070BDC04670B582B00190009102
:104A70000198002814D4FFE701980321C943084096
:104A8000864A8058019B9C07E40EFF25A540A84359
:104A9000009DAD01EDB2A54028430B40985018E0B1
:104AA00001980F21084008380322D24310407A4B66
:104AB000C058019CA507ED0EFF26AE40B043009EF6
:104AC000B601F6B2AE4030430C40083C1440E05012
:104AD000FFE702B070BDC04670B582B00190009192
:104AE0000198002814D4FFE701980321C943084026
:104AF0006A4A8058019B9C07E40EFF25A540A84305
:104B0000009DAD01EDB2A54028430B40985018E040
:104B100001980F21084008380322D24310405E4B11
:104B2000C058019CA507ED0EFF26AE40B043009E85
:104B3000B601F6B2AE4030430C40083C1440E050A1
:104B4000FFE702B070BDC04670B582B00190009121
:104B50000198002814D4FFE701980321C9430840B5
:104B60004E4A8058019B9C07E40EFF25A540A843B0
:104B7000009DAD01EDB2A54028430B40985018E0D0
:104B800001980F21084008380322D2431040424BBD
:104B9000C058019CA507ED0EFF26AE40B043009E15
:104BA000B601F6B2AE4030430C40083C1440E05031
:104BB000FFE702B070BDC04670B582B001900091B1
:104BC0000198002814D4FFE701980321C943084045
:104BD000324A8058019B9C07E40EFF25A540A8435C
:104BE000009DAD01EDB2A54028430B40985018E060
:104BF00001980F21084008380322D2431040264B69
:104C0000C058019CA507ED0EFF26AE40B043009EA4
:104C1000B601F6B2AE4030430C40083C1440E050C0
:104C2000FFE702B070BDC04670B582B00190009140
:104C30000198002814D4FFE701980321C9430840D4
:104C4000164A8058019B9C07E40EFF25A540A84307
:104C5000009DAD01EDB2A54028430B40985018E0EF
:104C600001980F21084008380322D24310400A4B14
:104C7000C058019CA507ED0EFF26AE40B043009E34
:104C8000B601F6B2AE4030430C40083C1440E05050
:104C9000FFE702B070BDC0461CED00E000E400E09C
:104CA000BFF34F8F034804490160BFF34F8FFFE705
:104CB00000BFFDE70CED00E00400FA0570B5C6B0DA
:104CC0004C9C4B9D4A9E419040913F923E93409810
:104CD00036903F983790B4483D903E9833904A982C
:104CE00034904B983590EFF303804290429838907F
:104CF000EFF30880439043983B90EFF30980449092
:104D000044983C9041983990EFF314804590459831
:104D10003A9030942F952E9606F0C8FE00203290DF
:104D2000A2482A212D902C9107F04AFA4C992B90F9
:104D300008462A9106F00CFB2A99299008462999E1
:104D400007F03EFA9A490222289008462791114618
:104D5000269207F035FA2D99259008462C9907F0F0
:104D60002FFA3299934A121D53180124E502691A49
:104D7000249023922293219420951F9106F036FBD4
:104D80008D4A22991E9008461F991E9B04F068F8D0
:104D9000329908183290329823990A18209B191AD0
:104DA0003798219CA043031F84481D9010461D9AEC
:104DB00004F056F83299081832903299239807F087
:104DC000FFF97F490A221C90084611461B9207F002
:104DD000F7F93E991A900846199106F0B9FA19990F
:104DE00018900846189907F0EBF92799179008468C
:104DF000269907F0E5F97349169008461B9907F0C4
:104E0000DFF94A9915900846149106F0A1FA149911
:104E100013900846139907F0D3F927991290084682
:104E2000269907F0CDF96849119008461B9907F0BB
:104E3000C7F94B9B654A239910900846209904F0C6
:104E40000FF832903299239807F0BAF927990F900A
:104E50000846269907F0B4F9369B5D4A23990E90CF
:104E60000846209903F0FCFF3290329823990A18E3
:104E7000209B191A379B57480D9010460D9A03F046
:104E8000EFFF3299081832903299239807F098F979
:104E9000389B514A23990C900846209903F0E0FF73
:104EA0003290329823990A18209B191A3898C30F08
:104EB0004400E40F8500ED0FC000C00F0290019583
:104EC000009446480B9010460B9A03F0C9FF3299A4
:104ED00008183290329823990A18209B191A38988A
:104EE0003F2420403E4C0A90104622460A9B03F085
:104EF000B7FF3299081832903299239807F060F979
:104F0000399B384A239909900846209903F0A8FF55
:104F10003290329823990A18209B191A3A9B3248EA
:104F200008901046089A03F09BFF329908183290B7
:104F30003299239807F044F93B9B2C4A2399079018
:104F40000846209903F08CFF3290329823990A1872
:104F5000209B191A3C9B264806901046069A03F09F
:104F60007FFF3299081832903299239807F028F978
:104F7000204931913699319A521A1F4B9A42059124
:104F800004D3FFE70120C002049004E03198369971
:104F9000401A0490FFE7049881083222059807F030
:104FA0004FF946B070BDC04611114B4D69DF00008E
:104FB00039FF0000E8B40102D2ED0000E9ED000085
:104FC00048DF000053DF00005EDF00007CF00000DF
:104FD0006CEE0000A6EE0000C8EE0000E1EE00005E
:104FE000BCEE00003CEE00004BEE000078EE00004E
:104FF00083EE000000F802020108000080B582B0D4
:10500000019005480068BC2140580199009008466D
:105010000099884702B080BD0090010280B586B03B
:10502000049003910498002803D0FFE70120059025
:1050300040E01620029000F089FB029805F094FDF4
:10504000FFE7039800280AD0FFE7049880011B4976
:105050000818183003991422FBF78CF8FFE704981E
:105060008001164908182821405C002819D0FFE764
:1050700004988001114908184068002201911146E6
:10508000FFF782FC04988001019908184068FFF737
:1050900091FB04988001019908184068FFF712FC01
:1050A000FFE70498800105490818012101610020EB
:1050B0000590FFE7059806B080BDC0463490010218
:1050C0005A21014A50527047BC97010280B586B000
:1050D000059000200390029021480078052805D112
:1050E000FFE71F480178491E0170FFE71C48007860
:1050F0000190FFE70198012816DBFFE701981949A5
:1051000080000A18121F12680A500198800008587F
:10511000C117039A029B18184A4102900392FFE7B5
:105120000198401E0190E5E705980E49086008685F
:10513000C117039A029B18184A410290039208482B
:105140000178491C01700299039A007800230090AD
:1051500008461146009AFAF7E7FF06B080BDC04640
:10516000349801022098010210B586B0CB484C213A
:105170000171372141718171C1710021018141812A
:105180008181214A9388D4882404E31805931388E5
:1051900052881204D21804921C4A9388D48824049A
:1051A000E3180393138852881204D2180292184A03
:1051B0009388D4882404E318019313885288120436
:1051C000D218009204AAD3888382059B4382528816
:1051D0000282049AC28102AAD3888383039B4383F9
:1051E00052880283029AC2826A46D3888384019BD2
:1051F000438452880284009AC2835C2281545D22D7
:10520000815406B010BDC046B0E20000B8E2000014
:10521000C0E2000080B5FFF7A7FF80BD80B584B075
:1052200019484C210160FF20023000F059FA322069
:1052300000F042FC00F078F9012103900846029149
:1052400000F07EF9029800F04BF800F067F90F4982
:105250000190084600F044FA00200090009900F008
:1052600011FB0298009900F00DFB0298000200F07B
:1052700037FA022000F034FA2920C00006F088F83E
:1052800006F0FAF804B080BD4800004001020000BA
:1052900080B582B005200421019102F063FD062053
:1052A000019902F05FFD0A20019902F05BFD0920DF
:1052B000019902F057FD00200121009002F052FDFB
:1052C00002210098009A02F08BFD02B080BD000020
:1052D0000248016801229143016070475800004074
:1052E00081B00090FFE78548006800990840884237
:1052F00001D0FFE7F7E701B07047C04680B584B042
:10530000664800788007002805D5FFE763480079E4
:1053100000F086F9FFE7614840788006002806D54E
:10532000FFE75E485E21405C00F016F9FFE71720BA
:1053300000F00CFA5A480168032291430391039943
:105340000222114301605748574901605748002124
:105350000170574801781F22114003910399017091
:105360005448007802A908705348007853490978D6
:10537000090240185249097809044018514909782E
:1053800009064018504988422BD1FFE74F48007862
:105390004F490978090240184E4909780904401814
:1053A0004D490978090640184C49884219D1FFE750
:1053B0004B4800784B4909780902401880B24A49A5
:1053C00088420ED1FFE702A80078012809DBFFE739
:1053D00002A80078132804DCFFE74448202101706C
:1053E000FFE743480078039003A80078C006002830
:1053F00006D1FFE70398102108433D490870FFE7F5
:105400003C48016820229143016052483A490160BA
:10541000FFE73A480068C00F002801D1FFE7F8E72E
:1054200003F018FD0190019B354A0220032106F08C
:105430006BFF0199002912D0FFE701980121890231
:1054400088420CD0FFE701980121C902884206D0AA
:10545000FFE7019803218902884207D1FFE72E4A1E
:105460000220032106F050FFFFE7FEE72548016810
:105470000F22914303910399016023480168234A55
:10548000114003910399016019200001204908602F
:1054900020481F21016004B080BDC0463898010239
:1054A000040200400C060040AF6B100A720001407D
:1054B00071000140750001407C0001407D00014009
:1054C0007E0001407F0001404D3836507800014099
:1054D000790001407A0001407B000140312E3236D4
:1054E000760001407700014007340000730001405E
:1054F0006B0001402C000040FE1C00800460004056
:10550000D2EA0000D4600040C8600040FEFFC3FF44
:10551000100400400C04004057EA000080B517203A
:1055200000F008F9002080BD80B582B017200190FE
:1055300000F00CF9019805F017FB002002B080BDC7
:1055400081B0009000980121C90708430149086013
:1055500001B070470060004010B584B0014603AA56
:1055600010700E4803680293029B7F24A3430293AA
:10557000137823401370029B127813430360006872
:105580002040074A02230324019018460091214637
:10559000019B06F0B9FE04B010BDC0464C000040AF
:1055A000A5EA000080B584B003902E480068029000
:1055B00002987F21084001A908700398032805DBA1
:1055C000FFE70198401C01A908700CE00398022134
:1055D000C943884205DCFFE70198401E01A9087015
:1055E00000E017E0FFE702987F218843029001A8BE
:1055F00000780840029A024302920298194A106009
:10560000039B029808400090034A0448032106F0D7
:105610007BFEFFE704B080BD88EA000002080000BE
:1056200010B584B0014603AA10700E4803680293B7
:10563000029B7F24A3430293137823401370029BA1
:1056400012781343036000682040074A02230324B2
:105650000190184600912146019B06F055FE04B0CA
:1056600010BDC04648000040BBEA000080B584B0D1
:10567000014603AA10701078002827D0FFE703A87E
:105680000078022805D0FFE703A8007803280ED190
:10569000FFE703A80078012102220328029201916A
:1056A00001D002980190019800F0A0F9FFE7FFE710
:1056B000C04800688007002801D4FFE7F8E7BC482D
:1056C0000168012252071143016006E0B8480168F1
:1056D0000122520791430160FFE704B080BDC0463C
:1056E00080B584B00390039802A908700398000A5B
:1056F00001AA107008780028009008D0FFE70098F1
:10570000012809D0FFE7009802280AD00EE001A87E
:105710000078FFF7ABFF0AE001A8007800F0FAF884
:1057200005E001A8007800F047F900E0FFE704B0C9
:1057300080BD000081B000900098012181409C480C
:1057400002688A43026001B07047C04681B0009091
:10575000009801218140964802680A43026001B026
:105760007047C04681B0924800680121C90300908B
:10577000084601B07047C04680B500F04DF89A4920
:105780000968032212071140090FC84080BDC046B6
:1057900080B5FFF7F1FF9449096803229206114092
:1057A000890EC84080BDC04680B500F035F88E49EE
:1057B0000968032292041140890CC84080BDC0468C
:1057C00080B584B0039000200290039805280190D2
:1057D0001FD80198784400794000874402060A0ED9
:1057E000121600F019F8029013E0FFF7C5FF0290BF
:1057F0000FE0FFF7CDFF02900BE000F02FF80290D2
:1058000007E0FFF7AFFF029003E0FFF7CDFF029044
:10581000FFE7029804B080BD83B06548006840008F
:1058200000280ED5FFE762480068C00009490A4A0F
:1058300000280192009101D40198009000980290F4
:1058400005E05B4800680121C9030291FFE7029867
:1058500003B070470026B803006CDC0280B582B04C
:10586000614800684000002804D5FFE7FFF790FF7B
:10587000019003E0FFF776FF0190FFE7019802B087
:1058800080BDC04683B00A46029001A8017002980C
:10589000042800903CD80098784400794000874460
:1058A000020D18232E00504801680322120791436D
:1058B000019A920792088918016029E04A48016814
:1058C000032292069143019A9207120989180160F6
:1058D0001EE045480168032292049143019A920711
:1058E000120B8918016013E03F480168FF22120281
:1058F000914301AA127812028918016008E03A481F
:105900000168FF22914301AA127889180160FFE71C
:1059100003B0704780B584B0014603AA10702448D4
:10592000006802901078002806D1FFE70298012154
:1059300089078843029035E003A8007801280AD13E
:10594000FFE7029801218A07104302900298090795
:105950008843029025E003A80078032805D0FFE7DC
:1059600003A8007804280ED1FFE703A800780121DE
:10597000022204280192009101D001980090009821
:1059800000F048F8FFE7FFE70A48006840060028F3
:1059900001D4FFE7F8E702980521090708430290C0
:1059A000FFE7FFE702980249086004B080BDC046E7
:1059B000200000402C02004081B001466A46107071
:1059C0001078002807D0FFE70748016801229207F6
:1059D0001143016006E004480168012292079143E7
:1059E0000160FFE701B070472400004082B00190E1
:1059F0000748016800910099032212049143009125
:105A00000099019A12041143016002B07047C04628
:105A10004C00004082B001900D480168009100994F
:105A20000C4A114000910099019A1204114301603F
:105A300009480021016009480949016009480168D5
:105A4000009100990D2252021143016002B070478B
:105A50004800004080FFFCFF1002004004010040AD
:105A6000FF0F00001402004010B584B003900291B3
:105A700001A8002101800091FFE700980299884267
:105A800013D2FFE701A801880A02090A039B5C1CE4
:105A900003941B7859404900064B595A4A400280EA
:105AA000FFE70098401C0090E7E701A8008804B0D9
:105AB00010BDC04600E0000081B0009000280AD070
:105AC00030B407252C02CD256419604340091238F3
:105AD000001FFDD830BC01B07047F0B583B01F4641
:105AE00016460D460146E8680291FAF7C0FB0446E7
:105AF0000F2E11D8082E04D320462146FAF75EFB5C
:105B000009E0042E02D38120C10501E041200106F5
:105B10002046FAF7ACFB04460999089E2B20C043A7
:105B2000874205DB20460F462146FAF747FB0DE08A
:105B30003F20C04387420BDA4920C04387420CDB39
:105B4000FF200F4681052046FAF791FB39460446AF
:105B5000688A0880346003B0F0BD01915320C043CF
:105B6000874206DB20462146FAF728FB0446688A6E
:105B700010E0A8690299FAF7A3FD002801D1A88BCB
:105B800000E0E88BFAF7FDFD01462046FAF76FFBCF
:105B90000446002001990880346003B0F0BD000085
:105BA00080B586B0049003910498072804D8FFE7D5
:105BB0000398002803D1FFE70120059056E05B48D9
:105BC00000680069C00700281CD1FFE7052002908B
:105BD000FFF7BCFD029804F0C7FF544801680A694A
:105BE00001231A430A614168019008461946FEF7ED
:105BF00003FF01984068FEF7EDFD01984068FEF74D
:105C000071FEFFE70398C169C906890C8069C0006D
:105C1000C0B2081845490A68049B5B01D2184123A9
:105C20009B00D050039802685207520943685B07F3
:105C30005B0BD21883685B079B0CD218C3685B07A9
:105C40005B0DD21803695B01DBB2D2184069800793
:105C5000C00E1018802210430968049A5201891856
:105C600001221202885000200590FFE7059806B037
:105C700080BDC04610B586B0089C04900391029286
:105C800001930298002806D1FFE725482549264BB5
:105C9000742205F059FC25480068C0680499083151
:105CA000C840C007002803D0FFE70220059033E07A
:105CB0000898049989001D4A511888601068049951
:105CC000490140184121890043580724A343435008
:105CD00003981168049B5B01C91843239B00C850BB
:105CE00002981168049B5B01C91811231B01C8505D
:105CF00001981168049B5B01C9182123DB00C8507F
:105D0000106804994901401801210A0283580B4385
:105D1000835000200590FFE7059806B010BDC046EF
:105D2000E2EA000015EB0000FBEA000084920102A9
:105D300081B00090009800015D490858406801B0AA
:105D40007047C04680B586B004900391049801283E
:105D500004D8FFE70398002803D1FFE7012005904E
:105D60007FE00498002804D1FFE70E20FFF7EEFC47
:105D700008E00498012804D1FFE70F20FFF7E6FCB4
:105D8000FFE7FFE7FFE703988068002805D1FFE7FA
:105D90000398C08900280BD0FFE70398806801288A
:105DA00006D0FFE730483149314B492205F0CCFBA2
:105DB000049800013E4908580021C1600398816899
:105DC000C907890F42689207120F89180069C00736
:105DD000800E0818029003980068012805D1FFE79B
:105DE00002980121084302900AE003980068022803
:105DF00005D1FFE70298402108430290FFE7FFE743
:105E00000298049909012A4A515888600398C06889
:105E1000049909015158086003980069049909011F
:105E20005118886003984069049909015118C860A5
:105E3000049800011018406802210192FEF714FE38
:105E400004980001019908184068FEF7D3FC0498F3
:105E50000001019908184068FEF754FD00200590E4
:105E6000FFE7059806B080BD22EB000054EB000070
:105E700042EB000082B00190009100980199090165
:105E80000B4A51580860019800011058816880221F
:105E90001143816002B0704781B00090009800010A
:105EA00003490858816880229143816001B070479E
:105EB000CC920102F0B58DB0019315460E460A90C2
:105EC0001298002408900480149F3C801398099035
:105ED0000460159804900480FF2081053046FAF78D
:105EE000C6F90290304603963146FAF767F92B4619
:105EF0003D460690274607950B9311E011801888C0
:105F000080002858099908600120079D28800520F5
:105F1000049908807F1CBCB21888844200D9A0E094
:105F200028880028F6D1A0000A9D2E5830460699F0
:105F3000FAF7B8FB002817D030460399FAF7B2FBFE
:105F400000280B9B079DE5D1089A1780099D2E60BC
:105F50001888011B012934D11080198889000A9AF8
:105F600051582960059035E0089A17800998066015
:105F70000B9B1988081B0128C0D00C960198251886
:105F80007E1CB0B28542BFD389B2B2B28A420ED86B
:105F900080000A990C5820460C99FAF775FB0B9B68
:105FA000002804D109980460089806800C94761C97
:105FB000B0B28542A8D3198889B2B2B28A42E7D971
:105FC000F5E70C96019962187D1CA9B216468A4223
:105FD00005972CD2059884B2A5000A9E7259002C10
:105FE000104609D0A819001F016810460C92FAF754
:105FF000E5F80C9A062C07D80446A8194168104603
:10600000FAF7DCF80C902046079D0299FAF758FB46
:1060100000280B9B07D10C980299FAF743FB0B9BC6
:10602000002800D076E701202880032070E780B2A6
:10603000AAB282420FD888000A990C5820460C99BF
:10604000FAF722FB0B9B002805D1099804600898F9
:10605000058005950C946D1CA9B28E42BAD31888A0
:10606000E5E70DB0F0BD00000A490A680A480240A1
:106070000A60FD214900094A1268515C002908D0D4
:1060800007490A6C02400A64012000060A6882433C
:106090000A60704700040040FFFFFF7F2894010260
:1060A0002000004000207047B0B588B006900591F0
:1060B000059806997C224A43AE498918CA69096A3B
:1060C00003901046FAF706F80399814206D3FFE7DA
:1060D0003B483C493C4B3D4A05F036FA06980321C3
:1060E00001F04EF904900498002803D0FFE70498CB
:1060F000079062E0069801F099F80698062101F0F1
:10610000BDF906987C210A4642439A4883189C6947
:10611000059D1B6A6B43E31882589360069A5143AE
:106120004018C07DC009012818D1FFE706987C21DE
:106130000A4642438F488258D36920242343D361BF
:10614000069A0B465343C25813680124A5052B43F6
:106150001360069A51434018C466FFE7069805216C
:1061600001F08CF906987C21414382484018C07D9B
:10617000C00900281ED1FFE70698154909687D224D
:10618000D3000290084619460192F9F7A3FF01993E
:106190004A0142430298114601F02AF9069800216B
:1061A00001F00AFA06987C21414372484018012107
:1061B0000161FFE700200790FFE7079808B0B0BD36
:1061C000F2EB000018EC000096EB00005D0200000E
:1061D000E0B3010210B588B0069005A80021017057
:1061E00006987C210A464243F3488218D26E04ABDB
:1061F0001A70069A0C4654430219D26E120A03AC66
:106200002270069A514340186E21405A02A9087024
:106210001878012805D0FFE704A80078022812D1D9
:10622000FFE703A80078002804D1FFE705A80121B3
:10623000017007E0069800F0C7FF0121084005A99A
:106240000870FFE716E004A8007803280AD1FFE7EA
:1062500003A80078002804D1FFE705A801210170F8
:10626000FFE706E005A80078411E884107A90870ED
:1062700048E0FFE705A8007800283CD1FFE7069832
:106280007C214143CC4840180021C166069801F0AA
:1062900093F902A80078032805D0FFE702A8007848
:1062A000002808D1FFE706987C214143C2484018E6
:1062B0000121016107E006987C214143BE48401856
:1062C00006210161FFE706987C214143BA48401846
:1062D000006F00280ED0FFE706987C214143B648A6
:1062E0004018006F04A9097806AA01901046019A87
:1062F0009047FFE7FFE705A80078411E884107A9FE
:106300000870FFE707A8007808B010BD80B582B01C
:1063100000900098002803D0FFE70120019025E0BD
:1063200000987C214143A44840187821405C002813
:1063300003D1FFE70420019018E00098092101F043
:106340009DF80F20FFF7B8FB1520FFF7F3F9009831
:106350007C210A4642439848821800231361009A20
:1063600051434018782143540193FFE7019802B04C
:1063700080BDC046F492010270B590B00F900E91AE
:1063800000200D900F9909780CAA11700BA90870C4
:1063900010780D997C224A4387498918C968884238
:1063A0007DD1FFE70E98032871D1FFE70D987C217E
:1063B000414381484018416E806E814207D8FFE713
:1063C0000D9800F033FF0BA8012101705EE00D98DD
:1063D000062101F053F80D987C210A464243764885
:1063E0008318DB6D825893600D9A00230990104644
:1063F0000891194601F042F80D980899414309980F
:1064000041184A6E896E511A0A910A990D9A089B91
:106410005343C218928C914208D9FFE70D987C2112
:106420004143F3484018808C0A90FFE70D987C2187
:106430000A464243EE488318DC68825814321B6EC9
:106440000A9DAD085E4E00960790204606911146C3
:106450001A462B46FFF70EFC0A990D9A069B5343EA
:10646000079AD3189C6E611899660A990D9B069C31
:106470005C4313191C6E611819660A990D9B069CE2
:106480005C431319DC6D6118D965FFE706E00D98D0
:1064900000F0CCFE0BA801210170FFE76EE00CA814
:1064A00000780D997C224A43D1498918896888422D
:1064B0005CD1FFE70E98032853D1FFE70D987C21AC
:1064C0000A464243CA488218D38CD46DE318D36578
:1064D0000D9A0B465343C218D38C146EE3181366FF
:1064E0000D9A0B465343C218D38C946EE3189366EF
:1064F0000D9A51434018416E806E814204D8FFE7E7
:106500000BA8012101702BE00D98062100F0B6FFC9
:106510000D987C210A464243B5488318DB6D8258AA
:1065200093600D9A0123059010460491194600F0DE
:10653000A5FF0D9804994143059842189068136E81
:10654000059C61581431D28C92081D4D0095039121
:106550001946039B02921A46029BFFF78BFBFFE74B
:1065600003E00BA801210170FFE706E0A1481349F1
:10657000A24B4D22120104F0E7FFFFE70BA80078C1
:10658000002816D0FFE70D987C210A464243984820
:10659000825813680124E507AB4313600E9A120476
:1065A0000D9B59434018C16E0A4321020A43C2663B
:1065B000FFE710B070BDC046F49201023DEC000050
:1065C00079630000B0B58EB00D900C9100200B9057
:1065D0000D9909780AAA117009A9087010780B9909
:1065E0007C224A43824989188968884200D0DCE0CD
:1065F0000C98032800D0D3E00B987C210A46424334
:106600007B488218936A546D1B1913660B9A0B46CC
:106610005343C218926D0B9B0C465C430319DA6519
:106620000B9A0B465343C218536D93660B9A0B4655
:106630005343C218936C5B1C93640B9A51434018EC
:10664000416E806E814204D8FFE709A801210170E4
:10665000A5E0AF204000FFF72FFA0B987C214143C3
:10666000F6484018816C406C814242D1FFE70B989C
:106670007C214143F1484018806C022839D3FFE760
:106680000B987C210A464243EC488218D38C546D07
:10669000E31853650B9A0623089010460791194694
:1066A00000F0ECFE0B980799414308984218D26D10
:1066B00041588A600B99079A4A438218126D08461E
:1066C000114601F0FDF90B980799414308984218CB
:1066D0009068136E089C61581431126D494D0095F5
:1066E00006911946069B05921A46059BFFF7C2FACA
:1066F00054E00B987C214143D0484018816C406C99
:1067000081424AD2FFE70B987C214143CB48401895
:10671000806C022841D3FFE70B987C210A46424354
:10672000C6488218D38C546DE31853650B9A0B46F8
:106730005343C218D38C946DE31893650B9A0623C8
:10674000049010460391194600F098FE0B980399A7
:10675000414304984218D26D41588A600B99039ABC
:106760004A438218D28C0846114601F0A9F90B98C9
:1067700003994143049842189068136E049C615831
:106780001431D28C1F4D009502911946029B019243
:106790001A46019BFFF76EFAFFE7FFE7FFE703E00A
:1067A00009A801210170FFE705E012481249134BC7
:1067B000134A04F0C9FE09A80078002816D0FFE7A4
:1067C0000B987C210A464243EB4882581368012407
:1067D000E507AB4313600C9A12040B9B5943401816
:1067E000C16E0A4321020A43C266FFE70EB0B0BD84
:1067F000F4920102F2EB000050EC0000CBEB000041
:1068000072040000C565000010B596B01490139195
:1068100012921398800E00280CD0FFE7139812995B
:106820008122D204511A884204D8FFE71298002826
:1068300003D1FFE701201590FDE0139814997C2205
:106840004A43CD498918898CF9F744FC00290CD1B9
:10685000FFE7129814997C224A43C7498918898C0A
:10686000F9F738FC002903D0FFE701201590E2E09A
:10687000139814997C2213464B43BF49CB189B694C
:10688000C01A11901198149B14465C430B199B8CF1
:10689000059119460492F9F71DFC10901198129970
:1068A00040181499049A4A4305998A18918CF9F76B
:1068B00011FC0F9014980499414305984118086AF7
:1068C000898CF9F707FC0E900F981099401A0E99D1
:1068D00088421AD2FFE710980D90FFE70D980F99A4
:1068E000884211D2FFE714980D9900F0B3FCFFE73E
:1068F0001498FFF76FFC002801D0FFE7F8E7FFE7E7
:106900000D98401C0D90E9E792E0119814997C22B3
:1069100013464B439849CB181B6A039119460292C0
:10692000F9F7D8FB0C901198129940181499029A13
:106930004A4303998A18116AF9F7CCFB0B90119816
:106940001499029A4A4303998A18116AF9F7C2FB0B
:10695000002904D0FFE70C98401C0C90FFE7119829
:106960001299401814997C224A43834989180A6A6B
:1069700001911146F9F7AEFB019A938C00900846FD
:106980001946F9F7A7FB0A9010980990FFE70998B4
:106990000C990E9A4A43904211D2FFE71498099934
:1069A00000F058FCFFE71498FFF714FC002801D012
:1069B000FFE7F8E7FFE70998401C0990E7E70C9824
:1069C0000890FFE708980B99884211D2FFE71498C6
:1069D0000899FFF769FBFFE71498FFF7FBFB002816
:1069E00001D0FFE7F8E7FFE70898401C0890E9E7C7
:1069F0000B980E994143079100200690FFE70698F7
:106A00000A99884213D2FFE714980799069A8918C1
:106A100000F020FCFFE71498FFF7DCFB002801D012
:106A2000FFE7F8E7FFE70698401C0690E7E7FFE777
:106A300000201590FFE7159816B010BDF4920102E2
:106A400070B58AB009900891079206930798099942
:106A50007C2213464B43ED49CB18986209981346A4
:106A60004343C818002343650898099C15466543AD
:106A70004C19A0650898099C154665434C19E062BD
:106A80000898069C0019401E099C154665434C1940
:106A900020630898099C154665434C19A569401B5D
:106AA00060630998144644430819446BC58C0590EB
:106AB00020460491294603920293F9F70BFB0599AE
:106AC00088630998039A424304988218536B069C82
:106AD0001B19581ED18C0192F9F7FCFA0199C86371
:106AE0000998039A424304988218D36B946B1B1B3A
:106AF0001364099A039B5343C218136C5B1C5364C1
:106B0000099A039B5343C218029B9364099A039CFE
:106B100054430219126C002A0ED1FFE70698099916
:106B20007C2213464B43DA49CB18D8640998424378
:106B30008818002101651CE009987C210A4642431F
:106B4000D3488218D38C089C956B1E466E4395697A
:106B500075192C1B1B19D364099A51434018016BFA
:106B6000C26BC38C534382699A18891A491C016508
:106B7000FFE70AB070BDC046F4920102B0B58EB016
:106B80000C900B910C98002803D0FFE701200D908A
:106B900039E10C987C214143BD4840187821405C84
:106BA000002803D0FFE700200D902CE10B9800286F
:106BB0000CD0FFE70C987C214143B54840181430B5
:106BC0000B990CC90CC01CC91CC0FFE70C987C2198
:106BD0000A464243AE4882180023D3661522089025
:106BE0001046079106930592FEF7B0FD059803F055
:106BF000BBFF0C9800F01AFB0C98079941430898CA
:106C00004218938A947D2407240B1B19D27D940784
:106C1000E40F64051B19D406E40FE4051B1954079F
:106C2000E40FE4061B19D407E4081B199406E40FCB
:106C300064071B191207D20F9207134341580B60C8
:106C40000C980A2100F01AFC3220FEF735FF069856
:106C50000A900C98082100F011FC0C982021069A4B
:106C600000F0E4FB0C980799414308984158097DCE
:106C70000A910A99C22909D1FFE70C987C21414366
:106C80008348401874210122425408E00C987C216A
:106C900041437F484018742100224254FFE70A987C
:106CA00000020C997C2213464B437949CB581B7D3B
:106CB000C0180A900A9800020C9B14465C430B59BA
:106CC0001B7DC0180A900A9B51480224032504909A
:106CD000204603912946049C0292224605F014FBAB
:106CE00009A900220A700C99029A4A4303998A184A
:106CF0007423D25C012A0CD1FFE70C987C2141431C
:106D0000634A5118C97D01228A43114600F070FE82
:106D10002DE00C9800F070FA8007C00F09A90870E8
:106D20000C987C2141435A484018C07DC007002878
:106D300005D1FFE709A8007800280FD0FFE70C98DD
:106D40007C21414352484018C07DC00700280DD027
:106D5000FFE709A80078012808D1FFE70C9809A9E6
:106D600009784A42514100F043FEFFE7FFE70C98E3
:106D70007C214143464840187721405C012805D1D9
:106D8000FFE702200021FEF77DFDFFE70C980021C0
:106D900000F012FC0C987C2141433D484018C07D16
:106DA000C00901281FD1FFE70C987C210A46424305
:106DB000FE4882185268022301901046009119463D
:106DC000FDF78AFE0C9800994143019841184868E4
:106DD000FDF720FD0C98009941430198411848683F
:106DE000FDF7A0FDFFE70C987C210A464243EF48DF
:106DF0008218012313610C9A51434018782143549F
:106E000000200D90FFE70D980EB0B0BDF492010286
:106E1000E4EB000080B586B00590049103920293E4
:106E20000598062100F02AFB049805997C224A4324
:106E3000FD49895888600598029900F041FE0020BC
:106E40000190FFE70198029988420ED2FFE703986C
:106E50000199405C05997C224A43FD49895808758F
:106E6000FFE70198401C0190ECE705980949096883
:106E70007D22D200009008461146F9F72BF9062131
:106E80004143009800F0B4FA002006B080BDC0462F
:106E9000F4920102E0B3010270B59EB01C901B9108
:106EA0001A9219931C987C214143E9484018C07DEF
:106EB0004006C00F012806D1FFE719A80078800717
:106EC00000280AD003E00120002806D1FFE7B848D7
:106ED000B849B94BB94A04F037FB1B98800E00281B
:106EE0000CD0FFE71B9819998122D204511A8842CD
:106EF00004D8FFE71998002803D1FFE701201D906F
:106F000051E11C98022100F03BFA189018980028D3
:106F100003D0FFE718981D9045E11C9800F086F912
:106F20001C987C214143CA484018C07D4006C00FD0
:106F3000012800D090E01C987C210A464243C448B6
:106F4000825813680124E407234313601B9A1C9B97
:106F50000C465C430319DA651A9A1C9B0C465C4389
:106F600003191A66199A1C9B0C465C4303195A664E
:106F70001C9A0B465343C218002393661C9A0C4676
:106F8000544302190324D4661C9A06240A9010461E
:106F900009912146089300F071FA1B981C99099AEF
:106FA0004A430A998A5890601C98089900F066FA3A
:106FB000834810A93CC83CC13CC83CC119981C99E5
:106FC000099A4A430A998A18928C904208D9FFE795
:106FD0001C987C214143E4484018808C1990FFE7BD
:106FE0001C987C210A464243DF488218D26810ABC5
:106FF0000790104606911946FEF7D2FD1C99069A95
:107000004A4307998B18DB688A5814321A9C199DD9
:10701000AD086C4E009605901846114622462B4648
:10702000FEF728FE19991C9A069B5343079AD3181A
:107030009C6E6118996619991C9B069C5C431319F8
:107040001C6E6118196619991C9B069C5C431319E8
:10705000DC6D6118D965A3E019981C997C22134650
:107060004B43E249CB189B8C049119460392F9F7E4
:1070700031F80F9019981C99039A4A4304998A1879
:10708000918CF9F727F80E9100210D91FFE70D98EB
:107090000F9988423DD2FFE71C98062100F0EEF9D7
:1070A0001B980D991C9A7C235343F34AD418A48C43
:1070B0004C430019D15888601C980021029100F0BF
:1070C000DDF902980C90FFE70C981C997C224A434A
:1070D000E9498918898C884216D2FFE71C987C21DF
:1070E0000A464243E4488258127D1A9B0D9C1C9D1F
:1070F00069434018808C60430C9940181A54FFE78C
:107100000C98401C0C90DFE7FFE70D98401C0D9099
:10711000BDE70E98002834D0FFE71C98062100F048
:10712000ADF91B980F991C9A7C235343D24AD4186B
:10713000A48C4C430019D15888601C9800210191FF
:1071400000F09CF901980B90FFE70B980E9988428C
:1071500016D2FFE71C987C210A464243C648825853
:10716000127D1A9B0F9C1C9D69434018808C6043C4
:107170000B9940181A54FFE70B98401C0B90E4E75A
:10718000FFE71C9800F052F81C98002100F014FA58
:107190001C987C214143B848401801210161FFE758
:1071A00000201D90FFE71D981EB070BDF4920102F3
:1071B000F2EB00000DEC000064EB0000C6030000E1
:1071C00070E200007963000080B582B00190019800
:1071D000022100F053F901982021002200F026F945
:1071E00001987C214143F2484058007D694608706F
:1071F000087802B080BDC04680B582B00190019889
:10720000032100F03BF901982021002200F00EF943
:1072100001987C214143E6484058007D694608704A
:10722000087802B080BDC046F492010280B582B0F9
:10723000019001987C214143F74840581021C161D9
:1072400001980091009A00F0F1F802B080BDC046AC
:10725000F4920102B0B586B00490039103980499AA
:107260007C224A43EC498918CA69898C01901046EE
:10727000F8F730FF0199814206D3FFE73B483C49CC
:107280003C4B3D4A04F060F90498032100F078F883
:1072900002900298002803D0FFE70298059060E072
:1072A0000498FFF7C3FF0498062100F0E7F804985C
:1072B0007C210A464243D84883189C69039D9B8CD5
:1072C0006B43E31882589360049A51434018C07D81
:1072D000C009012818D1FFE704987C210A464243DF
:1072E000CD488258D36920242343D361049A0B46A6
:1072F0005343C25813680124A5052B431360049A15
:1073000051434018C466FFE70498042100F0B6F822
:1073100004987C214143C0484018C07DC009002822
:107320001CD1FFE70498154909687D22D20000901E
:1073300008461146F8F7CEFE4B21C900414300989C
:1073400000F056F80498002100F036F904987C21EA
:107350004143B148401801210161FFE70020059039
:10736000FFE7059806B0B0BDF4920102F2EB000011
:107370002AEC0000B0EB00002B020000E0B3010299
:1073800080B586B0059004910020039000F02AFC9F
:10739000029005987C2141439F48401800690028CD
:1073A000019019D0FFE7019801280AD0FFE7019862
:1073B000811E03290DD3FFE70198411F02290BD33A
:1073C0000DE0049805997C224A4393498918086185
:1073D00005E00220039002E001200390FFE70298FD
:1073E00000F078FC039806B080BDC046F49201021C
:1073F00080B584B00390029104F038F80190FFE763
:107400000398FFF7E1FEC00700280DD0FFE76420D6
:10741000FEF752FB04F02AF80199401A02998842BB
:1074200001D9FFE700E0EBE704B080BD80B584B090
:1074300003900291019204F019F80090FFE703987D
:107440007C21414374484058C06902990840019921
:1074500088420FD1FFE704F009F80099401A039918
:107460007C224A436C498918898A884201D9FFE7FE
:1074700000E0E4E704B080BDF4920102B0B588B04A
:1074800007900691079801210291029AFFF7CEFF1B
:10749000079802210191019AFFF7C8FF0798DC21A4
:1074A0000A4642435B488218069B142425465D43E6
:1074B0005219D27C05AB1A70079A0B465343C21877
:1074C000069B25465D43521992680492079A5143E0
:1074D000401806994C430019008A03A908800798B0
:1074E0007C2141434C4840187421405C01281DD147
:1074F000FFE70698012806D1FFE705A838210170AB
:1075000002200490FFE707987C214143424840183D
:107510007521405C012808D1FFE70698072804D1AF
:10752000FFE703A803210180FFE7FFE703A8018825
:10753000204A1140079ADC235343364CE318069C3B
:10754000142565435C195B59DB075B0CC91863683C
:10755000DB071B0CC918A37C5B075B0BC918049BDA
:107560009B07DB0AC918E3685B071B0AC918059B60
:107570001B06C9187C235343274AD2585160008800
:10758000002813D0FFE70798DC2141432148401829
:10759000069914224A4380184068012806D1FFE763
:1075A000079802210022FFF741FFFFE708B0B0BDB6
:1075B000F4920102FF3F000080B584B00390029175
:1075C000039801210191019AFFF730FF03980221EE
:1075D0000091009AFFF72AFF0398DC2141430D4AEE
:1075E0005118029A14235343C9188A7C5207520B2C
:1075F0008B689B07DB0AD218CB685B071B0AD21883
:10760000C97C090651187C224243F64880588161A2
:1076100004B080BDD0E30000F492010270B5A0B0C8
:107620001E901D911C921B931D98800E00280CD05B
:10763000FFE71D981B998122D204511A884204D871
:10764000FFE71B98002803D1FFE701201F90C6E148
:107650001E980421FFF794FE1A901A98002803D070
:10766000FFE71A981F90BAE11E981D991C9A1B9B60
:10767000FFF7E6F91E98FFF7D9FD1E987C214143DC
:10768000D8484018C07D4006C00F012800D08CE0CB
:10769000D54812A90A4678C878C278C878C21E9818
:1076A0007C2213464343CF48C3581C680125ED078D
:1076B0002C431C601E9B14465C4303199B6811906D
:1076C00018461092FEF76CFA1E99109A4A431199C7
:1076D0008A18926D1E9B109C5C430B19DA651E9AEA
:1076E000109B5343CA18936A13661B9A1E9B109CE7
:1076F0005C430B195A661E9A109B5343CA18002309
:1077000093661E9A109B5343CA180223D3661E9A8F
:10771000109B5343CA18D36C546DE31853651E9ADB
:10772000109B5343CA18D36C946DE31893651E9A4B
:10773000109B5343CA18936C5B1C93641E9A109B56
:107740005343CA18926C012A2ED1FFE71E980621D6
:10775000FFF794FE1E987C210A464243D6488318C0
:10776000DB6D825893601E9A0B465343C318DB6C43
:107770000F9010460E91194600F0A2F91E980E992E
:1077800041430F9842189068136E0F9C6158143152
:10779000D26C964D00950D9119460D9B0C921A4690
:1077A0000C9BFEF767FAFFE716E11E987C21414328
:1077B000F948401801218164FFE71E987C2141436C
:1077C000F5484018816C406C814200D9F8E01E9861
:1077D0007C214143F0484018006C00280B9004D0F5
:1077E000FFE70B98012815D066E01E987C210A4619
:1077F0004243E94B9A18926D1C9C1E9D694359188F
:107800004B6DE318C96C0A9111461A460A9BFFF7A3
:1078100001FBCBE01E987C214143DF484018806C7F
:10782000012828D1FFE71E987C210A464243DA4B03
:107830009A18926D1C9C1E9D0E466E439D196E6D8E
:10784000A419ED6C09911146224608932B46FFF7C7
:10785000E1FA1E99099A4A4308998A18D36C946DE3
:10786000E31893651E9A099B5343CA18D36C546D51
:10787000E31853651FE01E987C214143C648401819
:10788000816C406C814215D1FFE71E987C210A462D
:107890004243C14B9A18926D1C9C1E9D6943591816
:1078A0004B6DE318096D079111461A46079BFFF7C8
:1078B000B1FAFFE7FFE779E01E987C214143B64823
:1078C0004018806C012828D1FFE71E987C210A46C9
:1078D0004243B14B9A18926D1C9C1E9D0E466E43FE
:1078E0009D196E6DA419ED6C069111462246059303
:1078F0002B46FFF78FFA1E99069A4A4305998A1874
:10790000D36C946DE31893651E9A069B5343CA1873
:10791000D36C546DE318536547E01E987C214143B6
:107920009D484018816C406C814215D1FFE71E983C
:107930007C210A464243984B9A18926D1C9C1E9DCE
:10794000694359184B6DE318096D049111461A46A5
:10795000049BFFF75FFA27E01E987C210A4642430A
:107960008D4B9A18926D1C9C1E9D0E466E439D1960
:107970006E6DA419ED8C03911146224602932B469D
:10798000FFF748FA1E99039A4A4302998A18D38C42
:10799000946DE31893651E9A039B5343CA18D38CC6
:1079A000546DE3185365FFE7FFE7FFE7FFE71E9815
:1079B0007C21414378484018816C491C8164FCE675
:1079C0001E980021FFF7F8FD1E987C214143724864
:1079D000401801210161FFE700201F90FFE71F9879
:1079E00020B070BDF492010230E20000C5650000D5
:1079F00080B584B00A46039002A80170039806215E
:107A00000192FFF73BFD03980721FFF737FD03982D
:107A10007C214143604840187421405C012828D1F2
:107A2000FFE702A80078411E8841800103997C226B
:107A300013464B435849CB58187503981346434394
:107A4000C858002303750398424388187521405C89
:107A500001280DD1FFE703987C2141434E4842188D
:107A60007623D25C53425A41520040580275FFE7D8
:107A700011E003987C210A4642434748825800237C
:107A8000137502AA1278531E9A415200039B594360
:107A900040580275FFE70398084909687D22D20023
:107AA000009008461146F8F715FB2821414300983D
:107AB000FFF79EFC04B080BDF4920102E0B3010226
:107AC00080B586B005900491059801210191019A35
:107AD000FFF7ACFC059802210091009AFFF7A6FC85
:107AE0000598DC210A4642432A4882182723D25CA3
:107AF00003AB1A70059A51434018C069029005986B
:107B00007C214143244840187421405C012806D15F
:107B1000FFE703A83821017002200290FFE70498D4
:107B20001E4908400599DC224A431A4B9A185369AA
:107B3000DB075B0CC0189369DB039BB2C0182623DC
:107B4000D35C5B075B0BC018029B9B07DB0AC0186A
:107B5000126A5207120A8018039A120680187C22B1
:107B60004A430D4989584860049800280FD0FFE720
:107B70000598DC214143074840188069012806D157
:107B8000FFE7059802210022FFF750FCFFE706B04F
:107B900080BDC046D0E30000F4920102FF3F000028
:107BA000024800683121C9004058704784920102A0
:107BB00080B582B001200190FDF7C8FD019802F068
:107BC000D3FF002002B080BD81B00090044800685F
:107BD00000680099C8400121084001B07047C046C4
:107BE0007893010283B0EFF3108001900198009028
:107BF00068460078C007002805D1FFE7EFF3108042
:107C000072B60290FFE7009803B0704783B0EFF3BD
:107C1000108001900198009068460078C007002805
:107C200005D1FFE7EFF3108072B60290FFE70098EE
:107C300003B0704783B0EFF310800190019800907B
:107C400068460078C007002805D1FFE7EFF31080F1
:107C500072B60290FFE7009803B0704783B0EFF36D
:107C6000108001900198009068460078C0070028B5
:107C700005D1FFE7EFF3108072B60290FFE700989E
:107C800003B0704783B0EFF310800190019800902B
:107C900068460078C007002805D1FFE7EFF31080A1
:107CA00072B60290FFE7009803B0704783B0EFF31D
:107CB000108001900198009068460078C007002865
:107CC00005D1FFE7EFF3108072B60290FFE700984E
:107CD00003B0704781B0009068460078C007002864
:107CE00002D1FFE762B6FFE701B0704781B00090B4
:107CF00068460078C007002802D1FFE762B6FFE7B8
:107D000001B0704781B0009068460078C007002835
:107D100002D1FFE762B6FFE701B0704781B0009083
:107D200068460078C007002802D1FFE762B6FFE787
:107D300001B0704781B0009068460078C007002805
:107D400002D1FFE762B6FFE701B0704781B0009053
:107D500068460078C007002802D1FFE762B6FFE757
:107D600001B0704710B582B00190009101980728CA
:107D70000DD8FFE719480168019A92000F2393403C
:107D80009943009C94401C402143016020E00198ED
:107D90000F280ED8FFE710480168019A9200203A98
:107DA0000F2393409943009C94401C402143016061
:107DB0000DE008480168019A9200403A0F23934071
:107DC0009943009C94401C4021430160FFE7FFE77A
:107DD00002B010BD3C0000403800004034000040BC
:107DE00084B00390029101920398C0088000234957
:107DF000405803994907C90E07228A4090430090D2
:107E00000298002816D1FFE70398012181401C4801
:107E100002688A430260019803994907C90E8840A5
:107E200000990143009100980399C9088900134AF9
:107E3000885020E0029801280ED1FFE700980399AE
:107E4000C90889000D4A88500398012181400C48D7
:107E500002680A4302600DE000980399C90889008E
:107E6000064A8850039801218140054802688A43E8
:107E70000260FFE7FFE704B07047C0461001004012
:107E80000C01004084B0014603AA108010888007CE
:107E900000280ED1FFE703A800880121114A4243C0
:107EA000114810180222D041104A9042029114D871
:107EB000FFE703A800880B4941430B480818042139
:107EC000C8410B490122002388420193009201D34B
:107ED0000198009000980290FFE702980121084065
:107EE00004B07047295C8FC250B81E05285C8F0211
:107EF0000BD7A30010B582B014460A460146049879
:107F0000009301900820234600F092F802B010BDC3
:107F1000B0B584B014460A4601460898022500957B
:107F2000019302900720234600F052F904B0B0BD3F
:107F300070B500285BD031490A783149002A03D155
:107F40004A68012313434B60428803881B049A1834
:107F50000B46183B1A60828883891B049B180C46C9
:107F60000C3C23600B46083B84681C604469032377
:107F70002340057CAD00EB188569AD072D0D5B191D
:107F8000457C2D035B19C569AE07B60A9B19867C33
:107F9000B6059B190E1F3360036A122B04D1072408
:107FA0000C60541EA2410AE0032C05D1012D03D818
:107FB00007220A60012202E006220A600122114C17
:107FC000002525700F2464012034C57C6D022540F6
:107FD0001B069B0BD218C3791B07DB0ED2188079C6
:107FE0000007C00D101840191439086070BD06480C
:107FF00006A1862209A303F0A7FAC0464CA50102F8
:10800000181000504EA5010209F200006C73705F59
:10801000656E67696E655F72756E000050617261B2
:108020006D65746572206973206E756C6C0000005C
:10803000F0B58BB0109E34043ED00D46D64C214096
:10804000012701977F06B9423CD111462140B94230
:108050003FD11C40BC4243D1119902AC0027E781BB
:10806000E780668027802782A774E1749908A18140
:10807000A908A1800A90099708970797900880B2ED
:1080800004902046FFF754FFAA480078002801D04A
:108090000BB0F0BDAB480168C90708D10168C9073A
:1080A00005D10168C90702D10168C907F3D07F482B
:1080B000019901700BB0F0BDB8480D49AF22C14B1A
:1080C00003F042FA0095B5480949B022754B03F018
:1080D0003BFA0092B1480649B122724B03F034FAE0
:1080E0000093AE480249B2226E4B03F02DFAC0460F
:1080F000DFF10000F0B58DB00392139E340446D03A
:108100000A46A54C2140012502956F06B94244D18B
:1081100003992140B94247D11C40BC424CD114992B
:10812000129D04ACE174294921820027E781E78090
:10813000668027809908A1819108A1800B95012D67
:1081400001D16121CF43A7740C9002200A900990BD
:108150000398800880B206902046FFF7E9FE754834
:108160000078002801D00DB0F0BD76480168C9073D
:1081700008D10168C90705D10168C90702D10168A2
:10818000C907F3D04948029901700DB0F0BD83488A
:108190000D49FB228B4B03F0D7F900927F480A4927
:1081A000FC22404B03F0D0F9039800907B4806492D
:1081B000FD223C4B03F0C8F9009378480249FE22A7
:1081C000384B03F0C1F9C046ECF100008E8E000080
:1081D000F0B58BB0119E340447D00D466E4C214053
:1081E000012701977F06B94245D111462140B94286
:1081F00048D11C40BC424CD11299109F02ACE17492
:10820000294921820021E181E1806680218099084D
:10821000A181A908A1800997012F01D0712100E057
:108220006121C943A1740A90032008900790900827
:1082300080B204902046FFF77BFE3E48007800287D
:1082400001D00BB0F0BD3F480168C90708D10168F3
:10825000C90705D10168C90702D10168C907F3D070
:108260001248019901700BB0F0BD4C480C49D52261
:10827000544B03F069F9009548480949D622094B47
:1082800003F062F9009245480549D722054B03F0F7
:108290005BF9009341480249D822024B03F054F99C
:1082A000FBF1000029F20000868600004EA50102C5
:1082B00010B582B014460A46014600200093019092
:1082C00004202346FFF7B4FE02B010BD10B584B001
:1082D00014460A46014600200090019302900420B3
:1082E0002346FFF707FF04B010BD000070B50D4630
:1082F000064604242046FDF729FA204602F034FC05
:108300000B4805600B480670002E0ED00A48016825
:1083100080220A437F218A4302600120000307492B
:1083200008600749086007480460002070BDC04627
:1083300050A501024CA501020CE400E080E200E03F
:1083400000E100E01C100050B0B582B014460246B7
:108350001148204001256D06A8420DD1180413D004
:108360001748016000200093019006201146234623
:10837000FFF75EFE02B0B0BD0094FF228C320748CA
:10838000074908A303F0E0F8FF208C30421C0348A3
:1083900003490C4B03F0D8F80300FCFF09F200007E
:1083A000D1F10000447374206164647265737320BA
:1083B000257820697320696E76616C69640000001D
:1083C0000810005047F2000080B582B00B4601460D
:1083D00000200092019003200A46FFF729FE02B018
:1083E00080BD0000002801D0042100E00221C24A23
:1083F0005172411E8841800103490A6840239A4313
:10840000101808607047C04650A00050F0B583B007
:1084100002912E49CD7A0E7B771987424FD9089960
:108420000191182545434126F604BF00BE19745B2F
:1084300034490C4057033C199B07D90C6418324B44
:108440001B681B7A745375196C880326B603264083
:108450009B079B0C9B193F2404401819029CA30600
:108460001B0DC0186880012A184E13D8707B142287
:108470004243307B5023434324011B199A18F37A5B
:10848000C0181C234343D01880081E4A10400743DD
:108490000F432F800198686001F010FEA860E86823
:1084A0001A4908403030E860286908402721715C8B
:1084B0004018286100F090FD686103B0F0BDFF2214
:1084C0008832034803A108A303F03EF824A6010262
:1084D00098F200006D61635F63735F636F6E737426
:1084E0007275637400000000435320696E64657800
:1084F000206973206F7665722072616E67650D0A60
:1085000000000000FF070000289401020000F0FFB7
:10851000F0B581B0009314460D4607460626304656
:10852000FDF714F9304602F01FFB26211D48475481
:108530000021017041708171017181704171C170C0
:10854000C17102224272C16201634163816304739B
:108550004273C572009A561C134A1680017241205C
:10856000C00401214903F7F71EFE50206043290192
:10857000081861198A00801818224A438018B2B27C
:108580004A438018094940180949884204D200F03A
:10859000B5F8002001B0F0BD064807A19A2209A352
:1085A00002F0D2FF24A6010222A60102280008023E
:1085B0000120080298F200006D61635F696E6974C2
:1085C00000000000454D206F766572666C6F770D78
:1085D0000A000000A448C179002901D00120704799
:1085E000007A411E88417047F0B583B002912A4954
:1085F0004B7B834248D9CB7A0C7BE31818245C432D
:108600009B00E3184124E4041A1914240190054640
:1086100065430026565100925519EE882E4F0B46A1
:108620007A1C3240F54E3688497A711A2B4E0E402C
:10863000B618EE803740997BEF80AA88284F174004
:108640004A424A4191007918264A8918A980264F42
:108650000F402D1D029801280AD124490E400921FE
:10866000C902711869800121C9037918298000E0C5
:108670002F800198444300980019074A918C418249
:10868000118C018203B0F0BD3520C200034804A163
:1086900009A302F059FFC04624A6010298F2000087
:1086A0006D61635F6C696E6B5F646573635F636F5D
:1086B0006E737472756374004C696E6B20646573BD
:1086C0006320696E646578206973206F7665722017
:1086D00072616E67650D0A00FFFBFFFFFF0300007C
:1086E00003D0FFFFE80F0000EF1F0000FF83000032
:1086F000BE4A50639163704724A60102F0B581B071
:108700004348CC21016003214160B8490A7BD3046E
:10871000404C1B19CC7AA218541E1C4318235343F7
:1087200092009A184B7B14255D4352199201224303
:10873000012463061343436100228262C262026322
:1087400042638263C26342650267334B1A605A60B8
:108750009A60324B1A601A619A61DC61304C1C627B
:10876000304C251D1D6325460C3D5D632546283D87
:108770009D632D4EDE631C645C642C4D2F461C37BC
:108780009F642746143FDF64103C1C65284C5C65E1
:10879000284C9C650C369E67274CA5634035E563E5
:1087A000DA651A665A669A66DA661A67234DDD67D5
:1087B00002258561224DC561C325AD03CD620A63E3
:1087C000D2435A601F4A1368FF25AB4326254D5DEF
:1087D000AD072D0EEB1813601B4A102313601B4AC4
:1087E0001360272260238B5419498160C1600161A5
:1087F00021607D210901016641661649C16416495F
:1088000041641649016400F0D7FB01B0F0BDC046D9
:1088100004A000500000F8FF94A0005034A10050C4
:10882000FF185A0030040040041000401C20004093
:108830005430004060400040B8A1005014001400C3
:10884000FF3F3FFF04E400E080E200E000E100E0E1
:10885000DC05DC053F0270020133D007D007D007EA
:108860002921C64A5054704724A60102F0B58BB0A6
:10887000079208910146C14FB8780991FFF7B4FEFD
:1088800078793A7B79790691824200D89FE0FB7A29
:108890009A181823534392004124E104049152187A
:1088A000D2187B7B14214B43D218502460431558B7
:1088B00001230A93DB022E469E4316504E4B2B405B
:1088C00005937D7B03914D433E7B7443F97A0B0105
:1088D0001B195B1971181C24029461435918A84B89
:1088E0001B88069C5C430919C904490D059BC918DE
:1088F000115010180799416038787979089A0092D8
:108900000322099BFFF782FDF87A397B0918387832
:10891000814263D983000993049AD45C0894F721B7
:108920002140D154D1184D788E7836027619CB7803
:108930001B04F31807900A9886051E43330CCB706E
:10894000FB7A387BBC784D709F4D3540039E664363
:10895000C018029B4343981940029C4B03405C198A
:10896000200A8870200CC870F023089D2B401B1D26
:108970003D7B0895FE7A099D5355C8700620079ADD
:1089800050438019089A801848701F22D202224052
:108990000243100A88707879401C7871387B7979A5
:1089A000814201D3002179713978491C3970F97AF3
:1089B00008183978884201D80020387028200A9990
:1089C0003954387A401C3872387A0BB0F0BDA72081
:1089D0004200D2480649074B02F0B6FDA7204200EC
:1089E0007A32CE487349744B02F0AEFD24A60102E0
:1089F000B8F2000061F2000000F0FFFF22A60102C1
:108A00000320000605490A6882430A600A68024397
:108A10000A600348012101607047C0461C00004005
:108A20001CA0005080B50120FDF736FA80BD000083
:108A3000F0B587B006930646504C607A504B1B88C1
:108A4000181A0C9DA84200DC89E00F460592012E01
:108A500006D156480021C1620169554A8918016052
:108A6000A0783146FFF7C0FDE078E178069A2B4602
:108A700000F0AEF82078E1780097002206923346A5
:108A8000FFF7C4FCE07A217B0818217888426ED970
:108A90004120C20404918800815C0391F7250D40B8
:108AA000029285544549455C4549465C3602761933
:108AB0004449475C3F04F6190127BF0537433E0C84
:108AC0004654E67A217BA3783C4A85543E4D3D408E
:108AD00014275F4389191C234B43D91949023B4B87
:108AE0000B405D19290A364BC1542E0C35494654AA
:108AF000F02703990F400599002900D13F1D217BE4
:108B0000E37A029A87542F4A86540622049E7243BF
:108B1000D2185118294A81541F22D20215400D4300
:108B2000290A274A8154E078401CE070E07AE17815
:108B3000814201D30699E1702178491C2170217B83
:108B400008182178884201D806982070E079401CE6
:108B5000E071A07A401CA072E07907B0F0BD392026
:108B6000C2001632074808A109A302F0EDFC392023
:108B7000C20004480F49104B02F0E6FC24A6010293
:108B800022A6010298F200006D61635F7478000014
:108B90004D4143205458206C656E206973206F76D8
:108BA00065722072616E67650D0A0000080400405E
:108BB00090D00300CEF200007FF200000100080216
:108BC0000200080203000802FF07C0FF00F83F0090
:108BD000F0B589B00893019204914F4DEF7A874226
:108BE00000D891E0297B502632464A434124E304D1
:108BF0000693D218CC19A10051181822059254439B
:108C00000A19697B142307935943531802900001F2
:108C1000195804460390504A0A40A97AC9025118CB
:108C200008988205D2088A181A514C4911402A7BAB
:108C300000965643384CE57A2C0106982418A7195B
:108C4000354E5419A5007D19059844432819747BA5
:108C5000079D6C430519049FD21941480488544369
:108C60002A19089CD204520D51181D460398195018
:108C700000F0BCF90146707A001902043E460CD09F
:108C800080B2C000002900D1801E029FA5214900AA
:108C9000F7F720FA1F21014001E00021029F38016F
:108CA0002818427983791B029A18C3791B04D218B9
:108CB0002C4B1340437109045918090CC171002C45
:108CC00020D0154835460646007B009B4343F17A89
:108CD0000A01069F3A43D21841188B00D218059B0F
:108CE0004B43D118727B079B5343C91840191C4A48
:108CF0001288424388180199884203D0019922467C
:108D0000F7F738FA09B0F0BDFF225C32034804A13E
:108D100009A302F019FCC04624A6010298F2000043
:108D20006D61635F74785F646573635F636F6E73B7
:108D300074727563740000005458204445534320F6
:108D4000696E646578206973206F76657220726140
:108D50006E67650D0A000000FF0700E000F8FFFFE6
:108D600022A60102EFFFE00080B58CB000200B903E
:108D7000FCF754FAFCF78CFA01F058FE089001F069
:108D80004FFE2C4909688903C90F0A912A490968CD
:108D90008900890F09910A99002904D1FFE70998F0
:108DA000012808D1FFE7FBF779FAFCF733FA002036
:108DB000FDF7ACFA02E0FCF7D7F9FFE7FCF79EFA03
:108DC0000020079005F026F80690FEF7F1FE1B49FB
:108DD000079A0590104603F0B3FF0490FAF7A4FC3D
:108DE0001749184B6422079804F0D8F8039001F053
:108DF00049FB154A01200290029902F049FA0298B3
:108E0000800302F07DFA1148FAF742FFFFE71048AD
:108E10000078002809D0FFE70D480021017002F01A
:108E200057F80190F8F7BAFB02E0F8F7B7FBFFE755
:108E3000EDE7C0461800004030000140D894010220
:108E4000B8A5010215D200007DB200008DF100002E
:108E500077930102014800687047C0460C0000404B
:108E600081B080B585B007930490039102920020F1
:108E7000009007A8019004980399029A019B02F0C0
:108E800099FE0090009805B080BC02BC01B08E46EF
:108E9000704700207047000010B584B00020039098
:108EA0000399FDF76BFE1E49012293021D4A039CA4
:108EB0000290204601911146019AFDF7EDFF0199BC
:108EC0000A88194B9A4229D0FFE7154816490180B4
:108ED000164981807D218900C1800A2101810021FC
:108EE0004181134A82810122C28181834323C38647
:108EF00002230387782343878287C28760228152B7
:108F00006222815264228152C183442281521422FE
:108F100082825022815201F0A1FFFFE704B010BD10
:108F2000ECA0010200E00204AA5500003412000087
:108F3000E1FF000081B00090002001B07047000008
:108F400010B50024002809D0002905D003464A00A6
:108F500003481946F7F70EF9204610BDE04310BD4F
:108F6000EC920102014600200A2901DAC043704751
:108F7000014A11807047C0467493010282B00A46CC
:108F8000019068460170002002B0704780B50188EA
:108F9000064A11808178064A1170C178054A11701D
:108FA0000079FCF78DF8002080BDC04614940102C2
:108FB0001694010210A70102044805490160152119
:108FC00009044160034981607047C0469C300040FD
:108FD00041000800340007000748006840697047F6
:108FE000FD20400004490968085C70470248006899
:108FF0006221405C7047C0462894010210B50648C3
:109000000468064800686421F7F77AF80221C9432A
:109010004143081910BDC04614A7010218A7010258
:109020000A491A220A600A4948704878FF21090251
:10903000084A13688B43800380B2C018106006484A
:109040002021016005480160002070477020004029
:109050001894010204E400E080E200E000E100E096
:10906000F0B5A9B016460F460546C648002B024685
:1090700000D01A463921CC003D21C9005118119168
:109080008242189206D001204202BE491898F7F792
:1090900071F8189A6120111913910E21119C0A91EF
:1090A000A170002F0D9501D00A2100E0092159235C
:1090B00017938300E17078427841139908703078F3
:1090C00010901070F17AE17471785170B7789770E0
:1090D000F178D1703579157174795471B1799171D4
:1090E000F179D171317A1172717A5172B17A9172CA
:1090F0007E1EF0B200210328169106D870B28000BF
:10910000A1A210586A00805A1690179882001898E9
:10911000C0181490F81E022804D3012E084604D863
:109120009D4800E09D48031918781290189DA818D2
:1091300017902846303015902C4656346D2080000C
:109140002950974A974B149E33627262B362F2625F
:109150003176F182139B597009229A702818416068
:109160008160C1600161109880008F490858F7F74D
:10917000C1FB012F10900F9104D0022F05D17F2148
:109180007E2004E07C217B2001E05B215A20159D9C
:10919000A984207003200C90A080012666701F20F7
:1091A0000B90A8821820A8740A46083A179BDA7612
:1091B000169B129AD2184A439100189A9163B702EB
:1091C000791E8B420E9109D97848608034206884DA
:1091D0007748288277481399088339E07F2B10DD80
:1091E000802B18D031028B421BD071028B4227D1C9
:1091F0006E49618068846F4813990883CF20C0004E
:1092000025E0202B17D0402B1AD16848608004201D
:10921000688469481BE06548608006206884674868
:1092200015E06248608010206884624813990883C2
:10923000C520C0000BE0624860800220688404E022
:1092400004206884812040006080FF200230288252
:10925000104600F0D7FE1298102806D0402808D1FA
:1092600008201499C876072000E004201799887018
:1092700002E017980C9981701898169A8078C11E90
:1092800002290CD3022811D001280CD12672BA422F
:1092900000D900266672BA4213D8F44812E00D20B5
:1092A0000002119908800120800201E00C98000260
:1092B0002081BA4201D8EE4800E0FA201799886070
:1092C0000EE0FA2017998860139800780028119909
:1092D00001D0E8484880E848139A1083E74808809E
:1092E000A88CF7F769FA0026E54B3246F7F7ECF859
:1092F00002460B46E3493046F7F74EF9E24B324659
:10930000F7F7E2F8F7F7AAFA0746E080DF493046B8
:10931000109A0F9BF7F740F9DD4B3246F7F7D4F878
:10932000F7F79CFA78434042800B608116990E98BB
:10933000814208D90C20149FB872D64817998883A7
:109340001220189A0EE0480A189A149F01D00D2096
:1093500003E0080A00D1DBE20A98B872CE481799F8
:1093600088831220F872D078052844D87844007990
:10937000400087440227402C3339C848B881C84888
:109380002FE0C0468490010200E2000000E20000ED
:1093900010E2000010E200000CDF000013DF00000C
:1093A0003075000010270000C0DF0000050200003B
:1093B000FF060000040800000A0400003604000054
:1093C00003020000B748F881B748388013E0B74877
:1093D000F881B7483882B74838600CE0B448B881A3
:1093E000B5481799C88306E0B4487882B448B88075
:1093F0000B9800069064AE483881A748F880B148C1
:1094000002882A84B0480078E874B0480078119F38
:109410007875387D139000285ED0AD490A68102316
:10942000DA413A600A794B79CF8867801B029A1833
:109430006A840A7A4B7A8F7AC87A0D7B65701B0230
:109440009A183B04D21800061018179FF860487B42
:109450008A7BCB7B3B77120210186081087C78777F
:10946000487C149A9072887CD072C87C159B1874C2
:10947000087D5874487D11909874C87D0A7E120248
:1094800012181A84887DD87418464B7EC375887E5E
:10949000CD7E2D022818B880087F4D7F2D02281818
:1094A000F880887FB877C87FF8772020085C149D03
:1094B00028732120085C68732A20085C2A314D78C3
:1094C0002D0228188D782D044019C97809064018F6
:1094D00018998864119801E0EB7DA87C7D498B7018
:1094E0000A8080001F38C882C883139800281FD0C4
:1094F00022227748825C034622335B781B029A184B
:109500000A842422825C034624335B781B029A1867
:10951000CA842622825C034626335B781B029A1893
:109520008A832822825C2830407800028018888450
:109530006948032569A2294602F0E6FE189F38789B
:1095400014907B78B8780F90FA78B8791390F879FE
:109550001190387A1090787AB97A0890099100932E
:109560000F98019002921698039012980490139805
:1095700005901198069010980790FAA2F84829468D
:10958000149B02F0C1FE3D46643580212846F6F763
:109590000AFEB878C11E02290ED3012800D18FE13E
:1095A000022800D0ABE11691149078787F225043C6
:1095B000F7494018F74907E01691149078785B2234
:1095C0005043F1494018F14941182846F6F7D2FDB9
:1095D0000D9D1898C6870E34324602E0641C0F2A8F
:1095E0000ADA21780029F9D0491C8907C90F91406E
:1095F0000E43C687521CF1E71699022907D3149926
:10960000491E012900D97DE14279D24901E0427920
:10961000CF4989180C78002D00D177E1C1790E91DE
:10962000032900D94AE14279062A00D979E1492182
:10963000890041181191E43010900E98401E12904C
:1096400019A800190F9000231392149403E018989E
:10965000290600D15AE1052A5AD8C0467A4412791F
:1096600052009744455C728598ABC0468813000051
:10967000E20400000C080000060A0000040F0000CD
:109680000000104130C1BD41000070400000F040BA
:109690000000D041120C0000140B00001212000058
:1096A000140E00000E160000130D0000121600002C
:1096B0000E120000140B0E0A120800001016000013
:1096C0000E0B0000149401021694010210A701026F
:1096D0001CA7010280940102010800004361736528
:1096E00020706172616D65746572733A200D0A00B5
:1096F0001693DFB2002F04D019A801223946F6F7DD
:109700004BFD002C00D191E019A8C019BB498AE09B
:10971000E8B2022867D00027022867D06BE00E98D5
:10972000022872D1E8B2022800D103461693DFB2B4
:10973000002F04D019A801223946F6F72DFD002C80
:1097400074D019A8C019ACA16DE0E8B2022800D10C
:1097500004231693DFB2002F04D019A80122394642
:10976000F6F71AFD002C61D019A8C0199FA15AE084
:10977000E8B2022800D106231693DFB2002F04D0EE
:1097800019A801223946F6F707FD002C4ED019A87A
:10979000C01992A147E0E8B2022800D10C23169329
:1097A000DFB2002F04D019A801223946F6F7F4FCE5
:1097B000002C3BD019A8C019874934E0E8B2811EBB
:1097C0004A424A419700022804D119A80122394689
:1097D000F6F7E2FC002C16D019A8C0197CA122468D
:1097E000F6F7C8FC0FE00627022804D119A80122C9
:1097F0003946F6F7D1FC002C05D019A8C0198049CC
:109800002246F6F7B7FC169710E01693DFB2002F4A
:1098100004D019A801223946F6F7BEFC002C05D069
:1098200019A8C01973492246F6F7A4FC3C193F2C2D
:1098300005D80F98C0194021091BF6F7B4FC1298FF
:109840000228189801D2002002E0C078411E884109
:1098500015990870611E2E46E8B202280CD1179A9D
:10986000517019A9119AB8C9B8C2B8C9B8C2B8C953
:10987000B8C2B8C9B8C20DE0179A117019A9109AE8
:10988000B8C9B8C2B8C9B8C2B8C9B8C2B8C9B8C2EC
:10989000C10709D180073546149C139A169B00D442
:1098A000D5E602208543D2E6FE20354605401898CD
:1098B000149C139A169B290628D0CCE637A231E0D7
:1098C0001691149078780B994143334808181F3843
:1098D0006F21C9430D9D7A180378D427D355437857
:1098E000D827D3558378DC27D355002900D170E6DB
:1098F000C378E027D3551031001D189FEBE70120F6
:10990000404A10E00024002D00D087E629B0F0BDC9
:1099100080290ED30F20B872104817998883102021
:1099200020E525A20120014602F0EEFC189829B09E
:10993000F0BD1020402904D3B8720849179B9983C1
:1099400010E5B87204481799888314200AE5C046C8
:1099500013DF00000CDF0000150F0000140B0000E7
:10996000010800002564202564202564202564204A
:109970002564202564202564202564202564202575
:10998000642025640D0A000054FC00001DF7FFFF51
:109990006CF3000089FBFFFF5CFB00007472785FD2
:1099A0006D6F646520706172616D657465722065AC
:1099B00072726F720D0A00004E73666420706172DD
:1099C000616D65746572206572726F720D0A0000B8
:1099D000FFFFFFFF01FF000090E20000FFFFFFFF1D
:1099E000FF0101FFFF01FF01FFFF01FFFFFFFF017B
:1099F000FFFF01FFACE40000FFFF01FFC8E2000031
:109A000020E200000AF30000002800D101480649C6
:109A10000860704784900102F0B586B0002805D137
:109A20000148006802E0C046289401023121C900C3
:109A3000049141188A791F231A40CD79ED06AD0DA6
:109A4000AA180D7AED066D0C52194D7AED062D0B04
:109A500052198D7AED06ED095219CD7AED06AD0851
:109A600052194D7CED075219BD4C22600A7B1A40F9
:109A70004E7BF606B60DB2188E7BF606760C921962
:109A8000CE7BF606360B92190E79F606F609921978
:109A90004E79F606B608921962604A6AB14D2A40BC
:109AA000A2608A6A2A40E2602D22D20087183A7E9C
:109AB0001A4003937E7EF606B60DB218BE7EF606F9
:109AC000760C9219FE7EF606360B92193E7FF6064C
:109AD000F60992197E7FF606B60892190E7CF607F3
:109AE00092192261BA7F1A400597FE7FF606B60DDD
:109AF000B218049BC35CDB065B0CD2184B78DB0608
:109B00001B0BD2188B78DB06DB09D218CB78DB066F
:109B10009B08D2186261CA692A40A2610A6A2A4077
:109B2000E2618A7C01252A40CB7CDB079B0F9A18D7
:109B30000B7DDB075B0FD2184B7D9B07DB0ED2182A
:109B40008B7DDB079B0ED218CB7D1B079B0D9A18D4
:109B50000B7E1B079B0CD2184B7E5B06DB0A134364
:109B60008A7E520612091A43CB7E5B075B081343B9
:109B70002362CA6A62620A6BA2624A6BE2628A6B01
:109B800022633922D200835C1E462E4066635E4209
:109B90005E41B304AE04744F3C68B443E3183B60C9
:109BA00083185A782A409C782407E40EA2188C8FD8
:109BB0006401A2186D4C1440C98FC905490A0919DE
:109BC000DA78D207120A89181A7912071209891845
:109BD0005A79D207D2088918FB4EB1639968F163AC
:109BE000997904952940DA79D207920F51181A7B96
:109BF0005207D20E89185A7BD206920D51189A7BC1
:109C00005207D20C8918DA7BD206920B89181A7C7B
:109C1000D206520A89185A7C520792090A43997C43
:109C2000C906490851183164D97C039A11401A7D3C
:109C3000D206920D51185A7DD206520C89189A7D7F
:109C4000D206120B8918DA7DD206D20989187164FE
:109C5000197E0F2421405A7E120151189A7E120358
:109C60008918DA7E1207120A51181A7F1207120990
:109C700089185A7F12078918B164997F019421408D
:109C8000DA7F1207120E51183D22D200835C5B0767
:109C90005B0D5918841862781207520C8918A27843
:109CA000D206120B8918E278D206D2098918F1641B
:109CB000217907220A406179C9008918A2795206E0
:109CC000920B5118E2799207120B8918227AD20767
:109CD0008A18BF490A60627AA37A1B029A18E37A4B
:109CE0001B04D2184A60E289BA4B13400394228ABB
:109CF000D2049209D2188A6003463033598CB64A8E
:109D0000114002939A8CD205D20A51185622825CD5
:109D100012068918B14D2960014656314A788C786F
:109D20002402A2188C8864056409A218CC78240740
:109D300012196A60CA880C7AA407A40BA2184C7A7C
:109D40006407E40A1219AA604989E9604921890077
:109D50004118FF226632821800921035002207E077
:109D600000300040FFFFFF0004040040FF3F000000
:109D700084186427E65D03273E406523E35C9B0768
:109D80001B0F9B196626A65DB607B60EF31867264D
:109D9000A65DB601F318DBB26826A65DB607B60D60
:109DA000F3186926A65DB607360DF3186A26A65D78
:109DB000B607B60CF3186B26A65DB607360CF3187B
:109DC0006C26A65DB607B60BF3186D26A65DB60722
:109DD000360BF3186E26A65DB607B60AF3186F2683
:109DE000A65DB607360AF3187026A65DB607B60953
:109DF000F3187126A65DB6073609F3187226A65D1C
:109E0000B607B608F3187326A45DA407E31808C5BF
:109E10001032802AACD1019AD243704EB4180B781C
:109E20003B404D78AD072D0FEB188D78AD07AD0E8B
:109E3000EB18CD78AD01EB18DBB20D79AD07AD0DA8
:109E4000EB184D79AD072D0DEB188D79AD07AD0CE5
:109E5000EB18CD79AD072D0CEB180D7AAD07AD0BD6
:109E6000EB184D7AAD072D0BEB188D7AAD07AD0AC7
:109E7000EB18CD7AAD072D0AEB180D7BAD07AD09B8
:109E8000EB184D7BAD072D09EB188D7BAD07AD08A9
:109E9000EB18CD7BAD07EB18A3641031121DBDD1BB
:109EA000009B19785A785207520D51189A78D207A8
:109EB000120D8918B164059B1968F164D97D5A683F
:109EC0001202511831659968454A0A40998A490534
:109ED00089187165D9683D4C2140B16519692140E7
:109EE000F165029E3178049D294082785207120F55
:109EF0005118C2799207920E8918427A9207920DF0
:109F00005118827A9207120D8918C27AD207920CE0
:109F100089189A7DD207520C891872789207D20B51
:109F20008918B2781207D20A8918F2781207D20972
:109F30008A182C490A60327C737C1B071B0D9A1807
:109F4000B37C9B069B0BD218F37C1B079B0AD21891
:109F5000337DDB065B09D218737DDB071B09D21842
:109F60004A60B27D2A40C38F5B009A188A60826C77
:109F7000CA60C26C22400A61F27D7F231340328C9A
:109F80005204520AD2184A6102698A614269CA615E
:109F900082690A62C2694A62026A8A62426ACA6263
:109FA000826A0A63C26A4A63039A927CD201121DD2
:109FB0000A64027A3A40CA65808F074A10400866F0
:109FC000002006B0F0BDC04600300040FFFFFF009B
:109FD0009C300040FF1F0000FF03000000400040D5
:109FE000FFFF1F000020004004480068806B8008CD
:109FF0000349096849004018093070472894010254
:10A000001004004010B52D21C9004118027A032A1E
:10A0100004D10079002807D0082006E08378DA1EF2
:10A02000022A05D2032412E0142088601C203DE09F
:10A03000012B02D1C8228A6012E00479042C01D3DA
:10A04000462404E0032C01D1322400E014248C6067
:10A050005B1E022B04D3022A10D24279154B01E079
:10A060004279154B9B181B78402B04D0102B06D13E
:10A070001423442405E02A233E2402E042793423B9
:10A0800048244B800C80022A06D0062A08D0052AD4
:10A0900008D118224C2301E0142250230B8000E049
:10A0A0001C224A80C078042803D1142048806420F0
:10A0B000088010BD13DF00000CDF000013480068AB
:10A0C0007047C04610B5104A107091700F490028B3
:10A0D00013D050680861042048619078FF22120272
:10A0E0000B4B1C689443800380B200191860012058
:10A0F0004007084A1060084A1060002008600749BD
:10A1000001220A6010BDC0461894010218040040E4
:10A110001CE400E080E200E000E100E070000040AC
:10A12000F0B591B0002801D1C04800688778F91EC9
:10A13000022913D3012F21D0022F3CD11021CA4371
:10A1400044782146193991423DD800970125B94AF2
:10A1500028462946234602F0D7F853E10821CA438E
:10A16000447821462139914218D800970125B14AF7
:10A1700028462946234602F0C7F843E10821CA438E
:10A18000447821460939914234D800970125A94ADB
:10A1900028462946234602F0B7F833E1032F3CD086
:10A1A000042F43D1C3780125042B00D02DE10646AE
:10A1B0002A02042343E00125A6A2284629463B465D
:10A1C00002F0A2F81EE1C3780125052B0AD8064645
:10A1D0002A02284698401B21084230D10021052B35
:10A1E00008462ED002200090914A2846294602F0C7
:10A1F0008BF807E10646C3780021022B1ED3032B00
:10A200001CD0042B08460A461BD001250095884A1D
:10A210002846294602F078F8F4E0C3780125032B9C
:10A2200000D0FAE006462A02032308E0012583A2B3
:10A23000284629463B4602F067F8E3E00A4601213A
:10A2400048020F91592189007518FD2149007118A4
:10A250000291314662313F05D219641E1F27274003
:10A260005C013C191443044332795207D20C224357
:10A270002B789B065B0BD218B379DB071B0B1343C0
:10A280006D4D2B60F279032310931A40737A9B076C
:10A290009B0E9A18B37A5B07DB0D9A18F37ADB07EB
:10A2A0009B0DD218337BDB075B0DD218737B1B072A
:10A2B0005B0CD218AA603269EA6072692A61B269DD
:10A2C0006A61F269AA61326AEA61726A2A62B26AF2
:10A2D0006A620F980870F06AA8623F20C4432C3568
:10A2E0003046E4300F903046E5300E903046E63090
:10A2F0000D903046E7300C903046E8300B903046F9
:10A30000E9300A903046EA3009903046EB30089048
:10A310003046EC3007903046ED3006903046EE3057
:10A3200005903046EF3004903046F03003903746C9
:10A33000F1373046F230F3360F990A194021525C5A
:10A34000109B1A400E9B1B195B5C9B071B0F9A18F6
:10A350000D9B1B195B5C9B079B0E9A180C9B1B1992
:10A360005B5C9B019A18D2B20B9B1B195B5C9B0731
:10A370009B0D9A180A9B1B195B5C9B071B0D9A1877
:10A38000099B1B195B5C9B079B0C9A18089B1B196C
:10A390005B5C9B071B0C9A18079B1B195B5C9B075C
:10A3A0009B0B9A18069B1B195B5C9B071B0B9A184F
:10A3B000059B1B195B5C9B079B0A9A18049B1B1946
:10A3C0005B5C9B071B0A9A18039B1B195B5C9B0732
:10A3D0009B099A183B195B5C9B071B099A18031988
:10A3E0005B5C9B079B089A183319595C890789188D
:10A3F00002C51034A0D102980078042101430E4810
:10A40000C1630025284611B0F0BD04200090084A21
:10A410002846294601F078FFF4E703200090044A1B
:10A420002846294601F070FFECE7C0462894010257
:10A43000DFF2000025F3000000100040556E646557
:10A4400066696E6564206D65616E205052462025F8
:10A45000640D0A00496E76616C6964206D65616EF9
:10A46000205052462025640D0A00000081B00146AC
:10A470006A46107001B0704781B001466A4610709C
:10A4800001B0704780B5124800688000002806D5EA
:10A49000FFE710480168114A1143016005E00D48CB
:10A4A00001680D4A11430160FFE70D480168082269
:10A4B00091430160012040040A4908600A4801688C
:10A4C0000322920491430160FAF702FF80BDC04667
:10A4D000200000402C000040800000802000008010
:10A4E00004020040000200402800004080B582B015
:10A4F0000190FDF79FFB0090019820490A68824374
:10A500000A6001984A6882434A6001988A688243D7
:10A510008A600198CA688243CA6001980A698243C6
:10A520000A610098FDF7EEFB02B080BD80B584B0F3
:10A5300003900291FDF77EFB019003980F490A6892
:10A5400082430A6003984A6882434A6003988A6893
:10A5500082438A600398CA688243CA6003980A6982
:10A5600082430A610398029A92008B5803438B50EE
:10A570000198FDF7C7FB04B080BDC04678A7010273
:10A5800080B582B022480168019101990322120727
:10A59000914301910199012252071143016000206A
:10A5A0000090FFF769FF0098FFF760FF8020FFF73A
:10A5B0009DFF02B080BDC046B0B586B00A460346D6
:10A5C00005AC207004A8017011480168039103993B
:10A5D00003252D0729430160802001210292019368
:10A5E0000094FFF7A3FF00980178002904D0FFE74B
:10A5F0000120FFF741FFFFE704A80078002804D0FE
:10A60000FFE70120FFF732FFFFE706B0B0BDC0460D
:10A610000004004082B0019000910098012808D108
:10A62000FFE70198012181400E4802688A430260D9
:10A630000CE00098002808D1FFE701980121814033
:10A64000084802680A430260FFE7FFE7019801211A
:10A650000A468240044803681A43C9070A43026055
:10A6600002B070474400004040000040032804D876
:10A6700040000649085A00B27047002000B27047F7
:10A68000032802D84000014A115270478CA70102EA
:10A690009E4908707047C04670B58AB00C460546A2
:10A6A000FF20FC30A8490E68315C59208000335CE3
:10A6B000B278307808AE069609AE05960C4E049630
:10A6C0002126760603960B4E0296012601960E264B
:10A6D00000965B1CDBB2F8F76BF80998F6F790F878
:10A6E00028700898F6F78CF820700AB070BDC04644
:10A6F0000000204100000443F0B58BB00446457CC7
:10A70000824800788249002822D000200880814AAF
:10A710001080814B01269E761E830A907F48007828
:10A720007F4E36786DB205957E4D04957E4D03952E
:10A730000AAD02957D4D01950096F7F777FD0A9DCC
:10A74000112020567A497B4A00F012FE064626E088
:10A7500000260E806F4A16806F4B01209876188372
:10A7600009966E4800786E4F3F786DB205956D4D35
:10A7700004956D4D039509AD02956C4D01950097BB
:10A78000F7F754FD099D112021567F20C005009048
:10A7900001900296664A674B3046F8F79BFE4320CD
:10A7A00001062846F5F763FDF6F72AF80890624897
:10A7B0000078002824D05120800060494A7D42431F
:10A7C0008D185F480068A8642F46403750480078CD
:10A7D000B87450480078F874554800783875554872
:10A7E0000078787557480078F87550480069F6F792
:10A7F00007F8B87552484069E8644C4800686864D6
:10A80000FF20FE3050490968085C3922D2008918BF
:10A81000022812D303D04E48007801280DD14B48AE
:10A820000660434800883A4A108042480088394A06
:10A83000108009200790089605E04448089A0260B5
:10A840003548C08B07900B780022002B01D01146B1
:10A8500000E0D1430125002B01D0042300E0EB43AD
:10A86000A67AAD1BEE175B1971416568AE0F277AAA
:10A87000AD00ED195641677A3F1FF817ED19704189
:10A880004000EE0F80196D00EB1848418001990ED1
:10A890004118980127239B02C31A91411D4805883E
:10A8A0001B480088854201D00798421B1020205683
:10A8B000C001194D2D8C032D07D1E468E5176D0AF1
:10A8C0006419E4150519EC170FE0E468E5176D0A43
:10A8D0006519EC17ED15C6174519744197B2002F8D
:10A8E00000D03446002F00D00546581BA141130468
:10A8F00009D012B2D2015242D31780185941089B95
:10A90000DA17C01A91410BB0F0BDC0467693010230
:10A91000F4A40102F2A401028094010275900102E4
:10A9200074900102989A010298980102F8A4010219
:10A9300042A5010240A50102749E0102AC9B0102E6
:10A9400064200040F0A4010228940102ECA401025A
:10A9500044A5010280B584B003900398FFF7CCFEB4
:10A96000019100902D48007BFFF780FEC10F401839
:10A970004110C017019A009B591A8241009101921F
:10A980000098019904B080BDF0B587B01C4615460B
:10A990000E46074603910290019300920398029994
:10A9A000019A009BC91A90410CDAFFE701980099BF
:10A9B000039A029B591A8241012040021018049107
:10A9C000059008E003980299019A009BC91A9041EA
:10A9D00004910590FFE70498059907B0F0BDC10DFB
:10A9E000400280307047000080B584B00390039827
:10A9F000FFF7F5FF019100900848007BFFF736FE56
:10AA0000C10F40184110C017019A009B59184241CC
:10AA1000009101920098019904B080BD76900102E6
:10AA20000120C007464908607047C04680B584B021
:10AA300043480068029002A80078C007002808D0A8
:10AA4000FFE7484A0220032101F05EFC0121039147
:10AA500072E002A800788007002809D5FFE7404A85
:10AA600002200321019001F04FFC0199039163E062
:10AA700002A800784007002809D5FFE7374A0220DE
:10AA80000321009101F040FC0099039154E002A8D9
:10AA900000780007002808D5FFE72F4A022003218D
:10AAA00001F032FC0421039146E002A80078C006C0
:10AAB000002808D5FFE7274A0220032101F024FCE3
:10AAC0000521039138E002A800788006002808D507
:10AAD000FFE71F4A0220032101F016FC0621039123
:10AAE0002AE002A800784006002808D5FFE7174AA8
:10AAF0000220032101F008FC072103911CE002A8B9
:10AB000000780006002808D5FFE70F4A022003213D
:10AB100001F0FAFB082103910EE0FFE7FFE7FFE7F2
:10AB2000FFE7FFE7FFE7FFE7064A0220032101F006
:10AB3000EBFB00210391FFE7039804B080BDC04602
:10AB40005C00004023ED0000B3EC0000E4EC0000EA
:10AB50003DED0000D2EC000014ED0000C3EC00005D
:10AB6000F6EC000005ED000081B0009000981F2871
:10AB700008D1FFE70098012181400A4802680A4392
:10AB800002600DE0009801210A46824005480368F2
:10AB900093430360009A914002680A430260FFE712
:10ABA00001B070471C00004010B586B00A4603464D
:10ABB00005AC207004A8018021780F4C0919491EAA
:10ABC00009780088039202930191FDF75BF9002157
:10ABD0000028009107D0FFE705A80078801E4142B9
:10ABE00048410090FFE700980121084001990818AA
:10ABF000C0B206B010BDC046B0E9000080B590B04C
:10AC00000F900E910F9849490991F5F763FA0B904F
:10AC10000B98099941430F98401A0F900B98FF2108
:10AC20006E310891F5F76CFA414940180CA908807B
:10AC3000088808994143401E820F821892106423AD
:10AC40000790069119460592F5F75AFA0599081AE0
:10AC500019210901079A04901046F5F751FA049951
:10AC60000818069908180B99081A324940180B90D1
:10AC70000B9800280ED5FFE70C98401E0CA9088001
:10AC80000888FDF7FFF80B994018FF216E31401836
:10AC90000B90FFE70C980E9908800DA80121017018
:10ACA000FFE70DA800780B281ADCFFE70B980DA929
:10ACB00009780CAA1288039008461146FFF774FF22
:10ACC0000399081A0A900A98002801D5FFE707E0BF
:10ACD0000A980B90FFE70D98401C0DA90870E0E75B
:10ACE0000D980E9988700B98401C0E99C8700F989B
:10ACF000E12109010291F5F7EDF90E9908710E981D
:10AD00000079029941430F98401A0F900F983C2107
:10AD10000191F5F7DFF90E9948710F980E994A796C
:10AD2000019B5343C01A887110B080BD805101004F
:10AD3000B2070000A7FA0A0010B58CB00B90FFF71D
:10AD40001FFC0B98808A344908800888002851D15C
:10AD5000FFE70B98C08A324908800B9880690A88FF
:10AD60003249099008460999F5F704FA0B990890B9
:10AD70000846FFF7EFFD2E4A51601060FFF79EF97D
:10AD80002C4908602C480168491C01600790FEF7B7
:10AD900035F92A4908600868FAF798F928490860DF
:10ADA00008682849496A06900846F5F7A3FD264A2F
:10ADB000264BF5F789FBF5F751FD069905900846F6
:10ADC0000599F5F79DF90A900A98FAF7EBFB2048E8
:10ADD0000368079801681F4A146852680392029436
:10ADE00000911D4A0321084601F08EFA0D49012207
:10ADF0000A700EE00B98808A0849088008480021F4
:10AE00000180084802210170FFF758F906490860DF
:10AE1000FFE70CB010BDC04658A801025AA80102B5
:10AE200056A8010298A70102B4B40102C0A701020A
:10AE3000B0A70102B0B40102A0A70102E4A0010280
:10AE4000E8A00102C0DF00008DEDB5A0F7C6B03E5E
:10AE500060A70102809E01029BF1000010B588B03E
:10AE600000200590FEF715F8002803D0FFE7012029
:10AE7000069026E0EFF3108072B607900020049051
:10AE80000499FBF77BFE05900598002815D1FFE794
:10AE90000120020300210C4B039008460291194641
:10AEA0000193FBF7B1FC094A03998B02029C0090C5
:10AEB00020460199FCF7B2FBFFE762B605980690C1
:10AEC000FFE7069808B010BD00E00204ECA0010204
:10AED00010B598B002F044FDC5494A781490104668
:10AEE000139102F0ADFBC348818815AA91800188B7
:10AEF00040880004401815901046FEF747F8139953
:10AF00000A784B78092B129203D1FFE700201190A9
:10AF10000CE0B748407801210222052810920F91D9
:10AF200001D010980F900F981190FFE71198B24937
:10AF3000081841791298C0B2AD4A531C0E921A46B5
:10AF400002F0C6FC0E994A7A0D901046FFF7A0FB5E
:10AF5000AA48AB49FDF7CCFB02F050FDA9480021FF
:10AF60000170FFF7ABF8C32189014018A6490860BA
:10AF7000A648007880000D300B68A54A01240C908B
:10AF800010460C9A0B911146224602F051FEA1493F
:10AF900008600B9801680A91FFF726F80A990818CB
:10AFA000FFF722FD9C4A51601060FFF787F89B492C
:10AFB0000860FFE7FDF70EFB002801D0FFE7F9E787
:10AFC000FFF77CF8964908608F480068954940185B
:10AFD000954908600868954908607D2002010020B5
:10AFE0000990099902F068FD8A490860FFF766F840
:10AFF0008F49086085480078C322120242438D4879
:10B0000010188D4A10600868116840188B49086054
:10B010000868401C002805D1FFE788480168491CE2
:10B020000160FFE7FFF74AF885490860FFE78448B9
:10B0300000688249096801228842089211D3FFE71B
:10B040007F4800687D4909687E4A891801220023EB
:10B0500088420793069201D80798069006980890B0
:10B06000FFE70898C007002800D1B4E0FFF726F8F2
:10B0700073490860FFF722F869490860FFE7FDF7A8
:10B08000A9FA002801D0FFE7F9E7FFF717F86E49A2
:10B0900008606E480078012800D082E06B480021EB
:10B0A00001706B48407A21287AD1FFE7694801781E
:10B0B00040780002401866494A798979090289185E
:10B0C00081426DD1FFE76248007863490978884280
:10B0D00066D1FFE75E488178604A51704078107011
:10B0E0005F480078002820D1FFE75C48008860496D
:10B0F00008804648012101705E48052101705A48C8
:10B1000003685A4800684449096802910190504810
:10B1100001462231009101461A311E30002205906D
:10B120001046059AF8F7C8FD32E04C480088F6F75B
:10B1300083F94C49088008784B4A13684B4A1268D7
:10B14000354C246802940192414A144622340094FA
:10B1500014461A341E3204912146F8F7ADFD0498C6
:10B1600001883F4A127891420CDBFFE727480178BB
:10B17000491C0170394800883A49098849003C4A0D
:10B180005052FFE7374800883A4905220A54FFE742
:10B190002F489621F5F707F8374800210180FFE78F
:10B1A00019E02A480078022813D1FFE72748002138
:10B1B00001707D200201084602F07EFC15490860FE
:10B1C000FEF77CFF20490860FEF778FF134908600E
:10B1D000FFE7FFE72BE7104841680068F5F708FF35
:10B1E000F5F7B2FEF8F7FCFB179818B010BDC04693
:10B1F0007690010218DF00003898010229C600008D
:10B2000039AD0000C8B401025CA70102C8A6010262
:10B210004CBE0102CCB4010270A70102B0B401021D
:10B22000B4B40102A06D01009CA70102C4B40102E4
:10B2300060A8010280E7010058A70102889E010270
:10B24000A89B01020026B803B8B4010298A7010226
:10B25000C0A70102789E010245A5010294A7010240
:10B2600048A5010296A70102B0A70102D0B40102CD
:10B27000CAA601028C9E010256A8010282B001906A
:10B28000009102480121017002B0704777930102DA
:10B2900010B586B0034605AC2070049103921120CE
:10B2A00002930194FAF752FA2548042101600398A9
:10B2B000214908610198027801231A408A60049AA2
:10B2C0000A60896800290CD0FFE703200221009062
:10B2D000F9F772FC0098F9F7ADFA0098F9F732FB2C
:10B2E000FFE71A200221FFF795F906B010BDC0460E
:10B2F00081B0009000981049C86001B07047C04606
:10B3000010B584B0039003980B49CA6842430B4BB5
:10B310000290104601911946F4F7F2FE02990818BE
:10B32000019A50600648002303605368054C23606F
:10B330001368036004B010BDC094010240420F00C6
:10B340002C1001402010014000480047C1000000BF
:10B3500080B582B0019005480068C06D01990090E9
:10B3600008460099884702B080BDC046009001029F
:10B3700080B582B013460A4600900348011D034879
:10B38000F8F754F802B080BD9CA80102BC970102F6
:10B3900080B584B0039003980F49884206D3FFE735
:10B3A0000E480F490F4BE62200F0CEF80398401EDE
:10B3B0002B4908600020C143032202900846114631
:10B3C0000192F9F7C1FB2748029901600648019AEA
:10B3D000026004B080BDC046010000018AEC00009C
:10B3E000A4EC000070EC000010E000E080B586B036
:10B3F000FCF70CFC05901948006804901848006898
:10B40000401C03901748006802901748006801210B
:10B410008906084001900198002806D0FFE70498AB
:10B42000401C04900398029007E00298002803D182
:10B43000FFE703980290FFE7FFE704982921C9007E
:10B4400041430398029A801A08181E214143009133
:10B450000598FCF74BFC009806B080BDCCB3010208
:10B4600014E000E018E000E004ED00E080B500200A
:10B47000FAF75EFC404280BDB0B58EB0194808A90D
:10B480000A4638C838C238C838C200200690FAF7D1
:10B4900059FC0B99069A05901046FAF7EBFC0998AF
:10B4A000002803D1FFE7012004900CE00998012156
:10B4B0000902102201280391029201D00398029000
:10B4C00002980490FFE7049807A9088002200191E0
:10B4D000FAF776F901990988F4F7FCFD024908604A
:10B4E0000EB0B0BD20DF0000E0B3010282B00090DA
:10B4F00068460078C007002803D1FFE700200190CC
:10B500001BE00098002808D0FFE768464088022822
:10B5100003D8FFE7012001900FE000980849884216
:10B5200008D3FFE700980749884203D8FFE70120C6
:10B53000019002E000200190FFE7019802B07047FF
:10B5400001000003FFFF010390B00E900D910C92DB
:10B550000B93FCF783FBEFF310810F910F990A9186
:10B56000694609917146089110A907910B9A079BAA
:10B570000F49091D0124E402059008460491214663
:10B5800000F018FB069006980021049A11540A98BE
:10B590000999089A0E9B0D9C0C9D049E029601959C
:10B5A0000094F9F78BFB00F005F800F023F8C04693
:10B5B000E8B4010280B582B000200190FFE7019855
:10B5C000002812D1FFE70198800009490858002897
:10B5D00006D0FFE701988000054908588047FFE73B
:10B5E000FFE70198401C0190E9E702B080BDC0462A
:10B5F000E4B4010282B009480C2100F0E1FD1E21F3
:10B6000001900846FFF7B0FAFFE700BF00BF00BF98
:10B6100000BFFFE701200028F7D1FFE7DCED0000C5
:10B62000B6B03590359834903498FE49816600F074
:10B630003DFA002033903398FB49091D0A18012375
:10B64000DB02181A2D912C922B932A90FFF7CEFE35
:10B65000F64A2C99299008462A99299BFDF700FC67
:10B6600033990818339033982D990A182B9B191A7F
:10B670003498C06C3F242040F64D289010462A464E
:10B68000289B2794FDF7ECFB3399081833903399E6
:10B690002D9800F095FD3499CB6BEF4A2D992690AB
:10B6A00008462B99FDF7DCFB33903498006C279902
:10B6B000084032903298002811D1FFE73398E449CE
:10B6C0000918091D0122D202101AE54A25900846E0
:10B6D0002599FDF7C5FB33990818339011E033988D
:10B6E000DB490918091D0122D202101A329BDB4ADC
:10B6F000249008462499FDF7B3FB3399081833903A
:10B70000FFE73399D248001D00F05AFD0021309127
:10B71000FFE730980C281BDCFFE730983499820053
:10B7200089580091CA49091DDF4A0123DB02239091
:10B73000084622911946239BFDF792FB33903399DB
:10B74000229800F03DFDFFE73098401C3090E0E784
:10B750003498436BBE48001DC24A0121C9022190A2
:10B760002091FDF77DFB3390339821990A18209B97
:10B77000191A3498836BBC481F9010461F9AFDF726
:10B780006FFB3399081833903399219800F018FD16
:10B7900034990B6CB54A21991E9008462099FDF703
:10B7A0005FFB3390339821990A18209B191A34981B
:10B7B000006CC30F4400E40F8500ED0FC000C00F04
:10B7C000029001950094AA481D9010461D9AFDF71D
:10B7D00047FB339908183390339821990A18209B16
:10B7E000191A3498006C3F242040A24C1C9010463B
:10B7F00022461C9BFDF734FB33990818339033998C
:10B80000219800F0DDFC34994B6C9B4A21991B90E8
:10B8100008462099FDF724FB3390339821990A18A4
:10B82000209B191A3498836C94481A9010461A9ADF
:10B83000FDF716FB3399081833903399219800F0DF
:10B84000BFFC34996422895C490700291DD5FFE7B4
:10B850003498036ED148001D894A0121C90219900C
:10B860001891FDF7FDFA3390339819990A18189B2F
:10B87000191A3498C36D834817901046179AFDF72C
:10B88000EFFA3399081833901CE03498C36DC3481D
:10B89000001D7B4A0121C90216901591FDF7E0FABF
:10B8A0003390339816990A18159B191A3498036E19
:10B8B000744814901046149AFDF7D2FA3399081878
:10B8C0003390FFE73398B549091D0A180123DB02BD
:10B8D000181A349C646E6C4D13901046139A129192
:10B8E00011462A4611932346FDF7BAFA33990818F0
:10B8F00033903399129800F063FC3499CB6C634A0F
:10B900001299109008461199FDF7AAFA33903398CE
:10B9100012990A18119B191A3498036D5C480F90FC
:10B9200010460F9AFDF79CFA339908183390339814
:10B9300012990A18119B191A3498436D55480E90A4
:10B9400010460E9AFDF78CFA339908183390339805
:10B9500012990A18119B191A3498836D4E480D904C
:10B9600010460D9AFDF77CFA3399081833903399F5
:10B97000129800F025FC3499496B032291433191D0
:10B9800046492F9100212E91FFE72E9800211F2874
:10B990000C9111D8FFE72E9880003499496B40181C
:10B9A0002F990122002388420B930A9201D30B980E
:10B9B0000A900A980C90FFE70C98C007002824D042
:10B9C000FFE731982E9989004218405851689368D2
:10B9D000D46803940293019100907048001D31498E
:10B9E0000123DB02099008911946089B07921A4629
:10B9F000079BFDF735FA33903399099800F0E0FB87
:10BA0000FFE72E98001D2E90BFE73498406B2F99CA
:10BA1000091A234A914206900AD3FFE70120C00287
:10BA200005900BE022224B4DE8B40102D2ED00005C
:10BA30002F983499496B401A0590FFE705988108C3
:10BA40003222069800F0FCFBFFF7B4FDFFF7D2FDB1
:10BA5000E8B4010205EE000064EF0000FAEE000019
:10BA600011EF000084EE0000A6EE0000C8EE00001A
:10BA7000E1EE0000BCEE00003CEE00004BEE0000EA
:10BA800078EE000083EE00005AEE0000B0EE0000F9
:10BA90008EEE00009BEE0000B5ED000000F8020203
:10BAA0000108000020EE0000D4EE0000B0B588B020
:10BAB0003A480068002805D0FFE7384800680128A8
:10BAC0000ED1FFE735480068411E88410790FFE727
:10BAD000079801F07FFD002801D0FFE7F8E706E0B6
:10BAE0002E480068022801D1FFE7FFE7FFE7FCF7D7
:10BAF000B5F80690FFE729482949415A294A805A52
:10BB0000814241D0FFE725482549415A254A805ABC
:10BB1000814209DDFFE721482149415A214A825AE1
:10BB2000891A224A815208E01C481E49415A0122C2
:10BB3000D202511A1D4A8152FFE718481949425A48
:10BB40008218121D0592194A835A0493059B049C7E
:10BB50000390184602912146019200F031FB0399AF
:10BB6000019A8B5A029C0D5BEB180B530B5B012562
:10BB7000ED02AB4207DBFFE708480A49425A0C4B8B
:10BB8000D2184252FFE7B6E7044807490022425460
:10BB90000698FCF7C3F808B0B0BDC046E8B401028F
:10BBA000080800000A0800000F0800000C08000048
:10BBB00000F8FFFF80B59AB019931890179116926C
:10BBC00018980D9017980E9000200F901090FFE796
:10BBD0001698007815A908701698401C16900878D9
:10BBE000002801D1FFE7E1E115A80078252800D061
:10BBF000D1E10020129001201490FFE71698007800
:10BC000015A90870087823380D2809902BD80998B1
:10BC100078440079400087441E26262626262626BC
:10BC200016260626260E1298012108431290169811
:10BC3000401C16901AE012980221084312901698A0
:10BC4000401C169012E01298042108431290169896
:10BC5000401C16900AE0129808210843129016988A
:10BC6000401C169002E000201490FFE7FFE71498B4
:10BC70000028C3D1FFE700201190FFE71698007855
:10BC800015A908700878302805DBFFE715A80078AB
:10BC90003A2801DBFFE70FE01698401C1690119838
:10BCA0000A21414315A80078401830381190FFE769
:10BCB00001200028E2D1FFE70020139016980078B9
:10BCC00015A9087008782E2823D1FFE71698401C84
:10BCD0001690FFE71698007815A9087008783028A4
:10BCE00005DBFFE715A800783A2801DBFFE70FE046
:10BCF0001698401C169013980A21414315A8007805
:10BD0000401830381390FFE701200028E2D1FFE708
:10BD1000FFE71698007815A90870FFE715A80078C6
:10BD20006C2805D0FFE715A80078682808D1FFE740
:10BD30001698401C16901698007815A9087000E017
:10BD400004E0FFE701200028E8D1FFE715A800780C
:10BD500025385328089000D918E108984000C046BB
:10BD600078448088400087440C01110111011101C1
:10BD70001101110111011101110111011101110133
:10BD80001101110111011101110111011101110123
:10BD90001101110111011101110111011101110113
:10BDA00011011101110111011101AD001101110168
:10BDB00011011101110111011101110111011101F3
:10BDC0001101110111011101110111011101800075
:10BDD00011011101110111011101110111011101D3
:10BDE00011011101530060001101AD001101110199
:10BDF0001101110111011101110111011101F900CC
:10BE00001101110190001101700011011101800058
:10BE10001998011D19910068149014980CA90870C4
:10BE200009780DA8F8F796FCB1E01998011D199151
:10BE3000006814901499139B1198129A0192009023
:10BE40000DA80A22F8F7B0FAA1E01998011D19917E
:10BE5000006814901499139B1198129A0192009003
:10BE60000DA80A22F8F792FB91E01998011D19918B
:10BE7000006814901499139B1198129A01920090E3
:10BE80000DA81022F8F782FB81E01998011D199185
:10BE900000680B90FFE70B98007815A908700B98C5
:10BEA000401C0B900878002801D1FFE709E015A895
:10BEB00001780DA8F8F74EFCFFE710980028EAD5A6
:10BEC000FFE764E01998C01D072188430146083147
:10BED000199101684068079008460799F4F71EFD1C
:10BEE0000A900A980021F4F7EBFB002805D1FFE740
:10BEF0000DA82D21F8F72EFCFFE70A98F4F780FC37
:10BF0000F9F77CF814901499139B1198129A0192E6
:10BF100000900DA80A2206900592F8F745FA2E2106
:10BF20000698F8F717FC0A982449F4F7A0F9F4F7F3
:10BF300067FCF9F763F8149014982149F4F7E0F8D6
:10BF400014911499119A129B019300920623069A58
:10BF500004901046059AF8F727FA18E01998011D81
:10BF60001991006814901499002001900820009005
:10BF70000DAA1023039010461A46039BF8F706FB00
:10BF800005E00DA82521F8F7E5FB00E0FFE716988E
:10BF9000401C169005E015A801780DA8F8F7DAFB0B
:10BFA000FFE7FFE71098002800D411E61098012859
:10BFB00001DBFFE7FFE710981AB080BD0024744949
:10BFC00040420F0080B58AB008900791002006908B
:10BFD0000798002804DCFFE70020C0430990D3E065
:10BFE000FBF73CFE039093486949405C002800D071
:10BFF000BEE090486649012242546A49415A6A4A61
:10C00000805A81420BDBFFE78A486649415A664AFB
:10C01000805A401A0121C9024018059007E085485E
:10C020006149415A5F4A805A081A0590FFE705980E
:10C03000079988424EDAFFE70020C04306907D480A
:10C040005B49405C002815D0FFE77A485649415AC1
:10C05000584A805A081802A9088008880121C90294
:10C06000884206DBFFE702985049401802A9088081
:10C07000FFE705E06F484C49405A02A90880FFE7F6
:10C080006C484849405A02A90988884208DBFFE702
:10C0900068484449405A0299401A01A908800AE0B8
:10C0A0000298FE493F4A895A081A0121C9024018DC
:10C0B00001A90880FFE70298F8493A4A88523448B3
:10C0C00000220A5401A803883B4A3C48012100F0A1
:10C0D0001BF94CE0F1483349405A0121C902081AC2
:10C0E000049004980799884203DBFFE707980490BF
:10C0F000FFE7EA482B49415A4018001D0899049A65
:10C10000F4F738F80499079A91420DDAFFE7089896
:10C1100004994018079A521AE049091D00900846F0
:10C120000099F4F727F8FFE70798DC491D4A8B5A76
:10C1300018188852885A0121C902884207DBFFE794
:10C14000D6481849425A194BD2184252FFE7D348F1
:10C150001749405C002803D1FFE700F0ABF9FFE787
:10C1600007980690CD480A4900224254FFE705E0AF
:10C1700008480949094B0A4AFFF7E6F90398FBF713
:10C18000CDFD06980990FFE709980AB080BDC0462A
:10C190000E080000E8EF000006F000006CEF000061
:10C1A0000E020000080800000A08000000F8FFFF67
:10C1B0000F0800000C08000020EF000002FF000044
:10C1C00085B004900391F3480068002805D0FFE78C
:10C1D000F0480068012823D1FFE7EE4800681649BF
:10C1E000164A00280192009101D001980090009811
:10C1F0000290FFE70398002811D0FFE702984069FA
:10C20000800700280AD5FFE70498411C04910078B4
:10C21000029908600398401E0390FFE7EAE706E0F2
:10C22000FB480068022801D1FFE7FFE7FFE7002095
:10C2300005B07047E8B401020090014000A0014041
:10C2400080B592B0119010910F9211980E9000202D
:10C250000D900C900B900A90099011A8007880071F
:10C26000002801D0FFE748E0254A09A814210590DD
:10C27000FCF7F6FD089008990598FFF7A1FF00214B
:10C2800007910691FFE707981099002288420492CF
:10C290000DD2FFE706980F990122002388420393ED
:10C2A000029201D30398029002980490FFE7049849
:10C2B000C007002821D0FFE70E9807998900405851
:10C2C000FFF714F9002813D0FFE70E9807998900AB
:10C2D00043580C4A09A814210190FCF7C1FD0890AD
:10C2E00008990198FFF76CFF0699491C0691FFE732
:10C2F000FFE70798401C0790C5E712B080BDC04615
:10C30000C2ED0000DAEE000081B0B0B5D5B05993AF
:10C310000B46044653AD288052A801705192BC4888
:10C3200081210901405C002803D1FFE700205490DF
:10C33000ACE00120010211A8F3F735FF00201090B6
:10C340000F9053980EA9087008780D2804DBFFE7BA
:10C350000020C043549099E052A80078042805DCDE
:10C36000FFE752A80078002804D1FFE70020C0436F
:10C3700054908BE052A800780EA90978484A515C85
:10C38000884203DDFFE7002054907FE053A8008837
:10C39000C00500281AD4FFE7109811A90A18012334
:10C3A0001B02181A0C910B920A90FFF71FF83D4AD6
:10C3B0000B99099008460A99099BFCF751FD0C99C5
:10C3C00008900846FEF7C4FF1090FFE753A80088C6
:10C3D000800500281BD4FFE7109811A90A18012333
:10C3E0001B02181A0EAB1B789B002F4CE3582F4CE6
:10C3F00007901046079A069111462246FCF730FD39
:10C40000069905900846FEF7A3FF1090FFE753A892
:10C410000088400500281DD4FFE7109811A90A18CC
:10C4200001231B02181A52AB1B789B00204C1B19CE
:10C430001B1F1B681D4C04901046049A0391114663
:10C440002246FCF70DFD039902900846FEF780FF97
:10C450001090FFE759A80D90109811A90A18012310
:10C460001B02181A519B0D9C01901046019A0091D5
:10C4700011461A462346FFF79DFB0F9010980F991F
:10C4800041180098FFF79EFD5490FFE7549855B06F
:10C49000B0BC02BC01B08E467047C046E8B4010291
:10C4A0002CFF00005CEF0000E093010203F00000AD
:10C4B000CC93010280B584B0FBF7D0FB03905448C5
:10C4C0003549415A544A805A814258D0FFE7504872
:10C4D0005349012242543049415A4F4A805A8142BD
:10C4E00009DDFFE74A482C49415A4B4A825A891ACA
:10C4F000484A815208E046484749415A0122D2023F
:10C50000511A444A8152FFE741484249405A23495F
:10C51000884206DBFFE73E48012189023D4A8152FD
:10C52000FFE73B483C49415A4118091D02913949EE
:10C53000415A01910068002805D0FFE7344800689F
:10C54000012814D1FFE732480068411E884100905D
:10C5500000980299019A124B00F06CFE002805D059
:10C56000FFE72B482E4900224254FFE706E0284807
:10C570000068022801D1FFE7FFE7FFE704E0244855
:10C58000244900224252FFE70398FBF7C7FB04B09F
:10C5900080BDC046E8B401020808000001040000A4
:10C5A000A5C5000080B584B003900291FBF756FB4F
:10C5B000019002A8C0780006800F002807D0FFE78E
:10C5C000029B184A02200121FFF79EFE1AE0104844
:10C5D0001049415A104A835A59188152805A0121F0
:10C5E000C902884207DBFFE709480B49425A0B4B57
:10C5F000D2184252FFE70648094900224254FFF789
:10C6000059FFFFE70198FBF789FB04B080BDC046E6
:10C61000E8B401020C0800000A08000000F8FFFF5F
:10C620000F0800004CEF000080B582B00190FDF7CC
:10C63000A7FF0198808A00281DD1FFE70F480168F5
:10C64000491C0160FDF73AFD0D4908600D4800687E
:10C65000002808D0FFE7FDF731FD0D4908600948C3
:10C660000021016007E008480068084908600548A3
:10C6700001210160FFE702B080BDC04660A7010252
:10C68000BCB40102C0B40102B0B40102A09B01021B
:10C69000A49B010270B588B0079006910798012805
:10C6A00004D8FFE706980E2806D3FFE7A7482449D9
:10C6B000244BDA22FEF748FF0798032104220028C2
:10C6C000084603910292019001D1029801900198CD
:10C6D0000699039A4A431C498A1892780091114698
:10C6E000F9F7D0F8079848210A46424396488258FD
:10C6F000D26880231A430592059A079C0D4665432C
:10C700004459E260069A039C5443009A15196D78C7
:10C710002D02145D2C190494049C079D0E466E4353
:10C720008559EC62059C9C430594059B079C6143DD
:10C730004058C3600498F9F7BFF908B070BDC0460F
:10C74000B3F000007FF0000094DF000010B588B067
:10C75000079006910798007805A9087000200490BA
:10C7600008787949C968884207D0FFE705A80078AA
:10C770007549496D884258D1FFE705A8007872498C
:10C78000C968401A411E88410390069803280CD1BD
:10C79000FFE70398482141436B484018806B0490A1
:10C7A0000398102100F08CFE28E0039848214143B3
:10C7B000654840188069302809D0FFE70398482170
:10C7C0004143614840188069102808D1FFE7039869
:10C7D000482141435C484018802181610DE0039865
:10C7E00048214143584A511889690191009057489E
:10C7F00057495A4B5B4AFEF7A7FEFFE703984821CB
:10C800000A4642435048821800231362039A0C469A
:10C81000544302199363039A0C46544302199362DA
:10C82000039A51434018436280E005A800784649C6
:10C830008968884207D0FFE705A800784249096D5A
:10C84000884269D1FFE705A800783F498968401A06
:10C85000411E88410390069803281DD1FFE70398E5
:10C860004821414338484018C069002808D0FFE7F4
:10C87000039848214143344840180021C16161E0D8
:10C8800003984821414330484018C06B04900398F6
:10C89000202100F015FE28E00398482141432A4852
:10C8A00040188069302809D0FFE7039848214143A8
:10C8B000254840188069202808D1FFE703984821BF
:10C8C000414321484018802181610DE003984821AF
:10C8D00041431D4A51188969019100901B481C4928
:10C8E0001E4B1F4AFEF730FEFFE7039848210A4619
:10C8F0004243154882180023D362039A0C465443DE
:10C900000219D363039A0C46544302195363039AE2
:10C9100051434018036308E005A8007800900B48D5
:10C920000B490C4B0C4AFEF70FFEFFE7049800285A
:10C9300008D0FFE70498069903AA02901046029ACD
:10C940009047FFE708B010BDF894010213F0000013
:10C9500090F0000065F00000DF0200002DF0000004
:10C96000D5020000B102000070B592B01190002015
:10C9700010900F90119848210A464243EB48825884
:10C98000D2690F231A400EAB1A70119A5143401806
:10C99000007C00285AD0FFE7119848214143E34822
:10C9A000405840690F900FA840789E2108420AD154
:10C9B000FFE70EA800780C2805D0FFE70EA8007846
:10C9C000012842D1FFE7119848210A464243D7483F
:10C9D000825893690424A3439361119A0B465343ED
:10C9E000C258022313620EAA13780124A4071B194C
:10C9F000119D0E466E438519EB61119B0D465D43FB
:10CA00004319DB6B1093127812190F92119A20239D
:10CA10000C9010460B91194600F052FD11980B999D
:10CA200041430C9841180022CA6211990B9B4B4359
:10CA3000C118CA6311990B9B4B43C1184A631199E2
:10CA40000B9B4B43C1180A63FFE761E10EA8007816
:10CA50000C280A9000D959E10A984000784480884F
:10CA6000400087440C0019001A005301B100530123
:10CA7000370145015301530153015301B10011988E
:10CA800048214143A9484058012101620EA800787D
:10CA9000C90740180F903AE139E1119848210A4638
:10CAA0004243A248825808231362119A5143401806
:10CAB0008069102809D0FFE71198482141439B481D
:10CAC00040188069302870D1FFE7119848210A4644
:10CAD000424396488218926A119B59434018406A13
:10CAE00082422FD1FFE7119848210A4642438F48DE
:10CAF000825893690224A3439361119A0B465343CE
:10CB0000C218926B1092119A102309901046089146
:10CB1000194600F0D5FC119808994143099841182D
:10CB200000220A621199089B4B43C1188A6311992C
:10CB3000089B4B43C1188A621199089B4B43C1184B
:10CB40004A6231E0FFE7119848210A46424377489C
:10CB50008218926A119B59434018406A0021824210
:10CB600007910BD2FFE71198482141436F48405885
:10CB700040690221084040080790FFE70798C00776
:10CB8000002810D0FFE7119848210A464243674821
:10CB90008218136A946A651C95621A5D119B594349
:10CBA00040580260CFE7FFE70DE01198482141436C
:10CBB000F94A51188969019100905D485D495E4BC1
:10CBC0005E4AFEF7C1FCA2E0119848214143F248B9
:10CBD00040188069202809D0FFE711984821414377
:10CBE000ED4840188069302872D1FFE7FFE71198BF
:10CBF00048210A464243E8488218526B119B594328
:10CC00004018006B0021824206910BD2FFE7119879
:10CC100048214143E0484058406908210840C00885
:10CC20000690FFE70698C007002813D0FFE7119889
:10CC300048210A464243D848825852680DAB1A70C0
:10CC40000D9A119B59434018C16A436B5C1C4463A5
:10CC5000CA54CCE7119848210A464243CE4882186C
:10CC6000526B119B59434018006B82422FD1FFE752
:10CC7000119848210A464243C748825893690524BF
:10CC8000A3439361119A0B465343C218D26B10927F
:10CC9000119A2023059010460491194600F010FCCB
:10CCA000119804994143059841180022CA621199CC
:10CCB000049B4B43C118CA631199049B4B43C11891
:10CCC0004A631199049B4B43C1180A63FFE700E0D4
:10CCD000FFE71CE0119848214143AF48405802212A
:10CCE00001620EA800780121890740180F900EE01C
:10CCF000119848214143A8484058042101620EA8D8
:10CD000000780121090740180F9000E0FFE7FFE7D6
:10CD10001098002808D0FFE710980F9911AA0390E7
:10CD20001046039A9047FFE712B070BDF8940102D5
:10CD300013F00000A2F0000049F000003D030000E5
:10CD400010B588B0069005910698022807D3FFE732
:10CD50000598002803D1FFE70120079018E1069805
:10CD6000002808D1FFE708200390F8F7EFFC0398AC
:10CD7000FDF7FAFE0CE00698012808D1FFE709202C
:10CD80000290F8F7E3FC0298FDF7EEFEFFE7FFE7FD
:10CD9000FFE7069848210A4642437F488258936934
:10CDA0001F24A3439361069A0B465343C25806239C
:10CDB0009360069A0B465343C2580F231362069A98
:10CDC0000B465343C21800231362069A0C46544381
:10CDD00002199363069A0C46544302199362069A09
:10CDE0000C46544302195362069A0C4654430219E6
:10CDF000D362069A0C4654430219D363069A0C4632
:10CE0000544302195363069A0C46544302191363A0
:10CE1000059A127F069B0C465C4303191A74059A07
:10CE2000527F069B0C465C4303195A74059A927F05
:10CE3000069B5943401882740598C1688068800039
:10CE40000143049105984068012805D1FFE7049843
:10CE500008210843049020E005984068022805D185
:10CE6000FFE7049818210843049015E005984068EE
:10CE7000032805D1FFE704982821084304900AE01D
:10CE800005984068042805D1FFE704983821084335
:10CE90000490FFE7FFE7FFE7FFE7049806994822C1
:10CEA00013464B43DA49CB58D860059843699B0138
:10CEB000DBB280698007800E1818069B14465C431D
:10CEC0000B191B7CDB071B0FC018401C0490049837
:10CED000069B14465C430B5998600498069B5A4382
:10CEE0008918486105980069012808D1FFE706986C
:10CEF00048214143C648405822210161FFE7069876
:10CF000005990968FFF7C6FB069848214143C048C8
:10CF10004018807C002812D1FFE706984821414341
:10CF2000BB484018407C002809D1FFE706984821FB
:10CF30004143B7484018007C00281FD0FFE70698FF
:10CF400048210A464243B24882185268022301909F
:10CF5000104600911946F7F767FE0698009941437D
:10CF6000019841184868F7F775FC06980099414305
:10CF7000019841184868F7F7F5FCFFE70698482143
:10CF80004143A34840180121816100200790FFE739
:10CF9000079808B010BDC046F8940102B0B59AB029
:10CFA00018901791169215931798002804D0FFE750
:10CFB0001698002803D1FFE70120199024E1189862
:10CFC000202100F0A5FA14901498002803D0FFE760
:10CFD0001498199018E117981899482213464B4352
:10CFE0008B49CB18D862189813464343C8180023BE
:10CFF00043631698189B14465C430B1918631598E5
:10D00000189B14465C430B19D86318984243885800
:10D010004069139013A840789821084215D0FFE783
:10D02000189848210A46424379488258062393605B
:10D03000189A0B465343C2580F231362189A514350
:10D040004218526940588260FFE7189848214143CE
:10D050006F484018007C002847D0FFE700200B9065
:10D060000C900D900E9002210F911090189919229A
:10D070001723012907900693059201D00698059081
:10D0800005981190079812901899482213464B431F
:10D090005F49CB18D861189B14465C430B1958683C
:10D0A00004920391F7F7D6FB18980499414303982B
:10D0B000415814228A611899049A4A438118886851
:10D0C0000BA9F8F76DFD1899049A4A4303998B1838
:10D0D0009B688A58111D179A169CF84D009502906E
:10D0E00018462346F8F7C6FD8BE0189848214143BF
:10D0F000F1484018407C00280AD0FFE718984821E2
:10D100004143ED484058816995221143816177E0A0
:10D11000189848214143FD48405880690A900AA860
:10D120000078000600280AD5FFE70A988021884386
:10D13000189948224A43F54989588861FFE7002039
:10D140000990FFE7189848210A464243EF488218A1
:10D15000526B189B59434018006B824235D2FFE74F
:10D16000189848214143E94840584069099009A866
:10D1700040789E2108420ED0FFE71898482141438D
:10D18000E248405802210162099801218A071043B0
:10D190000990149119E009A84078C007002813D01D
:10D1A000FFE7189848210A464243D84882585268F7
:10D1B00008AB1A70089A189B59434018C16A436B10
:10D1C0005C1C4463CA54FFE7BCE71898202100F0B8
:10D1D00077F9189848214143FD484018C06B002852
:10D1E0000DD0FFE7189848214143F9484018C06B1B
:10D1F000099918AA01901046019A9047FFE7FFE7A6
:10D20000FFE714981990FFE719981AB0B0BDC0460F
:10D21000F894010280B582B0019000910349044B5B
:10D2200001206422FFF7BAFE02B080BDB8A501025A
:10D2300015D2000070B598B0169015911492139302
:10D240001598002804D0FFE71498002803D1FFE7C1
:10D25000012017902CE11698102100F059F9129036
:10D260001298002803D0FFE71298179020E1159834
:10D270001699482213464B43E549CB181862169875
:10D2800013464343C818002383621498169B144620
:10D290005C430B1958621398169B14465C430B1998
:10D2A0009863169842438818007C002834D0FFE722
:10D2B00000200A900B900C900D900E9002210F917F
:10D2C000109016981A21182201280792069101D071
:10D2D0000798069006981190169848210A464243EE
:10D2E000CB488218D2680AAB0590104604911946C3
:10D2F000F8F756FC1699049A4A4305998B18DB688F
:10D300001599059CA258149D6C4E009603901846E2
:10D310002B46F8F7AFFCC8E0169848214143BC48BB
:10D320004018807C00283BD0FFE7FFE71698482193
:10D330000A464243B6488218926A169B59434018DF
:10D34000406A0021824202910BD2FFE716984821E1
:10D350004143AF48405840690221084040080290CC
:10D36000FFE70298C007002810D0FFE71698482171
:10D370000A464243A6488218136A946A651C95625D
:10D380001A5D169B594340580260CFE71698482112
:10D3900041439F484058816982221143816183E063
:10D3A0001698482141439A4840588069099009A835
:10D3B0000078000600280AD5FFE7099880218843F5
:10D3C000169948224A43924989588861FFE700200C
:10D3D0000890FFE7169848210A4642438C48821875
:10D3E000926A169B59434018406A824236D2FFE740
:10D3F000169848214143864840584069089008A83B
:10D4000040789E2108420ED0FFE7169848214143FC
:10D410007F48405802210162089801218A07104381
:10D42000089012911AE016984821414378484058D4
:10D4300040698007002810D5FFE7169848210A4662
:10D44000424373488218136A946A651C95621A5D98
:10D45000169B594340580260FFE7BBE7FFE7169869
:10D46000482141436A484058406A002801D0FFE7FC
:10D47000F5E71698102100F023F81698482141434B
:10D4800063484018806B00280DD0FFE716984821AC
:10D4900041435F484018806B089916AA01901046D6
:10D4A000019A9047FFE7FFE7FFE712981790FFE721
:10D4B000179818B070BDC046F89401024DC700001F
:10D4C00010B584B003900291FAF7DCFB019002984A
:10D4D0000399482213464B434D49CB189C6984431A
:10D4E0009C610398424388188069002808D1FFE7AF
:10D4F0000398482141434648401801218161FFE7D4
:10D500000198FAF717FC04B010BDC046F894010268
:10D5100080B586B00590049100200390FAF7B2FB25
:10D5200002900598482141433948401880690028F5
:10D53000019043D0FFE70198012814D0FFE701983C
:10D54000102828D0FFE70198202814D0FFE7019881
:10D55000302830D0FFE7019840282FD0FFE701980E
:10D5600080282BD02DE00498059948224A43284969
:10D570008918886125E00498102808D1FFE70598EC
:10D5800048214143224840183021816102E00220B5
:10D590000390FFE715E00498202808D1FFE70598DD
:10D5A000482141431A4840183021816102E002209D
:10D5B0000390FFE705E00220039002E001200390C2
:10D5C000FFE70298FAF7B6FB039806B080BDC046A5
:10D5D000F894010282B001900198482141430C481F
:10D5E000401880690021C006002800910AD5FFE795
:10D5F00001984821414306484058406901210840AC
:10D600000090FFE700980121084002B07047C04633
:10D61000F894010206480068202804D1FFE7054875
:10D620000649016003E0034803490160FFE77047D2
:10D630000C0000400090010230CF010324D601030A
:10D64000F0B59DB001461CAA10701078092803D1CE
:10D65000FFE7002019900CE01CA8007801210222AD
:10D6600005281892179101D01898179017981990BB
:10D67000FFE719981BA908701AA800210170FFE79D
:10D680001AA80078032813DCFFE71AA800781BA962
:10D690000978C9004D4A5118420089180E22895E46
:10D6A000FCF7EEFFFFE71A98401C1AA90870E7E79D
:10D6B0001BA80178C900454A51180E23CB5E1024DF
:10D6C0000C5F12254D5F1426895F0291019500942D
:10D6D0003F49022403251690204615912946159EA0
:10D6E0001492324613941295FEF70EFE16990A789C
:10D6F000149B2633D2009A18042411901046214618
:10D7000010930F94FBF71CFC16990A78D200109B1B
:10D710009C189B5E139AA55E0F9EA75F0621645E10
:10D720000294019700952B4A139C0E902046129D5F
:10D730000D912946FEF7E8FD16990A78149B3E33B1
:10D74000D2009A180C9010460F990B93FBF716FC19
:10D7500016990A78D2000B9B9C189B5E139AA55EC3
:10D760000F9EA75F0D99645E0294019700951A4A77
:10D77000139C0A9020461299FEF7C6FD5621149A72
:10D78000535E099018460891FBF7ECFB1499089A30
:10D790008B5E124A139C079020461299FEF7B4FD47
:10D7A00014995831069008460591FBF7C3FB5821A0
:10D7B000149A535E0599139C0D5F0095084A0490D6
:10D7C00020461299FEF7A0FD1DB0F0BD3898010269
:10D7D000F4F00000DAF00000C1F000002CF10000CD
:10D7E00011F1000010B582B0014601AA10702A485C
:10D7F00003680F24A3430093009B12781343036034
:10D800002648274A0260FFE72648006800070028EC
:10D8100001D4FFE7F8E701A800780A2806DBFFE754
:10D820002148254901602248016012E001A80078E2
:10D83000052807DBFFE71C481E4901601C481E49FC
:10D84000016005E018481949016019480160FFE7C7
:10D85000FFE701A800780C2804D1FFE717481B490F
:10D86000016017E001A80078092804DBFFE71348EE
:10D87000154901600DE001A80078052804DBFFE7E9
:10D880000E481049016003E00C480D490160FFE7B4
:10D89000FFE7FFE702B010BD040400400060004055
:10D8A0000004008004600040000600400F040F04E4
:10D8B0000406004003040304000400042C94010245
:10D8C0001DE600004EE700007FE80000ECE40000E9
:10D8D000B0B58AB00B46044609AD287008A801709F
:10D8E000079207980078059304940395FFF77AFF51
:10D8F0000798C07A00F028F903980078079A002169
:10D900000291029BFBF7ACFB0690069B134A022098
:10D910000321FEF7F9FC03990A7806990190104655
:10D9200000F04BF803980178C907002905D0FFE7FC
:10D9300008A8007800F0C8F9FFE709A80078800778
:10D94000002803D5FFE700F025F9FFE70798007BE3
:10D95000FAF748FD06980AB0B0BDC0465BF100007A
:10D9600080B588B01820FDF7FFF81920FDF7FCF806
:10D97000002007900799F7F751FB07990690084692
:10D98000FAF7B4FC012103227F2305900846049195
:10D990001146FAF7BDFD049903900846FAF760FFB7
:10D9A0000220FBF73DFB049902900846FCF78AFB36
:10D9B00007990190084608B080BD80B584B0024642
:10D9C00003AB18700291029801920093FCF71CF8C7
:10D9D00000980178C907002904D0FFE70298FCF7F6
:10D9E0009FFBFFE703A800788007002804D5FFE726
:10D9F0000298FCF711F8FFE704B080BD10B584B0C1
:10DA000003A800210170FFE703A8007821490978E5
:10DA100088420EDAFFE703A800788100254A5158B2
:10DA20004000224A1152FFE70398401C03A90870E6
:10DA3000EAE71948007819490870194842788A714C
:10DA40000078487117480278531C0370CA70114857
:10DA500002788A72027852000B460B33124C029005
:10DA6000184601912146F2F785FB02990A78520087
:10DA7000019BD4180B340D4900902046F2F77AFB35
:10DA80002021019A51720A494B789370097851709C
:10DA900004B010BDC8A6010245A501024CBE01029A
:10DAA000789E0102E0A00102CAA601021ABE01028C
:10DAB00060A6010264A6010210B58CB003460BAC4F
:10DAC00020700A9109920020089001210693059484
:10DAD000FCF772FDFAF7EAF807900598017800293B
:10DAE00016D0FFE70A9909982722520142430A20DB
:10DAF00004901046049A03911146F2F7EBFA0021C4
:10DB0000029008460399029AFAF7B0FE089013E0D3
:10DB100009982721490141430A20019008460199AB
:10DB2000F2F7D8FA02210022009008461146009A26
:10DB3000FAF79CFE0890FFE7FAF762FF0798FAF7FA
:10DB400005F908980CB010BD80B582B0019001981D
:10DB5000FF2804D1FFE70D480021016012E0019881
:10DB600003210840084A105C40221043074A106015
:10DB700001980840064A022300901846009BFEF7D1
:10DB8000C3FBFFE702B080BDBCE9000028060040EF
:10DB900040F1000080B584B017481849016018486A
:10DBA0000160184801601848016018481849016070
:10DBB0001848194901601949194A0A6015239B043C
:10DBC0000B60642103900846029201930091F7F7DD
:10DBD00073FF029803990860019A0A600098F7F7AA
:10DBE0006BFF1048039908600F4A10480321FEF7A5
:10DBF0008BFB04B080BDC04654600040200882000A
:10DC0000586000405C600040606000405060004030
:10DC100002D50F009060004002025500986000405D
:10DC200001005400040054004DF1000002080000FF
:10DC3000B0B58AB014460D46099008A8018007A81F
:10DC400002700693002105910078022810D1FFE7A9
:10DC5000012004900499FCF7AFFC0699099B08A8E1
:10DC60000088009000220498FAF7E2FE059025E073
:10DC700007A80078012810D1FFE7012000210391B7
:10DC8000FCF79AFC0699099B08A800880090039865
:10DC9000039AFAF7CDFE05900FE0012000210291D2
:10DCA000FCF78AFC099B08A80088009002200299D2
:10DCB000029AFAF7BDFE0590FFE7FFE7FAF7A0FE2C
:10DCC00005980AB0B0BD000010B584B0014603AAA3
:10DCD00010701248124B03601248134B0360134834
:10DCE000134B036013481523036013480368029322
:10DCF000029B402423430360104803680724240345
:10DD0000A3430293029B012464032343036010781E
:10DD1000019100F015F804B010BDC046A0600040AD
:10DD200012A83E00A46000409DD79B5AA860004006
:10DD3000D579BD49AC600040340200401406004073
:10DD4000F0B589B0014608AA10702A4803682A4C29
:10DD500023400793294B1C681578052637466F43E7
:10DD6000E519E45D2407640E6D7807273D406419CA
:10DD70000694079C069D0390E8030443E8010443CE
:10DD80001F480443039804601E4C25683C208543CB
:10DD900007951868157802966E4380198078384088
:10DDA00005900798059DED00284304252843206031
:10DDB000154804681F25AC4307941B681278029C21
:10DDC00054431A19D3785B07DB0E127903242240DF
:10DDD0009A180492079A049B1A4302600B480C4A53
:10DDE000026055225203026064200191F7F764FE3D
:10DDF00009B0F0BDC46000407F4080FF2C94010258
:10DE000040400000C8600040100600402C60004008
:10DE100001A00A0010B588B006900698002803D02B
:10DE2000FFE70120079036E0069800011B490858DB
:10DE3000032293021A4CC45006980001085800248B
:10DE400084600D2005900491039202930194F6F7EB
:10DE500023FD0598F6F70EFD0698000104990818B1
:10DE6000019A027206980001081842720698000191
:10DE7000081882720698000108580123029C035179
:10DE80001020F7F757FC074A02200399FEF73CFAE7
:10DE900001990791FFE7079808B010BD8895010226
:10DEA00051E5CC1A72F100002021020C01D01021A2
:10DEB0001046020A01D010460839020901D0104666
:10DEC000091F820801D01046891E420801D0881E11
:10DED0007047081A704702E008C8121F08C1002ADC
:10DEE000FAD170477047002001E001C1121F002ADB
:10DEF000FBD17047000084C1000008C10000C03F92
:10DF0000000038410000AC410000D4410840080046
:10DF10000008100804081020280004000000000079
:10DF2000000000000000000001000000FFFFFFFFF4
:10DF30000000000000000000303132333435363745
:10DF4000383941424344454646494C45202020202B
:10DF50003A200046554E4354494F4E3A20004C4912
:10DF60004E45202020203A20002D2D2D2D2D2D2D09
:10DF70002D2D2D2D2D2D2D2D2D2D2D2D2D2D2D2DD1
:10DF80002D2D2D2D2D2D2D2D2D2D2D2D2D2D2D2DC1
:10DF90002D0D0A0059062014032145012882003264
:10DFA0004100321900411300390300B506002D036A
:10DFB000002D02002201002201003E01002000008D
:10DFC0008009EE4D5048504F80096E4F58E5854FFF
:10DFD00080096E4FB867C14F5048D04FB867C14FE6
:10DFE000E828DF4F8009EE4F18EAFC4F8009EE4F1A
:10DFF00058E50550A4550D50F0C51450A4550D50CA
:10E0000000002110422063308440A550C660E770B4
:10E01000088129914AA16BB18CC1ADD1CEE1EFF15C
:10E020003112100273325222B5529442F772D66204
:10E03000399318837BB35AA3BDD39CC3FFF3DEE3AC
:10E040006224433420040114E664C774A444855454
:10E050006AA54BB528850995EEE5CFF5ACC58DD5FC
:10E060005336722611163006D776F6669556B446A4
:10E070005BB77AA719973887DFF7FEE79DD7BCC74C
:10E08000C448E5588668A7784008611802282338F4
:10E09000CCC9EDD98EE9AFF9488969990AA92BB99C
:10E0A000F55AD44AB77A966A711A500A333A122A44
:10E0B000FDDBDCCBBFFB9EEB799B588B3BBB1AABEC
:10E0C000A66C877CE44CC55C222C033C600C411C94
:10E0D000AEED8FFDECCDCDDD2AAD0BBD688D499D3C
:10E0E000977EB66ED55EF44E133E322E511E700EE4
:10E0F0009FFFBEEFDDDFFCCF1BBF3AAF599F788F8C
:10E100008891A981CAB1EBA10CD12DC14EF16FE16B
:10E110008010A100C230E3200450254046706760A3
:10E12000B9839893FBA3DAB33DC31CD37FE35EF3BB
:10E13000B1029012F322D2323542145277625672F3
:10E14000EAB5CBA5A89589856EF54FE52CD50DC50B
:10E15000E234C324A0148104667447642454054443
:10E16000DBA7FAB79987B8975FE77EF71DC73CD75B
:10E17000D326F2369106B016576676761546345693
:10E180004CD96DC90EF92FE9C899E9898AB9ABA9AB
:10E190004458654806782768C018E1088238A328E3
:10E1A0007DCB5CDB3FEB1EFBF98BD89BBBAB9ABBFB
:10E1B000754A545A376A167AF10AD01AB32A923A33
:10E1C0002EFD0FED6CDD4DCDAABD8BADE89DC98D4B
:10E1D000267C076C645C454CA23C832CE01CC10C83
:10E1E0001FEF3EFF5DCF7CDF9BAFBABFD98FF89F9B
:10E1F000176E367E554E745E932EB23ED10EF01ED3
:10E20000100040008000000100020004000800101F
:10E210001000180020003000400060008000000165
:10E22000FFFFFFFF01FF01FFFF0101FFFF010000F2
:10E2300000000000000000000000000000000000DE
:10E2400000000000020000000000000014000000B8
:10E2500002000000070000000200000002000000B1
:10E260000000000002000000000000001400000098
:10E270000200000001000000020000000200000097
:10E280000200000000000000140000000000000078
:10E29000FFFFFFFFFFFFFF01FFFF01FFFF01FF0186
:10E2A000FF01FFFFFF0101FFFFFF01FF0101FFFF72
:10E2B0000000000000007A000000000000007A006A
:10E2C000000000007A000000000100FF010000FFD4
:10E2D000000064009E00C800E800020119012C0142
:10E2E0003D014C015A01660172017D0187019001D7
:10E2F0009901A101A901B001B701BE01C401CA0180
:10E30000D001D601DB01E101E601EB01EF01F401EF
:10E31000F801FD010102050209020D0211021402B9
:10E3200018021B021F022202250228022B022E02C3
:10E330003102340237023A023D023F0242024502F4
:10E3400047024A024C024F0251025302560258023F
:10E350005A025C025F02610263026502670269029F
:10E360006B026D026F02710273027502760278020F
:10E370007A027C027E027F0281028302840286028C
:10E38000880289028B028C028E028F029102920215
:10E3900094029502970298029A029B029D029E02A5
:10E3A0009F02A102A202A302A502A602A702A9023D
:10E3B000AA02AB02AD02AE02AF02B002B102B302DA
:10E3C000B402B502B602B702B902BA02BB02BC027D
:10E3D0000000000000000000020000000400000037
:10E3E000001003EB0000000001000000010000002D
:10E3F00004000000000100320000000000000000E6
:10E400000000000001000000010000050000000005
:10E4100000000000000000000100000001000035C5
:10E4200000000000010000000000000004000000E7
:10E4300000000020000000000100000000000000BB
:10E4400004000000000000D80000000001000000EF
:10E4500000000000010000000000000600000000B5
:10E4600001000000000000000100000002000001A7
:10E47000000000000000000000000000010000009B
:10E480000300009F000000000100000000000000E9
:10E4900001000000000000B90000000001000000C1
:10E4A0000000000001000000000000AB000100FFC0
:10E4B000010000FF000100FF010000FFFF0000015C
:10E4C00000FF00010001000000FF00FF00FF00004E
:10E4D0000100FFFF00FF010000000001010000FF3C
:10E4E000FFFF01FF01010000000001010003020124
:10E4F0000000050201000001030100000303010008
:10E5000001000301000102030100020003010002F7
:10E5100002030100030203010003040301000402DB
:10E5200003010000000302000003030200000603D1
:10E5300002000100030200010303020001060302BE
:10E5400000020103020002040302000207030200AA
:10E550000303030200000107030000060703000194
:10E560000004030001000703000104070300010782
:10E570000703000200070300020407030002070765
:10E580000300030207030003060703000402070356
:10E590000004060703000501040300050207030049
:10E5A000050607030006000703000604070300062C
:10E5B0000707030007030703000707070300080214
:10E5C00007030008060703000902070300090607FE
:10E5D00003000A020703000A070703000B050703ED
:10E5E000000C030703000C070703000D07070300D7
:10E5F0000E070703000E060704000E070704030EAC
:10E60000070704030E070704030E070704030E079A
:10E610000704030E070704030E070704030007009F
:10E6200002020100000202000401020200070102CE
:10E6300002020200020201010102020106010202BD
:10E6400003050002020402000202020601020203A4
:10E650000001020203050102020503000202040593
:10E660000102020204020202020702020205030181
:10E67000020205060102020600010202060301026F
:10E68000020205030202020603020201060402025C
:10E690000106070202020304020202030702020249
:10E6A000060702020302070202030507020203072C
:10E6B0000702020407040202050104020205010721
:10E6C000020205030702020506070202060207020C
:10E6D00002060507020207010702020704070202F9
:10E6E00008010402020802070202080507020209E3
:10E6F0000304020209040702020A000702020A02D6
:10E700000702020A050702020A070702020B0307B3
:10E7100002020B060702020C010702020C040702A8
:10E72000020D010702020E000702020E0407020298
:10E730000F010702020F050702020E040703030F71
:10E74000030703030F070703030F07070303000073
:10E7500000020200000002020000000202000000AD
:10E76000020200000002020000000202000100029A
:10E77000020004000202000700020201010002027E
:10E78000010400020201070002020203000202016A
:10E790000401020201060102020305000202020452
:10E7A000010202030101020203030102020401014A
:10E7B0000202040401020202060202020302020231
:10E7C0000201060302020202030202010207020220
:10E7D000010407020203030302020204040202020C
:10E7E00005070202030107020203050402020401F5
:10E7F00007020204030702020506030202050007DE
:10E8000002020502070202050407020206000702CF
:10E8100002060207020206050702020607070202B5
:10E82000070407020207070402020802070202089F
:10E8300005070202090107020209040702020A0091
:10E840000702020A030702020A060702020B020776
:10E8500002020B050702020C010702020C05070267
:10E86000020D020702020C010703030C0607030353
:10E870000D020703030E020703030E07070303003D
:10E88000000002020000000202000000020200007C
:10E890000002020003000202010000020201020065
:10E8A000020200050102020202000202030100024C
:10E8B000020201010202020401020201020202023A
:10E8C0000104020202030401020202020202020225
:10E8D000050202020002070202000407020200060B
:10E8E00007020201020702020104070202010607F1
:10E8F00002020203070202020507020203020702E4
:10E9000002030407020204020702020404070202CF
:10E9100004060702020501070202050307020205B9
:10E9200005070202060207020206040702020606A3
:10E930000702020704070202080107020209000792
:10E940000202090107020209030702020A00070284
:10E95000020A020702020B000702020B0207020270
:10E960000C000702020B060702020C040702020C4D
:10E97000060702020D030702030C000703030C0243
:10E980000703030C050703030C070703030D050723
:10E9900003030D070703030D070703030D07070311
:10E9A000030D070703030D070703030D0707030301
:10E9B0001F1C1F1E1F1E1F1F1E1F1E1F0E0D0B07BD
:10E9C000556E6578706563746564204144432069C1
:10E9D0006E746572727570740D0A00696E636C7581
:10E9E00064652F647269766572732F6D6B5F616405
:10E9F000632E63004144435F49525148616E646C29
:10EA0000657200414553206F757470757420756E82
:10EA1000646572666C6F770D0A0041455320696E1C
:10EA2000707574206F766572666C6F770D0A006979
:10EA30006E636C7564652F647269766572732F6D91
:10EA40006B5F6165732E63004145535F49525148C6
:10EA5000616E646C6572004F6C642063686970203D
:10EA60006D6F64656C206973206E6F7420737570B0
:10EA7000706F7274656420627920746869732053C2
:10EA8000444B2121210D0A005854414C206C6F61E8
:10EA900064206361702074756E65202564203A20BF
:10EAA00025640D0A0033324B206C6F616420636172
:10EAB000702076616C2025640D0A005854414C206A
:10EAC0006C6F6164206361702076616C2025640D39
:10EAD0000A00436869702049443A20253038780D8F
:10EAE0000A00696E636C7564652F6472697665727D
:10EAF000732F6D6B5F646D612E6300496E76616C80
:10EB00006964207472616E73666572206473742028
:10EB10006164647200646D615F7472616E736665D6
:10EB20007200696E636C7564652F647269766572D4
:10EB3000732F6D6B5F6475616C5F74696D65722EA8
:10EB40006300636F6E66696720697320696E766122
:10EB50006C6964006475616C5F74696D65725F6F88
:10EB600070656E0054686520444D41207265616493
:10EB7000206C656E6774682073686F756C642062C2
:10EB80006520746865206D756C7469706C65206FA4
:10EB90006620340D0A00626C6F636B206964782014
:10EBA0006973206F7665722072616E67650D0A0069
:10EBB000736563746F7220696478206973206F765F
:10EBC00065722072616E67650D0A00556E6578701A
:10EBD000656374656420646D61206368616E6E6551
:10EBE0006C0D0A006A656465635F69642025780DB1
:10EBF0000A00696E636C7564652F6472697665726C
:10EC0000732F6D6B5F666C6173682E6300666C6159
:10EC100073685F7265616400666C6173685F626CE3
:10EC20006F636B5F657261736500666C6173685FCB
:10EC3000736563746F725F657261736500666C61A2
:10EC400073685F646D615F63616C6C6261636B00CC
:10EC5000666C6173685F646D615F77726974655F2C
:10EC60006E62797465735F63616C6C6261636B0083
:10EC700052656C6F61642076616C756520696D709A
:10EC80006F737369626C650D0A00696E636C7564FD
:10EC9000652F647269766572732F6D6B5F6D697332
:10ECA000632E63007379735F7469636B5F73746160
:10ECB000727400526573657420627920445644442E
:10ECC0000D0A0052657365742062792050494E0D1B
:10ECD0000A005265736574206279204C4F434B558E
:10ECE000500D0A00526573657420627920535953A0
:10ECF0005245510D0A0052657365742062792042B5
:10ED00004F520D0A00526573657420627920504F8E
:10ED1000520D0A005265736574206279205744547D
:10ED20000D0A00526573657420627920756E6B6EF2
:10ED30006F776E20736F757263650D0A005265738D
:10ED40006574206279205357205265626F6F740D8D
:10ED50000A0052434F33324B2070706D2025640DF2
:10ED60000A00696E636C7564652F647269766572FA
:10ED7000732F6D6B5F736C6565705F74696D657221
:10ED80002E6300534C4545505F54494D45525F49F1
:10ED9000525148616E646C657200556E657870659D
:10EDA0006374656420736C65657020696E74657248
:10EDB00072757074004343523D253038580D0A0D6A
:10EDC0000A000D0A4261636B74726163653A200D3B
:10EDD0000A0025313064207C200D0A0043726173E3
:10EDE0006865642121210D0A000D0A232323204197
:10EDF0005353455254204020307825303858202332
:10EE000023230D0A000D0A0D0A232323204558430E
:10EE1000455054494F4E202564202323230D0A00DA
:10EE2000253038583A202530385820253038582099
:10EE30002530385820253038580D0A005052494D99
:10EE400041534B3D253038580D0A00434F4E545224
:10EE50004F4C3D253038580D0A004558435F524508
:10EE60005455524E3D253038580D0A000D0A535066
:10EE70003D253038580D0A004D53503D2530385847
:10EE80000D0A005053503D253038580D0A004149B5
:10EE90005243523D253038580D0A005343523D2508
:10EEA0003038580D0A004C523D253038580D0A00B4
:10EEB000494353523D253038580D0A0049505352AA
:10EEC0003D253038580D0A00785053523D253038D2
:10EED000580D0A0052252D32643D253038580D0A50
:10EEE000004E3D25642C205A3D25642C20433D25B1
:10EEF000642C20563D25640D0A002C20457863655E
:10EF00007074696F6E4E756D6265723D25640D0A91
:10EF1000002C205468726561644D6F64650D0A00B1
:10EF20000D0A5472616365206275666665722069B8
:10EF3000732066756C6C2C206469736361726473F2
:10EF40002025752062797465730D0A00554152546D
:10EF5000204572726F722025780D0A0025313075B8
:10EF6000207C200050433D25303858005452414306
:10EF7000452042555359005B53435030335D005B8D
:10EF8000464952415D005B5557425D005B4D414330
:10EF90005D005B4343435D005B564552424F534522
:10EFA0005D005B53455D005B5543495D005B574128
:10EFB000524E5D005B494E464F5D005B4150505DD7
:10EFC000005B4552524F525D005B4F535D005B4208
:10EFD0004F4F545D005B544553545D005B445256A3
:10EFE0005D005B5048595D00696E636C7564652F08
:10EFF000647269766572732F6D6B5F74726163659D
:10F000002E630025730074726163655F6F757470A1
:10F01000757400696E636C7564652F6472697665DA
:10F0200072732F6D6B5F756172742E6300556E6520
:10F03000787065637465642075617274202564203E
:10F0400073746174652025640055617274202564B1
:10F0500020737461746520676F65732077726F6EBB
:10F060006720256400556E6578706563746564205B
:10F07000646D61206368616E6E656C20256400506C
:10F080006172616D74657220696E76616C6964008D
:10F09000756172745F646D615F63616C6C62616302
:10F0A0006B00756172745F6972715F68616E646C28
:10F0B000657200756172745F626175645F73657417
:10F0C0000050446F41206761696E732025642025DC
:10F0D000642025642025640D0A0050446F4120649B
:10F0E000656C6179732025642025642025642025C2
:10F0F000640D0A00546F4620616E742064656C6173
:10F1000079732025642025642025642025640D0A58
:10F110000050446F4120616E676C65206F666673B6
:10F120006574732025642025640D0A0050446F41E6
:10F1300020616E742073706163652025640D0A0080
:10F140004F70656E20414E5425640D0A007577623C
:10F150005F72785F696E69740D0A005048592070BB
:10F160006172616D73207365747320253038780D7A
:10F170000A0057445420636C6F73650D0A00BDF894
:10F18000C8EBC9FDBCB6C4A3CABD0D0A00BDF8C812
:10F19000EB617070B2E2CAD40D0A00706F6C6C5FE4
:10F1A00074785F6E756D2069732025642C726573A9
:10F1B000705F72785F6E756D2069732025642C64B2
:10F1C000697374616E636520697320256C660D0A2E
:10F1D000006C73705F7363616C655F663332006CE3
:10F1E00073705F675F6F705F663332006C73705F60
:10F1F000675F6F705F696E743136006C73705F6744
:10F200005F6F705F696E7438002E2E2F2E2E2F2E9A
:10F210002E2F2E2E2F2E2E2F647269766572732F4D
:10F220006D6B5F6C73702E63004F706572616E64FE
:10F230002061646472657373202578206973206986
:10F240006E76616C6964004E656564206174206C43
:10F2500065617374206F6E65206F706572616E6496
:10F26000005258204445534320696E6465782069F4
:10F2700073206F7665722072616E67650D0A0045B6
:10F280005420696E646578206973206F76657220FA
:10F2900072616E67650D0A002E2E2F2E2E2F2E2ED8
:10F2A0002F2E2E2F2E2E2F647269766572732F6D7E
:10F2B0006B5F6D61632E63006D61635F72785F6485
:10F2C0006573635F636F6E737472756374006D61F1
:10F2D000635F65745F636F6E7374727563740055FA
:10F2E0006E646566696E656420626974207261741B
:10F2F0006520256420666F72206D65616E20505216
:10F3000046206F662025640D0A004D45414E205071
:10F31000524620706172616D65746572206572720B
:10F320006F720D0A00436F6465206964782025645C
:10F3300020616E64206D65616E2050524620256408
:10F3400020636F6E666C6963740D0A002E2E2F2E7B
:10F350002E2F2E2E2F2E2E2F2E2E2F647269766595
:10F3600072732F6D6B5F7068792E6300010000016E
:10F37000000000FF00FFFF0000FFFF01000100018F
:10F380000000FF01FF01010001000000000101FF7A
:10F39000000000010000FF0000FFFF00FF0100016E
:10F3A00000FFFF00FF01010100010100000001FF5B
:10F3B00000010000FF000101FF000101010000FF4A
:10F3C00001000001000100FF000101FF01FFFF013A
:10F3D000000000000000010000000000FF0100002C
:10F3E0000000FF00FF000000FFFF0101010000011D
:10F3F00000FF01000001000001000000000000FF0C
:10F40000000000FF0000FFFF000000FF0001FF01FF
:10F4100000FF0001FF00FF01000000000001FF00ED
:10F4200000010100FF00010000FFFF0100000101D9
:10F43000FF010001FF000100000000FF00FF00FFCE
:10F4400000FF0101FF0100010000010001000000B8
:10F45000FF0100010101000000FFFFFFFF010101AA
:10F460000000000001010100FFFFFF01FF0000009C
:10F4700000010000FFFF0000000000FF000100018C
:10F480000001FF000100000100000100FF0000FF7B
:10F49000010101000001000000FF01000100FF0068
:10F4A0000000000101010101FF010001FFFF000157
:10F4B000FF000101FFFF00FF0000000100FF01004D
:10F4C00000010001FFFFFFFF000000FF000000003F
:10F4D0000000FF01000001FF000101000000010128
:10F4E000FF00000101FF00FF00FF0100010100001B
:10F4F00000000000FF000100FF0100FFFFFF01FF0F
:10F5000001010000FF0100010100010001000100F4
:10F510000000FF0000FF0000FF01000001FF0101EB
:10F52000000000FF01FF00FF010100FF00010101D9
:10F530000100FF0000FF00010100000100010000C8
:10F540000101FF00000100000001FF000000FF00BA
:10F55000FFFF0100000000FF00000000FFFF0001AE
:10F56000000000000001FFFF01000000FFFF00009D
:10F570000000FFFF010100FF0101010100FF000188
:10F5800001000100FF0000FF010001010000010176
:10F59000FF0001010001FF0100FF0000010000FF6A
:10F5A00000FFFF000000FF01FF000001000000005D
:10F5B000FF000101FF000000000001FF00FF00004C
:10F5C00000000000FF0000FF01FF0101FF0100003B
:10F5D00000FF0001000100010101FF0000FFFF002A
:10F5E0000001000100000001000000010100FF0017
:10F5F0000100FF000001FF00FF0100FF000001000B
:10F600000100000000010001FF00000000010100F6
:10F610000001000101010101FF0100FF0001FF00E5
:10F62000FFFF01000101FFFF000000FFFFFF0001DD
:10F6300000000001000100FF01FF000000000000C9
:10F6400001FF01FF00FFFF00000101000000FF00BB
:10F65000000100000101FF0000FFFF0101FF0000A9
:10F66000FF00000000000001FF00000100FF00009B
:10F6700000FF010100000000FFFFFF01010000008A
:10F68000010001FF00FF010000FF01000000FFFF7B
:10F6900000FF0000FFFF00FFFF010101FF0100FF6D
:10F6A0000101000001FF0101000100000000000154
:10F6B00000FF00010101FF00000100000100000047
:10F6C000FF00000000010000FFFF01000101000138
:10F6D000000100FF0000FF00FF01FF000100010129
:10F6E0000000000000010100000000010000000116
:10F6F000000001FFFF0001FF010100FF000000FF0B
:10F70000FF000001FF0001000001010000000101F5
:10F7100001000001000100FF00FF01FF00FF0001E8
:10F72000000001000001000101FFFFFFFF010000D8
:10F730000101FFFF010001FF00FFFF0100000000C9
:10F740000000FF00FF00000000FF0100FFFF0000BD
:10F7500001000000000001FF0101000000FF00FFA8
:10F760000100010001FFFF000000FF00FF0000009A
:10F770000001FF0000000000010000000000000187
:10F78000FFFF01FF010100FF00010001000001FF78
:10F79000000001010100FF010100FF00000100FF66
:10F7A00001000000010100010101FF00FFFF000155
:10F7B0000001FF00FFFF0000FF000001000000FF4C
:10F7C00001010000000001000101FF01FF00000134
:10F7D00000010001FFFF0000FFFF00FF000000012B
:10F7E000000001FFFF000101010000000001010114
:10F7F000FFFFFFFF0000000101010001FF0000000A
:10F800000100010000010001FF0101FF00FF00FFF6
:10F8100000FF000000000100FF010001FF010100E6
:10F820000001FFFF00000100FF0001010000FF01D7
:10F83000000000000001FF00FF0100FF0001FF01C8
:10F8400000FF000000FFFF0000FF000000FF0000BD
:10F850000000000001000001000001FF00010000A5
:10F860000101FF00FF01010000FF01010000000194
:10F870000100FF01000001FF000000000000FF0088
:10F880000000FFFFFFFF010001000001FF00010079
:10F890000000FF00FFFF010100FF0100FFFF01006A
:10F8A00001FF010101010100000000FF0001000152
:10F8B000FF000000010000010101FF0000FF000146
:10F8C00000000100000100FF010001000100FF0035
:10F8D00000000000FFFF00000100000000FF01FF2A
:10F8E00000FFFF0100000000000100FFFF0000001A
:10F8F00000FF0000000001FFFF00FF000000FF010B
:10F90000000000010000FF010100000100010000F3
:10F91000010100FF0000FF000101010100FF0001E3
:10F9200001FF00FF01FF0000000101FF01000001D5
:10F93000FF0000FF0000FF000000010001000100C7
:10F9400001010001FF00000101FF01FFFFFF0001B5
:10F95000FF000100FF00000000000001010001FFA6
:10F960000100010000FFFF0000FF01010100010094
:10F970000100FF00000001FF0101FF01FF0000FF87
:10F98000000000000000FF00FF010000000000FF79
:10F99000010100FF00000000010000FF01FF000066
:10F9A00000FFFF00FF0000010000FF0001FF010059
:10F9B000010100FF0101000001010001FF0000FF43
:10F9C000000100010100FF0001010101FF00010130
:10F9D000FFFF00000000FFFF00000001000000002A
:10F9E000FF0000FF0101FFFF0000FF010100000117
:10F9F0000000FF00000001010000FFFF00FF01FF09
:10FA000001000000000000FF01FF000100010000F4
:10FA1000000100FFFFFF000000FFFF01010001FFE8
:10FA2000FF00FF0100FF0001FF01010101010001D2
:10FA30000000010100000000FF01000100000000C3
:10FA40000100010000FF0001FF00FF010000FF00B6
:10FA50000100FF00010100000001000000000000A3
:10FA6000000101000100FF01FF00FF0000FF000195
:10FA700000010001010001FFFF0000010000000083
:10FA8000FF000000010000010000FF01010100FF74
:10FA90000001000000000001000101FF0100000161
:10FAA00001FF0001FF010101FFFF00FFFF0000FF58
:10FAB00000FFFF00000001FF000001FF00FF010048
:10FAC000010000000101FFFFFF000000000101FF35
:10FAD000000000FF00010000FF0100000001000124
:10FAE000FF00FF0000000101FF0100000000000115
:10FAF0000000FFFF0001FF00000000FF00FF00000A
:10FB00000000000001FFFF00FF010001FFFF0101F5
:10FB1000000001FFFFFFFF010100010000010000E4
:10FB20000100FF00FF01FF00FF00010001000001D4
:10FB30000101000000010100000100FF010000FFC1
:10FB4000FF000000FF000101FF0100FFFF010000B6
:10FB5000010000000100000000010100FF000000A2
:10FB6000000100FF000101010001FF00000001FF92
:10FB70000101010000FF0100FF000000010001FF82
:10FB800000010001000000FF010100FF01FFFFFF75
:10FB900000000100000101000000FF010001010060
:10FBA0000000FF01FF01010000010100010000FF52
:10FBB00000000000FF000100FF0000000001FF0046
:10FBC00000FF0000FF010101010001FF0100000032
:10FBD0000100FF00010100FFFF0001FF0000010123
:10FBE00001FF01000000FF010001010100FF000111
:10FBF00000000000FF000001010000010000FFFF05
:10FC0000FF01FF000101FF00000001000100FF01F2
:10FC1000000100000000010000000001FF000100E1
:10FC20000100000100000001000101FFFFFF00FFD3
:10FC3000010000FF0100010000FF00FF00010100C2
:10FC4000000000FFFF010000FF01000101FF0101B2
:10FC500000010000FF0001010101FFFF01FFFF01A2
:10FC6000FF01010101FF01FFFFFF0101FFFF010192
:10FC700001010101FF0101FF01000001FFFF01007F
:10FC8000FFFF01000101010101FFFF010101FFFF71
:10FC900000FFFF0001FF01FFFFFFFF00FF01FF0169
:10FCA000FF010001FFFF0101FF01FF010101000150
:10FCB000010001FF01FFFFFF0101010101FF01FF41
:10FCC0000101FFFF01FFFF0101FFFFFF01FF000135
:10FCD000010100FF01010101FF01000100FFFF0020
:10FCE00001FF0101FF010101010101FFFF01FF010E
:10FCF000010000010101FFFF0001FFFFFFFFFF0105
:10FD0000FF0001FF01FF01FFFFFF010101FFFF01F4
:10FD10000101FFFFFF01FF01FF00FF01FFFF0001E5
:10FD200001FF01FF0100FF010101010101010101CA
:10FD300001FFFF01FFFF0101FF0101000101FF01C0
:10FD4000FF01FFFF01FFFF010101FFFFFF00FF01B6
:10FD50000101FF00010000FFFFFF0101FF01FFFFA4
:10FD600000FF0101000101010101FFFF010101FF8D
:10FD70000101FFFFFF01FF01FFFF000101FFFFFF86
:10FD800001FF010001FFFFFFFFFF0100010101FF73
:10FD9000FF01FF01FFFF01FF0101FF010101010060
:10FDA000FF00FF0101000001FF010101FF0101FF50
:10FDB0000100FF0100FFFF01FFFFFF010101000142
:10FDC00001FF00FFFF01FF0101FFFF000101000033
:10FDD0000101FF0101FFFFFFFFFF0101010101011F
:10FDE000FF0001FFFF01FF0101FFFF01FF01010112
:10FDF000FFFF01010101010101FF0101010001FFFC
:10FE000001FF00FF00FF0101FFFFFF0100FFFFFFF7
:10FE1000010100FF01FF01FF0101FFFF010100FFE0
:10FE2000FF000101FF0000FFFF0101FF0101FF01D1
:10FE3000FFFF0101010101FFFFFF010101FF01FFC0
:10FE40000001FF01FF01000101010101FF010101AA
:10FE5000FF010101FF0100FFFFFFFFFFFF0101FFA5
:10FE60000101FF0100FFFFFFFF01FF01FF00010093
:10FE700001FF010101FFFF01FF010100010101FF7D
:10FE8000FF0101FF0001010000FFFF0101FFFF0171
:10FE90000101FF01FFFFFFFFFFFF00010101FF0163
:10FEA00001010101FFFF01FF0101FFFFFF01FF0150
:10FEB000FFFFFF01FF0100FF01FFFF00010001FF45
:10FEC0000101FF01010001FF01FFFF00010101012C
:10FED00001FF0101010101010101010101FFFFFF1A
:10FEE00001FF0101FFFF01010000FF01FF0100FF11
:10FEF00001FF00FF0101FFFF010101FF01010100FE
:10FF0000FFFF000101FF01FF01FF00FFFFFF0101F3
:10FF1000FF00FFFFFFFF01010101FF01FF000100E2
:10FF2000FF01FF0101FF0101FFFF01FF04000004C9
:10FF30000404040404040400000D0A0060FF00002F
:10FF40000890010290050000800B0000780101007C
:10FF50009895010258290000E6DE0000000000002C
:10FF6000560026B8030145D0014009021D01459005
:10FF70000050084202C203001515C0C1C2C3C4C567
:10FF8000C6C7C8C9CACBCCCDCECF000101013C0148
:10FF90008003090902030202010133020365090219
:10FFA0000301420257140019412717901D07060547
:10FFB0000403020100F29798DDC89D5CB81CC0DE06
:10FFC000A7DB615BCA01020003524048051004062A
:10FFD000010001522D2C280004007C007B01050249
:10FFE0000308FF5B0F010065F901417B0707010171
:10FFF00060002000881333E0536420ACFF501B0DD9
:020000040001F9
:10000000070E080E080E080E080C030D050B050D53
:10001000070D070D070D0701012E01040200400323
:10002000FFFF7F00FFFF7F0816FFFFFF00FFFFFFBE
:100030003A010001000A00010106401E40051205B8
:10004000120005150402010203010240040201032B
:1000500003020C0E0900087A0232413428002A8279
:100060000303455006C570014013E620700140149B
:100070004C07001000D6FF00B000500B4202820374
:1000800045FFFF0F203204420832010455100001E1
:1000900042010A50B4000301002000500733C1EFB1
:1000A00033ADEF33B4EF7398EF338CEF33E2EF33CC
:1000B000DCEF33BBEF3386EF33A7EF33D5EF33CE2F
:1000C000EF33C9EF337FEF3392EF33A2EF3377EFA4
:1000D0009D2800040001020100FFFFFFFF3784900C
:1000E00001027FE80051151EC135BF80F3E2BDC09B
:1000F000B464BF871699BDAD178DBF941799BD33F2
:10010000A876BFC4780DBD2BC162BA0CB0AFBEA932
:10011000F6E9BAFC567BBE07254CBBEC8823BE5DD6
:10012000C0CBBB0CCE20BD7BA095BCD40F3A3E2DDE
:100130005EACBD5913073F6401004242094403000D
:10014000063201451001400FC20E420152033280B7
:10015000C2014201C207021003520145900140183A
:100160004204023D0545A00140194206023D0745F3
:080170004001400D8201000076
:020000040001F9
:1004F000A5A54B4D0000001000000002AAAA5A7FDB
:10050000F0040100000000000200000000000000F4
:1005100000000000000000000000000000000000DB
:1005200000000000000000000000000000000000CB
:1005300088050100000000000A56656E646F7209AC
:100540003A204D4B53454D490A43686970093A209A
:100550004D4B383030300A44617465093A2041759A
:100560006720323720323032340A56657273696F31
:100570006E093A2056302E362E3200000000000060
:08058000000000000000000073
:04000005000000C136
:00000001FF
